:0800000C312E322E302E39375F
:1000000A5873795B9F947A559AA6AA8964A48267E1
:1000000A85886AAA9786896F949A729CA075838656
:1000000A7C7F7E83808480C7BBAD78CDC0CAAF8732
:1000000AC7B2B68B9B9394999D98989CA09B989DF8
:1000000AA7A8A3A8A3A3A7ABA6A3B1B1B3AEB3AE47
:1000000AAEB2B6B1AEB5BABDB9BEB9B9BDC1BCB969
:1000000ADCBEE0B1E7D6D9BFE4E4C2DCE0C50E024B
:0500000AF4BFF5E4E77E
:020000040800F2
:4080000080E30010B58D0708C78D070831C20808CB8D0708CD8D0708CF8D07080000000000000000000000000000000049830008D38D0708000000000D84000881840008F2
:40804000D98D0708D98D0708D98D0708D98D0708D98D0708D98D0708D98D0708D98D0708D98D0708D98D0708D98D07088926070893260708D98D07089F260708AB2607084A
:40808000B7260708C3260708130607084F0B0708630C0708D98D0708D98D0708D98D0708D98D0708D98D0708D98D0708D98D0708D56B0708E16B0708D98D0708D359070840
:4080C000E3590708F3590708FD5907087D6A0708876A07081F3C0708793C0708833C0708D98D0708D98D0708D98D0708D98D0708D98D0708D98D0708D98D0708CF2607084C
:40810000D98D0708D98D0708EB6B0708916A07088D3C0708973C0708D98D0708596D0708E9260708F3260708FF2607080B27070817270708D98D0708D98D0708090C0708CC
:40814000D70C07084D0D0708D98D0708D98D0708232707082F2707083B270708C53C0708075A0708175A0708D98D0708D98D0708D98D0708D98D0708D98D07080000000042
:40818000D98D0708D98D0708CF3C0708D93C07089B6A0708D98D0708D98D0708D98D07080000000000000000D98D070800F002F800F087F80AA090E8000C82448344AAF100
:4081C0000107DA4501D100F07CF8AFF2090EBAE80F0013F0010F18BFFB1A43F00103184764231700A42317000A444FF0000C10F8013B13F0070408BF10F8014B1D1108BFAD
:4082000010F8015B641E05D010F8016B641E01F8016BF9D113F0080F1EBF10F8014BAD1C0C1B09D16D1E58BF01F801CBFAD505E014F8016B01F8016B6D1EF9D59142D6D37C
:40824000704700000023002400250026103A28BF78C1FBD8520728BF30C148BF0B607047662909F04A89692901F0048A642901F0018A752901F0FE89782901F0378A6329B4
:4082800002F05D8A732902F0628A002070471FB589F0C5F89DE8030081F077FF81F053FC81F054FF04000020002188F08DF9401C60600020002188F09DF9E0601FBD10B508
:4082C00010BD82F051FE1146FFF7E1FF10F039F983F0ECF803B4FFF7F2FF03BC83F01CF980F309887047EFF309807047684680F3098804480078C00714BF0220032080F3B0
:4083000014887047286C0A08DFF818C0EFF305831B0618BF6047EFF31483DB0708BF604700DF704717F70808DFF818C0EFF305831B0618BF6047EFF31483DB0708BF60478E
:4083400000DF70471DF90808EFF30980816911F8021C01B142E010B590E80F10E047BDE81040EFF3098C254B93E80600914232D041B91EF0100F16D12149086820F0010043
:40838000086010E00CB41EF0100F06BF2CED108A0323012381F826302CE9F00FC1F82CC087F06EFE0CBC1A60D2F82CC0BCE8F00F92F8263013F0020F1ABFBCEC108A6FF042
:4083C000120E6FF0020E8CF3098813F0010F08BF704792F82500CCF80000704710B5094A1268914209D8084C54F8214090E80F10A047EFF3098C8CE80F0010BDB0100020B7
:4084000034EF00E020C2080820C2080810B587F0CFFCBDE81040194B93E80600914208BF70470CB4EFF3098C1EF0100F06BF2CED108A0223002381F826302CE9F00FC1F863
:408440002CC087F01DFE0CBC1A60D2F82CC0BCE8F00F92F8263013F0020F1ABFBCEC108A6FF0120E6FF0020E8CF3098813F0010F1CBF92F82530CCF800307047B01000207E
:4084800010B587F0CDFEC4E710B587F043F987F0C7FEBEE70B49D1F800C04A685CF8043B1068184442F8040B8C4528BFA1F1DC0C8A4228BFA1F1DC02C1F800C04A6020F0EA
:4084C0000040704774DD001010B5044620464DF0C3FF10BD07B588B00020069000210A98017008980078C32882F0F585810000BF794449688F4400000C0300001003000073
:4085000048030000D603000054040000D2040000FC0500006C060000DE2B0000E20600003C070000C6070000F2070000BC080000860900001A0B0000F00B0000460E0000B5
:40854000DE2B0000DE2B00000E0F00005C10000078100000DE10000044110000DE2B0000741200004A1300002E1400003C1600000A170000DC1700008218000050190000FE
:408580001E1A0000C41A0000461B0000201C0000401C00005C1C00000C1D00002C1D00006627000092270000C8270000DE2B0000DE2B00004C1D000024150000B015000014
:4085C0005E1D0000B61D0000F21D0000341E00008A1E0000C41E0000DE2B0000DE2B0000DE2B0000041F0000581F0000C61F0000C0200000DE200000DE2B0000DE2B0000B8
:40860000DE2B0000DE2B0000DE2B0000DE2B0000DE2B0000DE2B0000DE2B0000DE2B0000E0200000FA20000016210000500A0000041500006A210000AA110000DE2B0000DF
:408640007A21000014220000EE210000DE2B0000DE2B0000DE2B0000DE2B0000DE2B000096070000DE2B0000DE2B0000DE2B0000DE2B0000DE2B0000DE2B0000E41F000017
:40868000DE2B0000A2200000DE2B0000DE2B0000DE2B0000DE2B0000DE2B0000DE2B0000DE2B0000DE2B0000DE2B0000DE2B0000DE2B0000DE2B0000DE2B00002822000030
:4086C0003C220000DE2B00004E220000DE2B00006022000074220000882200009C220000B0220000C4220000D8220000EC220000DE2B0000DE2B0000002300004E230000B4
:40870000DE2B0000DE2B0000DE2B000050230000DE2B0000DE2B0000B60C0000800D0000DE2B0000B22300000E2400006A240000C62400002225000078250000CE250000EB
:40874000242600003C26000090260000E4260000DE2B0000DE2B0000DE2B000058270000DE2B0000DE2B0000DE2B0000DE2B0000DE2B0000DE2B0000DE2B0000DE2B0000AB
:40878000F827000012280000DE2B0000DE2B0000FC2600002E280000DE2B0000DE2B0000E22800001E2900003A2900006A290000922900000A2A00001E2A00003A2A0000E2
:4087C000DE2B0000DE2B0000DE2B0000DE2B0000DE2B0000DE2B0000DE2B0000DE2B00003C2A00005C2A0000702A0000DE2B0000902A0000142B0000DE2B0000DE2B000097
:408800006E2B000002F068BC13F0D5F818B101210A98017013E00898007A03280FD10898807A0490FE4890F8E0040390089800790290DDE903127EF07FFC0A990870E1E7DE
:4088400013F0B9F8F0BB0898007A03280CD10898807A04900898808880B2039004990CF0B6F80A99087031E00898007A012812D1EB48B0F88C130122099802FB001080B2C6
:4088800003900898807A0146049003980CF09FF80A9908701AE00898007A022816D1E048B0F88C130122099802FB101080B203900898807A0146049003980CF088F80A99FE
:4088C000087003E0FFE701210A9801709AE70898007A03280CD10898807A04900898808880B2039004997EF0CAFB0A9908702AE00898007A012811D17DF07DF90122099902
:4089000002FB010080B204900898807A0146039004987EF0B4FB0A99087014E00898007A022810D17DF067F90122099902FB110080B204900898807A0146039004987EF02E
:408940009EFB0A990870012006905BE70898007A03280CD10898807A04900898808880B2039004997EF0A4FB0A9908702AE00898007A012811D17CF0AAFD0122099902FBC4
:40898000010080B204900898807A0146039004987EF08EFB0A99087014E00898007A022810D17CF094FD0122099902FB110080B204900898807A0146039004987EF078FB2E
:4089C0000A990870012006901CE70898406842F2067188420AD00898406846F21E31884204D008984068491C884209D18D48007830B101201DF068FC0520FFF765FD76E0BA
:408A00000898007A03280DD1089890ED010AB8EEC00A8DED040A9DED040A0CF081F80A99087064E00898007A01282ED13DF0F9FCA8B97B48D0EDE60A9DED090AB8EE401AB5
:408A4000F7EE001AB0EE600A01EE810A8DED040A9DED040A0CF064F80A99087047E07048D0EDE60A9DED090AB8EE401ADFED6E1AB0EE600A01EE810A8DED040A9DED040AC3
:408A80000CF04EF80A99087031E00898007A02282DD13DF0C6FCA8B96148D0EDE60A9DED090AB8EE401AF7EE001AB0EE600A01EEC10A8DED040A9DED040A0CF031F80A991A
:408AC000087014E05648D0EDE60A9DED090AB8EE401ADFED551AB0EE600A01EEC10A8DED040A9DED040A0CF01BF80A9908700120069087E612F05FFF78BB0898007A0328DF
:408B000007D10898406804900BF0BCFF0A99087020E00898007A01280CD14148D0F890230121099801FB002004900BF0ABFF0A9908700FE00898007A02280BD13848D0F802
:408B400090130122099802FB101004900BF09AFF0A9908700120069003E0FFE701210A9801704FE612F027FF90BB0898007A032808D10898808880B204900BF0B3FF0A99F5
:408B8000087022E00898007A01280DD12448B0F894130122099802FB001080B204900BF0A1FF0A99087010E00898007A02280CD11B48B0F894130122099802FB101080B23C
:408BC00004900BF08FFF0A9908700120069003E0FFE701210A98017014E612F0ECFEE8B90898007A032819D10D4890F878130898406881420BD000200CF002F800200B49FA
:408C000008700B480978405C04900BF0DEFF0898007904900BF0C1FF0A990870F2E50000781A0010A40400205C8F22409F040020F03A090812F0BFFE00BB0898007A032812
:408C400024D10898007903900CF004FD04900BF0D7FF0A9908700020F94908700898007904900CF0F7FC172809D1F64890F87803401EC0B2059005980BF0A7FF06E0F24843
:408C8000EF490978405C04900BF09FFFBAE512F092FE98B90898007A03280FD10898406800280BDD08980079E5490870E6480978405C04900BF089FF0A990870A2E513F06D
:408CC000EDFC142810D013F0E9FC15280CD00898007A032808D10898807A049008980079039004990BF0A4FF8CE50898007A032812D1D44890F8E1040490D24890F8E004FF
:408D000003900898808800B20290DDE9031211F0F9FA0A9908704AE00898007A012821D1C84890F8E01400F5946000EB8101C54890F8E10431F810200121099801FB0020D7
:408D400000B20290BF4890F8E1040490BD4890F8E00403900146049A029811F0D3FA0A99087024E00898007A022820D1B54890F8E01400F5946000EB8101B24890F8E104CC
:408D800031F810100122099802FB101000B20290AC4890F8E1040490AA4890F8E00403900146049A029811F0ADFA0A9908700120069027E50898007A032812D1A14890F8C1
:408DC000E10404909F4890F8E00403900898808800B20290DDE9031211F0ABF80A9908704AE00898007A012821D1964890F8E01400F58C6000EB8101924890F8E10431F817
:408E000010100122099802FB001000B202908D4890F8E10404908B4890F8E00403900146049A029811F085F80A99087024E00898007A022820D1834890F8E01400F58C60DC
:408E400000EB81017F4890F8E10431F810100122099802FB101000B202907A4890F8E1040490784890F8E00403900146049A029811F05FF80A99087001200690C2E4089872
:408E8000007A032812D16F4890F8E10404906D4890F8E00403900898808800B20290DDE9031211F0A7F80A9908704AE00898007A012821D1634890F8E01400F58D6000EBE9
:408EC0008101604890F8E10431F810100122099802FB001000B202905A4890F8E1040490584890F8E00403900146049A029811F081F80A99087024E00898007A022820D1EE
:408F0000504890F8E01400F58D6000EB81014D4890F8E10431F810100122099802FB101000B20290474890F8E1040490454890F8E00403900146049A029811F05BF80A99CC
:408F40000870012006905DE40898007A032812D13C4890F8E10404903A4890F8E00403900898808800B20290DDE9031211F006FA0A9908704AE00898007A012821D1314898
:408F800090F8E01400F5936000EB81012D4890F8E10431F810100122099802FB001000B20290284890F8E1040490264890F8E00403900146049A029811F0E0F90A9908704E
:408FC00024E00898007A022820D11E4890F8E01400F5936000EB81011A4890F8E10431F810100122099802FB101000B20290154890F8E1040490134890F8E00403900146C5
:40900000049A029811F0BAF90A9908700120069015E40898007A032818D10A4890F8E1040490084890F8E00403900898808800B20290DDE9031211F03BF80A99087050E063
:409040009F040020781A0010F03A09080898007A012821D1FD4890F8E01400F58E6000EB8101FA4890F8E10431F810100122099802FB001000B20290F44890F8E1040490C0
:40908000F24890F8E00403900146049A029811F00FF80A99087024E00898007A022820D1EA4890F8E01400F58E6000EB8101E74890F8E10431F810100122099802FB1010D8
:4090C00000B20290E14890F8E1040490DF4890F8E00403900146049A029810F0E9FF0A9908700120069030E40898007A032810D1D64890F8E1040490D44890F8E00403902F
:409100000898808800B20290DDE9031211F046F84AE00898007A012821D1CC4890F8E01400F58F6000EB8101C84890F8E10431F810100122099802FB001000B20290C34803
:4091400090F8E1040490C14890F8E00403900146049A029811F022F80A99087024E00898007A022820D1B94890F8E01400F58F6000EB8101B54890F8E10431F81010012254
:40918000099802FB101000B20290B04890F8E1040490AE4890F8E00403900146049A029810F0FCFF0A990870012006900CE40898007A032812D1A54890F8E1040490A34882
:4091C00090F8E00403900898808800B20290DDE9031210F0A7FF0A9908704AE00898007A012821D1994890F8E01400F5916000EB8101964890F8E10431F810100122099881
:4092000002FB001000B20290904890F8E10404908E4890F8E00403900146049A029810F081FF0A99087024E00898007A022820D1864890F8E01400F5916000EB8101834874
:4092400090F8E10431F810100122099802FB101000B202907D4890F8E10404907B4890F8E00403900146049A029810F05BFF0A990870012006903CE40898007A032810D19A
:40928000724890F8E1040490704890F8E00403900898808800B20290DDE9031210F0BAFF4AE00898007A012821D1684890F8E01400F5926000EB8101644890F8E10431F89B
:4092C00010100122099802FB001000B202905F4890F8E10404905D4890F8E00403900146049A029810F096FF0A99087024E00898007A022820D1554890F8E01400F5926085
:4093000000EB8101514890F8E10431F810100122099802FB101000B202904C4890F8E10404904A4890F8E00403900146049A029810F070FF0A9908700120069011E40898D1
:40934000007A032811D1414890F8E10404903F4890F8E0040390089800790290DDE9031210F094FF0A9908704AE00898007A012821D1364890F8E01400F5906000EB810177
:40938000324890F8E10431F810100122099802FB001000B202902D4890F8E10404902B4890F8E00403900146049A029810F06EFF0A99087024E00898007A022820D12348D5
:4093C00090F8E01400F5906000EB81011F4890F8E10431F810100122099802FB101000B202901A4890F8E1040490184890F8E00403900146049A029810F048FF0A990870BA
:40940000012006900AE40898007A03287CD108984068F1280CD111F0EEFB0146049000200DF07BFC1420DFF828C000DF03DF8AE008984068F22811D10648D0F86801014636
:4094400004900220DFF810C000DF7CE0781A001021F808080019002081F8080808984068F32803D1032019F09BFA6CE008984068F7280AD1FE48D0F86801014604904FF4AC
:409480000070DFF8F0C300DF5DE008984068F42809D1F748D0F86801014604908020DFF8D4C300DF4FE008984068F5280AD1F048D0F86801014604904FF48070DFF8B4C3EC
:4094C00000DF40E008984068F62809D1E848D0F86801014604900120DFF898C300DF32E008984068F8280BD1E148D0F86801014604904FF48060DFF87CC300DF23E003E036
:4095000006210A9801701EE00898007A012809D1D748D0F86801014604900420DFF854C300DF10E00898007A022809D1D048D0F86801014604900820DFF838C300DF02E0CD
:4095400007210A9801701420FEF7BEFF0D2039F0BBFD2EE40898007A012802D1002019F01FFA1520FEF7B0FF272039F0ADFD20E40898007A032808D10898808800B204904F
:4095800008F027FE0A99087022E00898007A01280DD1B948B0F8E2140122099802FB001000B2049008F015FE0A99087010E00898007A02280CD1B048B0F8E2140122099809
:4095C00002FB101000B2049008F003FE0A9908700120069052E40898007A032808D10898808880B2049008F05CFE0A99087022E00898007A01280DD19F48B0F8EC14012239
:40960000099802FB001080B2049008F04AFE0A99087010E00898007A02280CD19648B0F8EC140122099802FB101080B2049008F038FE0A990870012006901FE40898007A00
:40964000032808D10898808880B2049008F051FE0A99087022E00898007A01280DD18648B0F8EE140122099802FB001080B2049008F03FFE0A99087010E00898007A022860
:409680000CD17D48B0F8EE140122099802FB101080B2049008F02DFE0A9908700120069051E40898007A032812D1734890F8E1040490714890F8E00403900898808800B297
:4096C0000290DDE9031208F0AEFD0A9908704AE00898007A012821D1674890F8E01400F2E44000EB8101644890F8E10431F810100122099802FB001000B202905E4890F88D
:40970000E10404905C4890F8E00403900146049A029808F088FD0A99087024E00898007A022820D1544890F8E01400F2E44000EB8101514890F8E10431F81010012209980F
:4097400002FB101000B202904B4890F8E1040490494890F8E00403900146049A029808F062FD0A9908700120069051E40898007A032814D10898807A04903F4890F8E1043B
:4097800003903D4890F8E004029008980079019002A90EC979F033FE0A9908704EE00898007A012823D1344890F8E01400F5737000EB4101304890F8E104095C0122099842
:4097C00002FB001001900898807A04902A4890F8E1040390284890F8E00402900146DDE90323019879F00BFE0A99087026E00898007A022822D1204890F8E01400F573706B
:4098000000EB41011C4890F8E104095C0122099802FB101001900898807A0490164890F8E1040390144890F8E00402900146DDE90323019879F0E3FD0A9908700120069086
:4098400051E40898007A03281BD10898807A0490094890F8E1040390074890F8E004029008980079019002A90EC979F08BFE05E00019002081F80808781A00100A99087034
:409880004EE00898007A012823D1FE4890F8E01400F5747000EB4101FA4890F8E104095C0122099802FB001001900898807A0490F44890F8E1040390F24890F8E004029063
:4098C0000146DDE90323019879F05CFE0A99087026E00898007A022822D1EA4890F8E01400F5747000EB4101E64890F8E104095C0122099802FB101001900898807A04902D
:40990000E04890F8E1040390DE4890F8E00402900146DDE90323019879F034FE0A9908700120069042E40898007A032814D10898807A0490D34890F8E1040390D14890F868
:40994000E004029008980079019002A90EC979F0BDFE0A9908704EE00898007A012823D1C84890F8E01400F5757000EB4101C54890F8E104095C0122099802FB00100190CD
:409980000898807A0490BF4890F8E1040390BD4890F8E00402900146DDE90323019879F095FE0A99087026E00898007A022822D1B44890F8E01400F5757000EB4101B148D7
:4099C00090F8E104095C0122099802FB101001900898807A0490AB4890F8E1040390A94890F8E00402900146DDE90323019879F06DFE0A990870012006903CE40898007A67
:409A000003280AD10898807A049008980079039004997AF030FC0A9908702CE40898007A032811D1089890ED010AF8EEC00AB2EE041A80EE810A8DED040A9DED040A7AF0A8
:409A4000B1FB0A9908702CE00898007A012812D17AF09CFC0122099902FB110000EE100AB8EEC00A8DED040A9DED040A7AF09AFB0A99087015E00898007A022811D17AF0E1
:409A800085FC0122099902FB010000EE100AB8EEC00A8DED040A9DED040A7AF083FB0A9908700120069049E40898007A032811D1089890ED010AF8EEC00AB2EE041A80EEB8
:409AC000810A8DED040A9DED040A7AF0ADFB0A9908702CE00898007A012812D17AF05FFC0122099902FB010000EE100AB8EEC00A8DED040A9DED040A7AF096FB0A99087026
:409B000015E00898007A022811D17AF048FC0122099902FB110000EE100AB8EEC00A8DED040A9DED040A7AF07FFB0A9908700120069067E40898007A032818D1089890EDA5
:409B4000010AF8EEC00AB2EE041A80EE810A8DED040A807A03904B4890F8E104029003999DED040A79F05CFE0A99087046E00898007A01281FD1434890F8E11400F577707D
:409B800000EB8100D0ED000A9DED090AB8EEC00A30EE800A8DED020A0898807A0490394890F8E104039004999DED020A79F038FE0A99087022E00898007A02281ED13148ED
:409BC00090F8E11400F5777000EB8100D0ED000A9DED090AB8EEC00A30EEC00A8DED020A0898807A0490274890F8E104039004999DED020A79F014FE0A9908700120069041
:409C0000A7E40898007A032818D1089890ED010AF8EEC00AB2EE041A80EE810A8DED040A807A0390174890F8E104029003999DED040A79F0E2FE0A99087048E00898007A8F
:409C4000012821D10F4890F8E11400F57B7000EB8100D0ED000A9DED090AB8EEC00A30EE800A8DED020A0898807A0490054890F8E104039004999DED020A79F0BEFE0A9931
:409C8000087024E0781A00100898007A02281ED1F74890F8E11400F57B7000EB8100D0ED000A9DED090AB8EEC00A30EEC00A8DED020A0898807A0490ED4890F8E1040390A6
:409CC00004999DED020A79F098FE0A990870012006903EE40898007A032810D10898807A0490E34890F8E1040390089800790290DDE903127AF02AF90A9908703AE00898D7
:409D0000007A012819D1DA4890F8E11400F20440415C0122099802FB001002900898807A0490D34890F8E10403900146049A02987AF00CF90A9908701CE00898007A02282F
:409D400018D1CB4890F8E11400F20440415C0122099802FB101002900898807A0490C44890F8E10403900146049A02987AF0EEF80A990870012006902CE40898007A0328F4
:409D800018D1089890ED010AF8EEC00AB2EE041A80EE810A8DED040A807A0390B44890F8E104029003999DED040A79F005FF0A99087046E00898007A01281FD1AC4890F88A
:409DC000E11400F5797000EB8100D0ED000A9DED090AB8EEC00A30EE800A8DED020A0898807A0490A24890F8E104039004999DED020A79F0E1FE0A99087022E00898007A58
:409E000002281ED19A4890F8E11400F5797000EB8100D0ED000A9DED090AB8EEC00A30EEC00A8DED020A0898807A0490904890F8E104039004999DED020A79F0BDFE0A991E
:409E40000870012006902BE40898007A032818D1089890ED010AF8EEC00AB2EE041A80EE810A8DED040A807A0390814890F8E104029003999DED040A79F074FF0A990870DF
:409E800046E00898007A01281FD1794890F8E11400F57D7000EB8100D0ED000A9DED090AB8EEC00A30EE800A8DED020A0898807A04906F4890F8E104039004999DED020AA3
:409EC00079F050FF0A99087022E00898007A02281ED1674890F8E11400F57D7000EB8100D0ED000A9DED090AB8EEC00A30EEC00A8DED020A0898807A04905D4890F8E1045E
:409F0000039004999DED020A79F02CFF0A9908700120069029E40898007A032810D10898807A0490524890F8E1040390089800790290DDE903127AF09FF80A9908703AE03E
:409F40000898007A012819D1494890F8E11400F20640415C0122099802FB001002900898807A0490424890F8E10403900146049A02987AF081F80A9908701CE00898007A23
:409F8000022818D13A4890F8E11400F20640415C0122099802FB101002900898807A0490334890F8E10403900146049A02987AF063F80A9908700120069041E40898007A49
:409FC00003280CD10898807A04900898808880B20390049978F0C9FE0A9908702CE00898007A012812D12248B0F80E140122099802FB001080B203900898807A0146049066
:40A00000039878F0B2FE0A99087015E00898007A022811D11648B0F80E140122099802FB101080B203900898807A01460490039878F09BFE0A9908700120069072E4089890
:40A04000007A032816D10898807A0490084890F8E1040390064890F8E004029008980079019002A90EC979F026F90A99087050E0781A00100898007A012823D1FB4890F8E7
:40A08000E01400F5767000EB4101F84890F8E104095C0122099802FB001001900898807A0490F24890F8E1040390F04890F8E00402900146DDE90323019879F0FCF80A99C6
:40A0C000087026E00898007A022822D1E74890F8E01400F5767000EB4101E44890F8E104095C0122099802FB101001900898807A0490DE4890F8E1040390DC4890F8E004A4
:40A1000002900146DDE90323019879F0D4F80A9908700120069005E40898007A03280AD10898807A049008980079039004997AF05AFA0A99087060E40898007A032808D1FF
:40A140000898807A0490089800790390049976F03DFE52E40898007A032813D10898807A04900898808880B200EE100AB8EE400A8DED030A04989DED030A76F006FB0A99A4
:40A1800008703CE00898007A01281AD177F062F8F0EE400AB64890ED851A9DED090AF8EE401AB0EE410A00EEA10A8DED040A0898807A03909DED040A76F0E7FA0A990870CC
:40A1C0001DE00898007A022819D177F043F8F0EE400AA74890ED851A9DED090AF8EE401AB0EE410A00EEE10A8DED040A0898807A03909DED040A76F0C8FA0A99087001200F
:40A2000006900AE40898007A03280AD10898807A049008980079039004997CF0D0FD0A99087040E40898007A03280AD10898807A049008980079039004997CF04AFE0A999D
:40A24000087030E40898007A032803D1089800798849087027E40898007A03281DD1834890F8E11400F5777000EB810090ED000A8DED070A9DED070AB5EEC00AF1EE10FA06
:40A2800003D19FED7D0A8DED070A4FF0FF319DED070A082075F04AF808E00898007A28B900219FED760A082075F040F841E40898007A03280FD17AF069F800EE100AB8EEBB
:40A2C000C00A8DED040A6FF009019DED040A0A2075F02CF808E00898007A28B900219FED670A082075F022F823E40898007A032812D15E4890F8E11400F57B7000EB810012
:40A3000090ED000A8DED040A6FF001019DED040A082075F00BF808E00898007A28B900219FED560A082075F001F869E40898007A03281CD14D4890F8E11400F5797000EBB5
:40A34000810090ED000A8DED070A9DED070AB5EEC00AF1EE10FA03D19FED490A8DED070A01219DED070A082074F0E0FF08E00898007A28B900219FED410A082074F0D6FFB7
:40A380003EE40898007A03280ED17AF008F800EE100AB8EEC00A8DED040A0A219DED040A084674F0C3FF08E00898007A28B900219FED320A082074F0B9FF21E40898007A87
:40A3C000032811D1294890F8E11400F57D7000EB810090ED000A8DED040A02219DED040A082074F0A3FF08E00898007A28B900219FED220A082074F099FF6AE40898007AD4
:40A40000032807D108980079049017F031FF0A9908701CE00898007A01280AD1134890F87805401CC0B2049017F022FF0A9908700DE00898007A022809D10C4890F8780597
:40A44000401EC0B2049017F013FF0A99087040E40898007A032831D10898406890B9034890F8C803049009F08BFF27E0781A0010B01D0010D5010010CDCCCCBD0000000005
:40A48000CDCCCC3D08984068012806D1F74890F8C803049009F0B0FE10E008984068022802D109F0A8FC09E008984068032805D1EE4890F8C803049009F08DFD09E40898B4
:40A4C000007A032809D108980079049005F09FFC0A990870042006F0F6FA4DE40898007A032859D108984068062846D2DFE800F0030E19242F3A012005F0FFFB0A990870B4
:40A50000002005F0E4FB0A99087041E0032005F0F4FB0A990870852005F0D9FB0A99087036E0032005F0E9FB0A990870872005F0CEFB0A9908702BE0032005F0DEFB0A99F4
:40A5400008708A2005F0C3FB0A99087020E0042005F0D3FB0A990870782005F0B8FB0A99087015E0042005F0C8FB0A9908707E2005F0ADFB0A9908700AE0012005F0BDFB94
:40A580000A990870002005F0A2FB0A99087000BF00BF402006F097FA55E40898007A032809D108980079049005F0BCFC0A990870802006F088FA46E40898007A032809D120
:40A5C00008980079049005F084FC0A990870022006F079FA37E436E40898007A032807D13C21A3487FF041FC6CF062FBA049086329E40898007A032808D19E48D0F86801FE
:40A60000014604900220DFF870C200DF1BE434F060FC0899897A88420FD1984890F8D00008B9012000E00020049001F01AFB94480078A8B11BF059FE12E008984068012842
:40A6400008D1002001F00DFB8D48007840B11BF04CFE05E00898406810B9012001F001FB58E40898007A012802D1022011F0BCFC50E40898007A03280DD1089890ED010AA5
:40A68000B8EEC00A8DED040A9DED040A05F064FB0A99087026E00898007A01280FD1794890ED020AF7EE000A30EE200A8DED040A9DED040A05F050FB0A99087012E00898E4
:40A6C000007A02280ED16F4890ED020AF7EE000A30EE600A8DED040A9DED040A05F03CFB0A99087016E40898007A03280DD10898807A0490089800790390049978F090FA33
:40A700000898007904900FF0B4F856E40898007A032804D106F07CFB202006F0D4F94CE40898007A032804D108980079049006F025FD42E40898007A032803D10898007996
:40A74000514908701FE20898007A032803D1089800794E49087016E20898007A032804D108984068049005F014F90CE20898007A032804D108980079049006F0D6F902E237
:40A780000898007A032804D108980079049006F0F2F9F8E10898007A032804D108980079049006F00EFAEEE10898007A032804D108980079049006F02AFAE4E10898007AC4
:40A7C000032804D108980079049006F046FADAE10898007A032804D108980079049006F062FAD0E10898007A032804D108980079049006F07EFAC6E10898007A032821D1DE
:40A8000008984068052818D2DFE800F003070B0F1300002006F077FC13E0012006F073FC0FE0022006F06FFC0BE0032006F06BFC07E0042006F067FC03E0002006F063FC30
:40A8400000BF00BF9FE19EE10898007A03282BD1064890F8E00401281AD10898807A01460490002009F080FA19E00000781A0010102800100019002081F80808A8170010D0
:40A88000403E0010B0210010AD040020AE0400200898807A01460490012009F065FA00214FF4807018F047F86DE10898007A032809D10898808880B20121049064F070FC40
:40A8C0000A9908701EE00898007A01280BD1FB48B0F85A07401C80B20121049064F060FC0A9908700EE00898007A02280AD1F348B0F85A07401E80B20121049064F050FC8E
:40A900000A990870E8E30898007A032809D10898808880B20121049064F076FC0A9908701EE00898007A01280BD1E448B0F85C07401C80B20121049064F066FC0A99087038
:40A940000EE00898007A02280AD1DC48B0F85C07401E80B20121049064F056FC0A990870BAE30898007A032809D10898808880B20121049064F07CFC0A9908701EE00898C3
:40A98000007A01280BD1CD48B0F85E07401C80B20121049064F06CFC0A9908700EE00898007A02280AD1C548B0F85E07401E80B20121049064F05CFC0A9908708CE3089898
:40A9C000007A032809D10898808880B20121049064F082FC0A9908701EE00898007A01280BD1B648B0F86007401C80B20121049064F072FC0A9908700EE00898007A0228DE
:40AA00000AD1AE48B0F86007401E80B20121049064F062FC0A9908705EE30898007A032808D10898808880B2049064F089FC0A9908701CE00898007A01280AD19F48B0F8B9
:40AA40006207401C80B2049064F07AFC0A9908700DE00898007A022809D19848B0F86207401E80B2049064F06BFC0A99087033E30898007A032808D10898808880B20490CE
:40AA800064F08BFC0A9908701CE00898007A01280AD18A48B0F86407401C80B2049064F07CFC0A9908700DE00898007A022809D18248B0F86407401E80B2049064F06DFCCF
:40AAC0000A99087008E30898007A032808D10898808880B2049064F08DFC0A9908701CE00898007A01280AD17448B0F86607401C80B2049064F07EFC0A9908700DE0089849
:40AB0000007A022809D16D48B0F86607401E80B2049064F06FFC0A990870DDE20898007A032806D108980079049064F08EFC0A990870D1E20898007A032807D10898007965
:40AB4000049064F0ADFC0A9908701CE00898007A01280AD1594890F86907401CC0B2049064F09EFC0A9908700DE00898007A022809D1524890F86907401EC0B2049064F0B6
:40AB80008FFC0A990870A7E20898007A032807D108980079049064F0AEFC0A9908701CE00898007A01280AD1444890F86A07401CC0B2049064F09FFC0A9908700DE00898EB
:40ABC000007A022809D13D4890F86A07401EC0B2049064F090FC0A9908707DE20898007A032806D108980079049064F0AFFC0A99087071E20898007A032809D1089880889E
:40AC000080B20121049064F0DCFC0A9908701EE00898007A01280BD12848B0F86C07401C80B20121049064F0CCFC0A9908700EE00898007A02280AD12048B0F86C07401ED4
:40AC400080B20121049064F0BCFC0A99087043E20898007A032801D110F0F0FF3CE20898007A032810D10898807A0490089890ED010AB8EEC00A8DED030A04989DED030AD6
:40AC80007AF01FFF0A99087026E20898007A032812D10898807A04900898808880B200EE100AB8EE400A8DED030A04989DED030A7AF0EDF90A9908700EE20000781A00100A
:40ACC0000898007A032812D10898807A04900898808880B200EE100AB8EE400A8DED030A04989DED030A7AF02CFB0A990870F3E10898007A032805D1089800790121049008
:40AD000005F085F904F0EBF8E6E10898007A032808D10898807A0490089800790390049977F03CFAD8E10898007A032815D1089890ED010AF8EEC00A9FEDFE1A80EE810A77
:40AD40008DED040AFC4890F8E00403909DED040A0EF014FF0A9908703EE00898007A01281BD1F54890F8E01400F5F26000EB8100D0ED000A9DED090AB8EEC00A30EE800A0F
:40AD80008DED030AEC4890F8E00404909DED030A0EF0F4FE0A9908701EE00898007A02281AD1E54890F8E01400F5F26000EB8100D0ED000A9DED090AB8EEC00A30EEC00AF1
:40ADC0008DED030ADC4890F8E00404909DED030A0EF0D4FE0A9908707EE10898007A032818D1D54890F8E104012807D10898807A0146049000200AF04FFE06E00898807AB2
:40AE00000146049001200AF047FE00214FF4807017F091FD60E10898007A032808D10898807A0490089800790390049909F062FB52E10898007A032812D1089840680128F6
:40AE400004D0022805D0032809D105E029F032FE05E029F050FE02E029F098FE00BF00BF3AE10898007A03280ED1089890ED010AB8EEC00ADFEDB10A20EE200A8DED040A53
:40AE80009DED040A29F056FE26E10898007A032836D10898406808282DD2DFE800F004090E13181D22274FF4966004F0E9FF22E04FF4166004F0E4FF1DE04FF4965004F09F
:40AEC000DFFF18E04FF4165004F0DAFF13E04FF4964004F0D5FF0EE04FF4164004F0D0FF09E04FF4614004F0CBFF04E04FF4E13004F0C6FF00BF00BF4FF4804005F0E3FD16
:40AF0000EAE00898007A032804D108980079049006F0F6F9E0E00898007A032808D10898807A049008980079039004997CF003FCD2E0D1E00898007A03280AD1089890ED3B
:40AF4000010AB8EEC00A8DED040A9DED040A00F0E9FEC1E00898007A032804D10898007904900FF0FAFFB7E00898007A03280AD108980079049005F0BAFF0A9908704FF48F
:40AF8000007005F0A0FDA7E010F015FD18BB10F039FD00BB10F029FDE8B910F019FDD0B90898007A032805D108980079049006F0A4FC2AE00898007A012811D15E4890F811
:40AFC0009907042808DA5C4890F89907401CC0B2049006F092FC18E0012006F08EFC14E00898007A022810D1534890F89907012808DD514890F89907401EC0B2049006F053
:40B000007CFC02E0042006F078FC65E00898007A032806D10898007940B2049029F093FE20E00898007A01280CD1434890F89A0741B20122099802FB001040B2049029F047
:40B0400082FE0FE00898007A02280BD13A4890F89A0741B20122099802FB101040B2049029F071FE38E00898007A032809D10898807A049008984068039004990AF034FEAB
:40B0800026E00898007A01280FD12B48B0F882170122099802FB001003900898807A0146049003980AF020FE12E00898007A02280ED12148B0F882170122099802FB101087
:40B0C00003900898807A0146049003980AF00CFE0120069000E000BF00BF089800780490FDF7F2F906980BB000BD86B04FF6FF7438211348DFF84CC000DF0221124880F89A
:40B1000044110C228421114884F018FA00287BD103210D4880F8441100BF224605A90848DFF82CC000DF01285ED000208DF8000010E0000000007A44781A00106F12833AFD
:40B140004C11002009FA080800190020C810002099FB08088DF80D0001208DF80C0000208DF80E0005980078002838D004AA01210598FDF7AFF905469DF8100068B10025F7
:40B18000059908783CF0CCF906460598C37A827A9DF8101030463CF073FA10F00CFC08B1002504E00598007A032800D10025B5B19DF80D0098B90598007A80B1059A07CA87
:40B1C0008DE8070001208DF80D008DF80C004FF47A649DF80E00401CC0B28DF80E008D480599FDF7A1F898E79DF80000002894DD9DF80E0000283DDD9DF80E00032804D135
:40B2000002208DF80C000FE037E09DF80E00052803D106208DF80C0006E09DF80E00072802D110208DF80C009DF80E00FF2805DA9DF80E00401CC0B28DF80E009DF80C1050
:40B2400004AA6846FDF746F99DF8100078B100208DF80E00059908783CF062F906460598C37A827A9DF8101030463CF009FA4FF4FA6452E74FF6FF744FE70521664880F889
:40B2800044110020DFF894C100DF00BFFEE770B50023002100BF06E0614830F82100184383B2481CC1B20729F6DB002B55D05C48001F0078401C5A4A121F107010460078F8
:40B2C000C62801DD002010700CE05548001F0078401C534A121F107010460078C62801DD002010704E4C241F2278D41702EBD46465114B4C54F82540494D2D1F2878C5173B
:40B3000000EBD5656D11A0EB45160125B5402C40002CDAD0424C241F2078C41700EBD46465113F4C54F825403D4D2D1F2A78D51702EBD5656D11A2EB45160125B540AC4313
:40B34000374D2D1F2878C51700EBD5656E11344D45F82640281F007870BD0020FCE72DE9F04705460E4617469846DDF820904FF0010A2C48DFF8B0C000DFD0B900BF264884
:40B3800090F8450140F00201234880F84511B0F850014FF6FF71884207DA1F48B0F85001401C81B21C48A0F8501100BF4FF0000A2CE01848FCF7A8FF04466CB125706660DE
:40B3C000277284F80A8084F80B900A2221461548DFF858C000DF19E000BF0F4890F8450140F004010C4880F84511B0F850014FF6FF71884207DA0848B0F85001401C81B274
:40B400000548A0F8501100BF4FF0000A5046BDE8F0870000C8100020001900203D030908881100204C11002001FA0808F5FA08080020FE490870704710B5FD48007840B141
:40B440004FF47A71FB4800686BF04CFC08B9012010BD0020FCE710B5FFF7EEFF10B1F648007810BDF5480078FBE710B50446F04804706BF01DFCEF49086010BD31B52DED7F
:40B48000040B2DED028BB0EE408A0446FFF7D4FF10B3EA480078E8490978884214D0E848007820B9E748DDE9031206C00CE094ED000ADFEDE50AB4EEE00AF1EE10FA03DDB6
:40B4C000DD480078DD490870DC480078DA4909784840DB4908706EE00020FFF7C6FF1AF054FE022864D0D648007820BBB0EEC80AD648D0ED000AB4EEE00AF1EE10FA5ADD58
:40B500001AF043FE08B1012000E00020D049087008460078C9490978884204D0CC480078C649087047E0C748DDE9031206C00120C34908703FE094ED000ADFEDC30AB4EEEA
:40B54000E00AF1EE10FA13DDB0EEC80ABF48D0ED000AB4EEE00AF1EE10FA05DDB748007880F00100B54908700020B549087022E0B0EEC80AB548D0ED000AB4EEE00AF1EEDE
:40B5800010FA18DD1AF001FE08B1012000E00020AF49087008460078A849097888420AD0AB480078A54908700020A549087002E00020A2490870BDEC028B05B030BDF0EEEB
:40B5C000401AB0EE610A71EEE02AB0EE622AF0EEC22A9FEDA03AF4EEC32AF1EE10FA17D2B1EE003A21EE033AF0EE432AB7EE003AF4EEC32AF1EE10FA03DDB7EE003AF0EEE0
:40B60000432AB0EE603A02EE223AB0EE430A00BF7047F3B52DED040B2DED108B8BB00546F0EE41AA0C468C480078A84202D1B4F5FA7F0BD98848057000207C490870874910
:40B6400008700BB0BDEC108B06B0F0BD7748007850BB9FED830A834880ED000A9FED800A814880ED000A7748DDE91B1206C07F48DDE91B1206C0002078490870704908707B
:40B680007B4908709FED760A7A4880ED000A9FED740A794880ED000A0120644908706BF007FB64490860CCE79DED1C0A6F48D0ED010A30EE609A9DED1B0AD0ED000A70EE41
:40B6C000608A29EE090A08EEA80A10EE101A084685F034FE41EC1C0BB0EE4C0AF0EE6C0A83F0D2F8B0EE40BAF0EE60BA51EC1B0B84F0A2FF09905148007810B19FED5F0A30
:40B7000001E09FED5F0AF0EE40DA9DED090AB4EEED0AF1EE10FA45D2564890ED000ADFED590AB4EEE00AF1EE10FA20DD5248D0ED000A504890ED001AC0EE811AB0EE610A5D
:40B740004D4890ED001A00EE904AF8EE600A00EE601A80ED001A474890ED001A00EE904AF8EE600A71EE600AC0ED000A00BF1AF0ECFCF0EE400A00EE104AB8EE401A3E4831
:40B7800090ED000A00EE810A80ED000A3948D0ED000A00EE104AB8EE400A30EE800A80ED000A4EE72648007850B39DED1C0A2548D0ED010A30EE600AB0EE409A9DED1B0AC1
:40B7C000D0ED000A30EE600AF0EE408A29EE090A08EEA80A10EE101A084685F0AFFD41EC1C0BB0EE4C0AF0EE6C0A83F04DF8B0EE40BAF0EE60BA51EC1B0B84F01DFF099079
:40B80000B0EEC90ADDED090A80EE201AB0EE41BAB0EE4B0A1EF056F9B0EE408AB5EEC09AF1EE10FA3ADBF5EEC08A2DE00C00001004000010080000102300001021000010E0
:40B8400020000010280000109A99993EE06B0A08220000103333B33E300000100D000010000000001000001014000010180000102400001038000010340000109A99193E5D
:40B88000CDCCCC3D0000FA43F1EE10FA06D2F94890ED000A30EE480AB0EE408AB5EEC09AF1EE10FA0BD2F5EEC08AF1EE10FA06D2F04890ED000A30EE080AB0EE408AB5EE9D
:40B8C000C09AF1EE10FA0BD2F5EEC08AF1EE10FA06DBE94890ED000A30EE480AB0EE408A03F069FE8DED080AE448007820B19DED080AB1EE400A01E09DED080AB0EE40AABC
:40B900009FEDDF0AB4EEC0AAF1EE10FA0AD29DED091ADC48D0ED000AB0EE480AFFF74FFEB0EE408AD74880ED008AD7480078A8BBD648D74A06CA06C0D548DDE91B1206C0D3
:40B940001AF003FCF0EE400A00EE104AB8EE400A9FEDD01AC0EE011A20EEA10AB0EE40BA9DED080A6BEE000A9DED091A80EE810A38EE400AC84880ED000AC24880ED008A31
:40B980001FED490AC54880ED000A1FED4B0AC44880ED000A0120BC49087052E6FFE7BE4890ED00DA78EE4D9AB24890ED000AF4EEC09AF1EE10FA06DDAF4890ED000A39EE2C
:40B9C000C00AF0EE409AAB4890ED000AB1EE400AF4EEC09AF1EE10FA06D2A74890ED000A39EE800AF0EE409AA448067809A89DED1C1ADDED1B0AB0EE690AFFF73FFDA4488D
:40BA0000DDE91B1206C0A748007850B11FED6C0AA24880ED000A1FED6E0AA14880ED000A0FE696480078864249D09F48007840B9904890ED000A3AEE800A974880ED000A33
:40BA400002E0954880ED008A934890ED000A8A48D0ED000AB4EEE00AF1EE10FA0ADD8E4890ED000A8448D0ED000A30EE600A8A4880ED000A884890ED000AB5EEC00AF1EE55
:40BA800010FA09D290ED000A7B48D0ED000A30EE200A814880ED000A1FED8F0A7F4880ED000A1FED910A7E4880ED000AFFF7D3FC07461AF06DFB00207B490870C1E59FED2F
:40BAC000700AB4EEC0AAF1EE10FA24D21AF03DFBF0EE400A00EE104AB8EE401A704890ED000A00EE810ADFED6B0A80EE201AB0EE41BADDED090A8AEE200A20EE0B0AB0EEB5
:40BB000040BAB0EE4B0A1DF0DDFF38EE400A624880ED000A3AE01AEE100A85F00FFCCDE9060119EE900A85F009FCCDE900019DED000B82F07DFD8DED040B099885F0FEFB3A
:40BB4000CDE902019DED040B53EC102B9DED020B51EC100B85F0FCF841EC1C0B9DED060B53EC102B84F056FE41EC1B0B4A48006885F0E4FB41EC1E0B53EC1B2B84F08EFDF5
:40BB800041EC1F0B84F058FD434908601FEDCC0A434880ED000A1FEDCE0A404880ED000A0AE03D4890ED000A3348D0ED000A30EE600A394880ED000A374890ED000A2E4876
:40BBC000D0ED000AB4EEE00AF1EE10FAE9DC0AE0314890ED000A2848D0ED000A30EE200A2D4880ED000A2C4890ED000AB5EEC00AF1EE10FAECD300BF23E5244991ED010A22
:40BC0000D0ED010A30EE200A81ED010A91ED000AD0ED000A30EE200A81ED000A1C4991ED010AD0ED010A30EE200A81ED010A91ED000AD0ED000A30EE200A81ED000A70472F
:40BC4000154890ED000A704710B5FFF7F5FB28B10A48007815490978484010BD11480078FBE770B50446FFF7E7FB08B30F480578047024E0E46B0A08EC6B0A0821000010AB
:40BC8000CDCCCC3E140000100D000010280000101800001000007A441000001038000010340000102000001024000010230000101E480578047085EA04001D49087070BD6A
:40BCC0001C48007828B11C48007810B11B48007808B1012070470020FCE710B5FFF7BBFB20B9FFF7EDFF08B9012010BD0020FCE71048007820B11048007808B101207047A3
:40BD00000020FCE70E490870704710B5FFF7A3FB08B1002400E00124204610BD094890ED000A7047074880ED000A704721000010240000100C0000100D0000102000001032
:40BD4000230000100000001008B560212E48DFF8BCC000DF02212E4880F808114FF4367243F6EC012B4883F0E9FB002841D10321274880F8081100BF4FF47A726946224830
:40BD8000DFF894C000DF0128F6D0214890F840000328F1D1214890F84F030A2824D00098007805281ED2DFE800F003070C101400009820F0E1FD16E00098B03027F030FDAD
:40BDC00011E0009827F026FF0DE0009825F09CFC09E068F065FD044601220099B03167F07CFC00E000BF00BF0A480099FCF79CFAC2E70521064880F808110020DFF820C09C
:40BE000000DF00BFFEE7000064B9002009FA0808001900207880002099FB0808781A00103D0309080048704760E3022010B57EF08DF9001D10BD00BF9147080000000000A1
:40BE40000000000000000000000000000000000000000000000000000000000000000000000000000000000000000000526176656E20496E647573747269657320496E6342
:40BE80000000000000000000000000004175672D31382D323031380000000000312E322E302E39370000000000000000526176656E2047756964616E636520436F6E7472E8
:40BEC0006F6C6C6572000000000000003037373031373134343900000000000000000000000000000000000000000000FFFFFFFFFFFFFFFFFFFFFFFFFFFFFFFFFFFFFFFF30
:40BF0000FFFFFFFFFFFFFFFFFFFFFFFFFFFFFFFFFFFFFFFFFFFFFFFFFFFFFFFFFFFFFFFFFFFFFFFFFFFFFFFFFFFFFFFFFFFFFFFFFFFFFFFFFFFFFFFFFFFFFFFFFFFFFFFF41
:40BF4000FFFFFFFFFFFFFFFFFFFFFFFFFFFFFFFFFFFFFFFFFFFFFFFFFFFFFFFFFFFFFFFFFFFFFFFFFFFFFFFFFFFFFFFFFFFFFFFFFFFFFFFFFFFFFFFFFFFFFFFFFFFFFFFF01
:40BF8000FFFFFFFFFFFFFFFFFFFFFFFFFFFFFFFFFFFFFFFFFFFFFFFFFFFFFFFFFFFFFFFFFFFFFFFFFFFFFFFFFFFFFFFFFFFFFFFFFFFFFFFFFFFFFFFFFFFFFFFFFFFFFFFFC1
:40BFC000FFFFFFFFFFFFFFFFFFFFFFFFFFFFFFFFFFFFFFFFFFFFFFFFFFFFFFFFFFFFFFFFFFFFFFFFFFFFFFFFFFFFFFFF00C00008FFFF170800800008FBBF000828763B4E17
:40C00000012904D002290BD003291BD111E042F2107242436423B2FBF3F2FE4B1A8012E042F2107242436423B2FBF3F2FA4B1A8009E042F2107242436423B2FBF3F2F74B18
:40C040001A8000E000BF00BF704710B50446F44800882044F24908800846008842F21071884202DB0020EE490880ED480088E9490988884205DA0121EA48007868F009F8B8
:40C0800004E00021E748007868F003F8E4480088E1490988884205DA0121E348007867F0F8FF04E00021E048007867F0F2FFDC480088DA490988884205DA0121DB480078A3
:40C0C00067F0E7FF04E00021D848007867F0E1FF10BD70B505466AF0EBFD04460020D44988614FF47A71D248C1614462002180F8281003210020FFF783FF0020CC49C86244
:40C100004FF47A71CA4801638463002180F83C1002210020FFF774FF0020C54948604FF47A71C348816004610021017501210020FFF766FF0020BE4908644FF47A71BC4895
:40C140004164C464002180F850100020B84948654FF47A71B64881650466002180F86410122D7DD2DFE805F009233D569CC1F1EFEEEDECEBEAE9E8E7E6E54FF4FA70AC499B
:40C1800088610146AA48C1614462012180F82810014691ED080ABCEEC00A10EE101A88B20321FFF72DFF0120A149087007E34FF4FA709F49C86201469D480163846301210B
:40C1C00080F83C10014691ED0D0ABCEEC00A10EE101A88B20221FFF713FF012094490870EDE24FF4FA7092494860014690488160046101210175014691ED030ABCEEC00AE6
:40C2000010EE101A88B20121FFF7FAFE012088490870D4E202208649087032204860322183488160046100210175014691ED030ABCEEC00A10EE101A88B20121FFF7E0FE70
:40C240004FF4FA607A4948650021794881650466012180F864100020FFF7D2FE032100E0ACE20020FFF7CCFE02210020FFF7C8FE02206F4981F8680002216D4880F8691096
:40C2800080F86A1080F86B1080F86C10042180F86D10062180F87710002180F878108EE24FF4FA7062490864014661484164C464012180F85010014691ED080ABCEEC00A0E
:40C2C00010EE101A88B20321FFF79AFE584991ED030ABCEEC00A10EE101A88B20121FFF78FFE01205249087069E264205049086464214F484164C464012180F85010014651
:40C3000091ED080ABCEEC00A10EE101A88B20321FFF776FE464991ED030ABCEEC00A10EE101A88B20121FFF76BFE01204049087045E213E2E1E1AFE169E123E1BDE0EEE04F
:40C3400086E04FE035E01AE0FFE74FF47A703849886100213648C1614462012180F82810014691ED080ABCEEC00A10EE101A88B20321FFF745FE01202D4908701FE24FF406
:40C380007A702B49C8620021294801638463012180F83C10014691ED0D0ABCEEC00A10EE101A88B20221FFF72BFE01202049087005E24FF47A701E49486000211C488160B3
:40C3C000046101210175014691ED030ABCEEC00A10EE101A88B20121FFF712FE012014490870ECE14FF47A7011490864002110484164C464012180F85010014691ED080AA3
:40C40000BCEEC00A10EE101A88B20321FFF7F8FD07490FE002000020040000200600002008000020EA03001004040010EB030010A411002091ED030ABCEEC00A10EE101A35
:40C4400088B20121FFF7DCFD0120FE490870B6E10220FC4908704FF4FA7088610021F948C161446280F82810014691ED080ABCEEC00A10EE101A88B20321FFF7C1FD4FF403
:40C48000FA70F049C8620021EE4801638463012180F83C1002210020FFF7B2FD0120E94981F868000021E74880F86910022180F87710002180F8781081E10220E149087061
:40C4C0004FF4FA7088610021DE48C161446280F82810014691ED080ABCEEC00A10EE101A88B20321FFF78CFD4FF4FA70D54948600021D44881600461017501210020FFF7F3
:40C500007FFD0120CF4981F868000221CD4880F8691080F87710002180F878104FE10220C84908704FF4FA70C8620021C54801638463012180F83C10014691ED0D0ABCEE85
:40C54000C00A10EE101A88B20221FFF759FD4FF4FA70BC4948600021BA4881600461017501210020FFF74CFD0020B64981F868000221B44880F8691080F87710002180F8BE
:40C5800078101CE10220AF4908704FF4FA7088610021AC48C1614462012180F82810014691ED080ABCEEC00A10EE101A88B20321FFF726FD4FF4FA70A249C8620021A14869
:40C5C0000163846380F83C1002210020FFF718FD4FF4FA709B49486000219A4881600461017501210020FFF70BFD0120954981F868000021934880F86910022180F86A10C4
:40C60000032180F87710002180F87810D7E002208C49087040F24D10886100218948C1614462012180F82810014691ED080ABCEEC00A10EE101A88B20321FFF7E1FC40F2B6
:40C640004D108049C86200217E480163846380F83C1002210020FFF7D3FC40F24D10794948600021774881600461017501210020FFF7C6FC0120734981F868000021714845
:40C6800080F86910022180F86A10032180F87710002180F8781092E002206A4908704FF4FA70886100216748C161446280F82810014691ED080ABCEEC00A10EE101A88B2E6
:40C6C0000321FFF79DFC4FF4FA705E49086400215C484164C464012180F850100120594981F868000321574880F86910022180F87710002180F8781061E00220514908702B
:40C700004FF4FA70C86200214E480163846380F83C10014691ED0D0ABCEEC00A10EE101A88B20221FFF76CFC4FF4FA7045490864002144484164C464012180F850100020EE
:40C74000404981F8680003213E4880F86910022180F87710002180F8781030E00220394908704FF4FA70486000213648816004610175014691ED030ABCEEC00A10EE101A27
:40C7800088B20121FFF73CFC4FF4FA702D49086400212C484164C464012180F850100220284981F868000321264880F86910022180F87710002180F8781000E000BF00BF6C
:40C7C0002148057070BD20B1012806D002280CD107E01C4981ED0D0A08E01A4981ED080A04E0184981ED030A00E000BF00BF0121164A1170704770B5002515480078E0B92B
:40C80000802110487DF031FB9FED120A0020FFF7DAFF9FED110A0220FFF7D5FF9FED0D0A0120FFF7D0FF0020064981F879000220FFF74FFC0120064908706AF039FA044630
:40C8400000480BE0A411002000000020010000200A0000200000A0420000C84290F87900002845D167F09BFBFF280ED1FD480078022803D1FC480078012805D10220FFF799
:40C8800028FC0020F84908709BE001202AF0E2F870B9F4480078052803D1F34800780128F2D10520FFF715FC0020EF49087088E001F0E1FE70B1EB480078042803D1EA483C
:40C8C000007801287DD10420FFF703FC0020E649087076E0E348007818B9E348007801286FD10020FFF7F5FB0020DF49087068E0DE4890F8790001280ED1DA4800780E2886
:40C9000003D1D948007801285BD10E20FFF7E1FB0020D549087054E0D44890F87900022815D1D249C86F4FF47A616AF0DBF970B9CC480078082803D1CB480078012840D102
:40C940000820FFF7C6FB0020C749087039E0C74890F87900042815D1C449C86F4FF47A616AF0C0F970B9BF480078072803D1BE480078012825D10720FFF7ABFB0020BA4952
:40C9800008701EE0B94890F87900032815D1B749C86F4FF47A616AF0A5F970B9B1480078062803D1B048007801280AD10620FFF790FB0020AC49087003E00020AB4981F8ED
:40C9C0007900AA480078012802D002287DD1F9E0A64890F83C00E0B9A448C06AC8B1A348816B20466AF0AEF9A049096B88422AD301219E4880F83C108463014691ED0D0A3D
:40CA0000BCEEC00A10EE101A88B20221FFF7F8FA19E0964890F83C00012814D19348006B88B19248816B20466AF08CF98F49C96A884208D300218D4880F83C10846302216E
:40CA40000020FFF7DDFA8948007DD8B987484068C0B18648016920466AF074F983498968884227D30121814801750461014691ED030ABCEEC00A10EE101A88B20121FFF796
:40CA8000BFFA17E07948007D012813D17748806880B17648016920466AF054F973494968884207D3002171480175046101210020FFF7A6FA6D4890F82800F0B96B48806926
:40CAC000D8B16A48416A204600E008E26AF03AF96649C96988422AD30121644880F828104462014691ED080ABCEEC00A10EE101A88B20321FFF784FA19E05C4890F8280035
:40CB0000012814D15948C06988B15848416A20466AF018F955498969884208D30021534880F82810446203210020FFF769FA4F4890F8500038BB4D48006C20B34B48C16CEE
:40CB400020466AF0FFF84949496C884239D30121464880F85010C464014691ED080ABCEEC00A10EE101A88B20321FFF749FA3F4991ED030ABCEEC00A10EE101A88B201211C
:40CB8000FFF73EFA1DE0394890F85000012818D13648406CA8B13548C16C20466AF0D2F83249096C88420CD30021304880F85010C46403210020FFF723FA01210020FFF767
:40CBC0001FFA8CE1294890F878106830405C38BB264890F83C00012817D12448816B20466AF0B0F82149C96A88420DD300211F4880F83C10846302210020FFF701FA1B48F3
:40CC0000006B002800D10125D2E01848816B20466AF098F81549096B8842F5D30125C7E0124890F878106830405C02282BD10F48007D01281CD10D48016920466AF082F844
:40CC40000A4949688842DFD3002108480175046101210020FFF7D4F904488068002800D10125A5E00000002001000020A41100209C48016920466AF065F89A4989688842EC
:40CC800000D3012594E0974890F878106830405C012826D1934890F82800012816D19148416A20466AF04EF88E49896988427FD300218C4880F82810446203210020FFF735
:40CCC0009FF98848C06990BB012571E08548416A20466AF037F88349C969884268D3012566E0804890F878106830405C03282AD17C4890F8500001281AD17A48C16C2046D4
:40CD00006AF020F87749096C884251D30021754880F85010C46403210020FFF771F901210020FFF76DF96F48406C00B901253FE06C48C16C20466AF005F86A49496C88420D
:40CD400036D3012534E0674890F878106830405C04282DD1634890F8640001281ED16148016E204669F0EEFF5E49496D88421FD300215C4880F86410046602210020FFF773
:40CD80003FF903210020FFF73BF901210020FFF737F95448806D58B9012509E05148016E204669F0CFFF4F49896D884200D30125012D28D100254B4890F87800401CC1B228
:40CDC000484880F8781090F8781090F87700814203DB0021434880F87810424890F878106830405C80B901213E4880F83C108463014691ED0D0ABCEEC00A10EE101A88B23B
:40CE00000221FFF7FDF869E0364890F878106830405C02280FD10121324801750461014691ED030ABCEEC00A10EE101A88B20121FFF7E6F852E02B4890F878106830405CD1
:40CE4000012810D10121274880F828104462014691ED080ABCEEC00A10EE101A88B20321FFF7CEF83AE01F4890F878106830405C03281BD101211B4880F85010C46401468C
:40CE800091ED080ABCEEC00A10EE101A88B20321FFF7B6F8134991ED030ABCEEC00A10EE101A88B20121FFF7ABF817E00D4890F878106830405C042810D10121094880F844
:40CEC0006410046602210020FFF79AF803210020FFF796F801210020FFF792F800BF00BF70BD0000A411002070B59B201CE0C41700EBD4646511F74C54F82540C51700EB74
:40CF0000D5656D11A0EB45160125B5402C40C51700EBD5656D11A0EB45160125B540AC4200D103E0411EC8B20028E0DC00BF70BD10B50024E848006888B14FF47A71E648EB
:40CF4000006869F0CFFE50B10FF009FB38B9E3480078122803D1E248007800B90124204610BDE04A50547047DE4AFF3A5054704730B50346DA1703EBD2625411D54A52F87A
:40CF800024201946DC1703EBD4646411A3EB44150124AC40A2431846DC1703EBD4646511CC4C44F82520DA1703EBD2625411C94A143252F824201946DC1703EBD464641191
:40CFC000A3EB44150124AC40A243DC1703EBD4646511C04C143444F82520DA1703EBD2625411BC4A283252F82420DC1703EBD4646411A3EB44150124AC40A243DC1703EB3E
:40D00000D4646511B34C283444F825200020FFF7ABFF30BD30B50146CB1701EBD3635C11AC4B53F82430CC1701EBD4646411A1EB44150124AC4023400BB1012030BD0020C7
:40D04000FCE770B504460D4600BFA748055502461119A64A1019012208F012FF00BF70BD70B504460D4600BFA14820F81450A14A02EB44009E4A02EB4401022208F000FF29
:40D0800000BF70BD70B504460D4600BF9A48055502461119994AA018012208F0F1FE00BF70BD2DE9F0412DED028B0446944890ED201BB0EE410AF0EE610A51EC100B83F0FB
:40D0C000BBFA08EE100A9FED8F0AC8EE000ABCEEE00A10EE100AC5B29FED8B0AC8EE000ABCEEE00A10EE100A80B23C2190FBF1F201FB1200C6B269028448007E41EA001063
:40D100008249497E084387B27B48005D401C00F0FF0841462046FFF7B5FF39462046FFF79FFF31462046FFF78CFFBDEC028BBDE8F08110B504466948007812281AD1744893
:40D140000470007826280FD07148007825280BD06F480078202807D06D480078FFF7A1FF6B48007861F067FA8620FBF7ADF9C120FBF7AAF910BD2DE9F0412DED028B044696
:40D180000025512C6FD2DFE804F029EC2A2F306E6E6E6E6E6E313B4D5C6F6E6E6E6E6E6E707880EB886E6E6E6E6E6E6E6EEDFB6E6EE86EE7E6E5E4E3E2E1E0DFDEDD6E6E90
:40D1C0006EDC6E6E6EDBDAD9D8D7D66E6E6E6E6ED5D4D36E6E6ED2D16E6EA40067E167F02CFC80F0010562E161E160E101F0C5FB28B969F05DFD4749884200D9012556E1A1
:40D2000001F0BBFB68B1444890ED1A0ADFED430AB4EEE00AF1EE10FA02DC90F8700000B9012544E101F0A9FB50B13B4890ED1A0ADFED3B0AB4EEE00AF1EE10FA00D2012561
:40D2400035E101F09AFB68B1304890ED0A0ADFED350AB4EEE00AF1EE10FA02DC90F8300000B9012523E121E121E103F0CFFB08B9012000E00020054619E102F051FB0128A8
:40D2800000D100E00020054611E119F057F808B9012000E00020054609E10FF0FFF9142803D00FF0FBF9152812D11F48D0ED020A1348B0F8C80000EE100AB8EE400AF4EE03
:40D2C000C00AF1EE10FA01D8012000E000200546EDE0E7E0A00B0010100000209D040020403E0010FF04006810270010FE1E006812250010001D006812240010001C00689C
:40D30000A81700100000614500007042EC1400100D000020C0D4010090110010000048430000484200401C46B0210010B4E0AEE0A1E09BE095E08FE089E083E07DE077E029
:40D3400071E06BE065E05FE059E053E04DE047E041E03BE035E02FE029E016E010E001E08DE013E0F74890F82D01802803D1F54890F8F10408B9012000E00020054696E06F
:40D3800003F02AFB80F0010591E090E012F02CFA50B10FF083F9142806D0EA4890F87B07012801D0012000E0002005467FE003F0D1FE00F001057AE003F0CCFEC0F3400580
:40D3C00075E003F0C7FEC0F3800570E003F0C2FEC0F3C0056BE003F0BDFEC0F3001566E003F0B8FEC0F3401561E003F0B3FEC0F380155CE003F0AEFEC0F3C01557E003F0FB
:40D40000A9FEC0F3002552E003F0A4FEC0F340254DE003F09FFEC0F3802548E003F09AFEC0F3803543E003F095FEC0F380453EE003F090FEC0F3C04539E003F08BFEC0F39E
:40D44000005534E003F086FEC0F340552FE003F081FEC0F380552AE003F07CFEC0F3C05525E003F077FEC0F3407520E003F072FEC0F380751BE003F06DFEC50F17E00FF039
:40D480006EF808B1012000E0002005460FE008F0DBFC80F001050AE00125002500BF00BF00BF04E003F078FF054600E000BF00BF0FF0F4F8152872D0A24890F87B070128BD
:40D4C000F9D02046142C6BD00DDCA0F105000F2867D2DFE800F0455F1D6A72BA6666666666CEE1FAF50022287DD008DC15287BD01B287AD01F2879D0212852D119E04928F3
:40D5000075D04A2874D04B2873D04F28F5D179E08D488078FE2809D18A4890F89907032802D131F0FDFC08B9012000E00020054696E1844890F87D0703280ED0814890F8EF
:40D540007D07022809D07F4890F87D07012802D17E48007808B9012000E0002005467FE105F0EDFE20B106F063F808B1012000E0002005461DB10520FFF7DBFD09E006F0C3
:40D5800057F830B172480078052802D12020FFF7D0FD65E105F0A5F920B9012003E0E3E1A8E05CE1002005465AE106F0D8FA08B1012000E00020054652E166481CF0F0FF58
:40D5C000D8B965481CF0ECFFB8B964481CF0E8FF98B963481CF0E4FF78B962481CF0E0FF58B9614806E0DEE090E0BFE0D2E0E2E0FDE011E11CF0D4FF08B1012000E00020CC
:40D6000005462DE153481CF0CBFF012818D052481CF0C6FF012813D050481CF0C1FF01280ED04F481CF0BCFF012809D04D481CF0B7FF012804D04C481CF0B2FF012801D12D
:40D64000012000E0002005460AE105F0F1FF80F001051DB10A20FFF76CFD09E005F06FFE30B93B4800780A2802D12020FFF761FDF6E00FF013F814280DD10FF00FF815289C
:40D6800009D004F039FA20B90EF01EFA08B1012000E000200546E3E005F013FAA0B905F008FA88B905F0FEF970B905F0F3F958B905F0E8F940B974F019FD18B9012002E0DC
:40D6C0000CE002E000200546CAE074F02FFD012801D0012000E000200546C1E00EF0DEFF142806D10EF0DAFF152802D00EF00CF90546B5E00EF0D2FF142806D10EF0CEFF4C
:40D70000152802D00EF01FF90546A9E00EF0C6FF142816D10EF0C2FF152812D00EF0DEF868B90EF048F950B90EF06CF938B90EF05CF920B90EF04CF908B9012000E000204A
:40D7400005468DE0781A0010E8700220A40400200D00002024DB001034DB001044DB001054DB001064DB001074DB00100EF096FF14280ED10EF092FF15280AD0F74890F87B
:40D78000D00020B10CF0CDFB08B9012000E00020054665E073F032FC012801D0012000E0002005465CE012F01FF808B9012000E00020054654E005F084F998B905F079F9BB
:40D7C00080B905F06FF968B905F064F950B905F059F938B979F01AFC08B1012000E00020054603E00B2074F095F8054638E00EF0E2F840B90EF006F928B90EF0F6F810B975
:40D800000EF0E6F838B103F0D0F8B0EE408A0EF03EF880F0010523E00EF040FF14281DD10EF03CFF152819D00CF0A5FA90B905F048F958B905F03DF940B905F033F928B93C
:40D8400005F028F910B905F01DF928B1482074F061F808B1012000E00020054600E000BF00BF05F02EF960B905F023F948B905F019F930B905F00EF918B905F003F9002820
:40D8800072D0A4F14E004E286FD2DFE800F0276E6E364A6E5E63686F74797E83888D6E92979CA1A6ABB0B5EFF4F9FEEAE9E8E7E6E5E4E3E2E1E0DFDEDDDCDBDAD9D8D7D685
:40D8C000D5D4D3D2D1D0CFCECDCCCBCAC9C8C7C6C5C4C3C2C1C0BFBEBDBCBBBA74F00CF89F4BC01A71F1000104D205F0CEF908B1012000E000200546C6E109F0E8FB064641
:40D900000F4674F09EF8301A8F4107D205F0B3F920B166F070FB08B1012000E000200546B2E109F0D4FB06460F4674F08AF8301A8F4107D205F09FF920B166F033FB08B1DD
:40D94000012000E0002005469EE1012073F0E2FF054699E1022073F0DDFF054694E1032073F0D8FF05468FE18FE18CE1042073F0D1FF054688E1052073F0CCFF054683E16F
:40D98000062073F0C7FF05467EE1072073F0C2FF054679E1082073F0BDFF054674E1092073F0B8FF05466FE10A2073F0B3FF05466AE10C2073F0AEFF054665E10D2073F087
:40D9C000A9FF054660E10E2073F0A4FF05465BE10F2073F09FFF054656E1102073F09AFF054651E1112073F095FF05464CE1122073F090FF054647E1132073F08BFF05463B
:40DA000042E13BE135E12FE129E123E11DE117E111E10BE105E1FFE0F9E0F3E0EDE0E7E0E1E0DBE0D5E0CFE0C9E0C3E0BDE0B7E0B1E0ABE0A5E09FE099E093E089E083E062
:40DA40007DE077E071E06BE065E05FE059E053E04DE047E041E03BE035E02FE029E023E01DE017E011E00BE005E0FFE7142073F051FF054608E1152073F04CFF054603E1DE
:40DA8000162073F047FF0546FEE0172073F042FF0546F9E0182073F03DFF0546F4E0192073F038FF0546EFE01A2073F033FF0546EAE01B2073F02EFF0546E5E01C2073F01E
:40DAC00029FF0546E0E01D2073F024FF0546DBE01E2073F01FFF0546D6E01F2073F01AFF0546D1E0202073F015FF0546CCE0212073F010FF0546C7E0222073F00BFF054666
:40DB0000C2E0232073F006FF0546BDE0242073F001FF0546B8E0252073F0FCFE0546B3E0262073F0F7FE0546AEE0272073F0F2FE0546A9E0282073F0EDFE0546A4E0292013
:40DB400073F0E8FE05469FE02A2073F0E3FE05469AE02B2073F0DEFE054695E0A8170010981854772C2073F0D5FE05468CE02D2073F0D0FE054687E02E2073F0CBFE05467D
:40DB800082E02F2073F0C6FE05467DE0302073F0C1FE054678E0312073F0BCFE054673E0322073F0B7FE05466EE0332073F0B2FE054669E0342073F0ADFE054664E0352081
:40DBC00073F0A8FE05465FE0362073F0A3FE05465AE0372073F09EFE054655E0382073F099FE054650E0392073F094FE05464BE03A2073F08FFE054646E03B2073F08AFE4B
:40DC0000054641E03C2073F085FE05463CE03D2073F080FE054637E03E2073F07BFE054632E03F2073F076FE05462DE0402073F071FE054628E0412073F06CFE054623E009
:40DC4000422073F067FE05461EE0432073F062FE054619E0442073F05DFE054614E0452073F058FE05460FE0462073F053FE05460AE0472073F04EFE054605E0492073F0AD
:40DC800049FE054600E000BF00BF2846BDEC028BBDE8F0814FF00008C1464FF0500A0321FE4880F8CC10A421FD487CF0DEF8002436E10020FB490855FB48005DC4EB041169
:40DCC000FA4A02EB810189680870C4EB0410114601EB800080680078002804DCF248FF38005D00287DD0E21704EBD2625311EC4A121D52F823202146E31704EBD3635B1173
:40DD0000A4EB431C012303FA0CF31A432046E31704EBD3634FEA631CE14B1B1D43F82C20E21704EBD2625311DD4A183252F82320E31704EBD3635B11A4EB431C012303FA38
:40DD40000CF31A43E31704EBD3634FEA631CD44B183343F82C20C4EB0410D44901EB8000007BE0B1E21704EBD2625311CC4A2C3252F823202146E31704EBD3635B11A4EB25
:40DD8000431C012303FA0CF31A432046E31704EBD3634FEA631CC24B2C3343F82C2068F087FFC34941F8240000BFE21704EBD2625311BB4A403252F823202146E31704EB7D
:40DDC000D3635B11A4EB431C012303FA0CF39A432046E31704EBD3634FEA631CB04B403300E002E043F82C2000BFC4EB0410AF4901EB800090F8300001281CD1E21704EB06
:40DE0000D2625311A64A543252F823202146E31704EBD3635B11A4EB431C012303FA0CF31A432046E31704EBD3634FEA631C9C4B543343F82C20C4EB04109C4901EB8000A4
:40DE400090F83000022807D0C4EB041001EB800090F8300003281CD1E21704EBD26253118F4A683252F823202146E31704EBD3635B11A4EB431C012303FA0CF31A432046A7
:40DE8000E31704EBD3634FEA631C854B683343F82C20C4EB0410854901EB800090F8300004281CD1E21704EBD26253117C4A7C3252F823202146E31704EBD3635B11A4EBC9
:40DEC000431C012303FA0CF31A432046E31704EBD3634FEA631C724B7C3343F82C20102C1CD0E21704EBD26253116D4A903252F823202146E31704EBD3635B11A4EB431C88
:40DF0000012303FA0CF31A432046E31704EBD3634FEA631C624B903343F82C20601CC4B29C2CFFF6C6AE60F011FC4FF47A60DFF884C100DF5948D0F8F0100120DFF878C1FE
:40DF400000DF4FF47A60DFF86CC100DF00BF002251460320DFF864C100DF0646022E50D1DFF85CC100DF074607F0020078B3002442E0E31704EBD3634FEA631C484B1B1D83
:40DF800053F82C304FEAE47C04EBDC6C4FEA6C1CA4EB4C1B4FF0010C0CFA0BFC03EA0C034FEAE47C04EBDC6C4FEA6C1CA4EB4C1B4FF0010C0CFA0BFC634509D10120C4EBAC
:40DFC00004113A4A02EB81018968087008E018E00020C4EB0411354A02EB810189680870C4EB0411314A02EB8101896808782146FEF7B7FF601CC4B29C2CBADB4420FAF7C0
:40E0000063FA002463E22046FFF7B5F805462046FFF700F8A84225D02DBB4FF000092148005D012801D181460EE0C4EB04101F4901EB8000407B10B94FF0010904E021483C
:40E04000007808B14FF00109B9F1010F0AD10020144908554FF001082046FEF789FF4420FAF732FAF0E0E31704EBD3634FEA631C0B4B1B1D53F82C304FEAE47C04EBDC6C5F
:40E080004FEA6C1CA4EB4C1B4FF0010C0CFA0BFC03EA0C034FEAE47C16E00000001900209C0B0010000B0010FF04006800160908F407001021F8080881F80808E1F8080882
:40E0C00029F80808403E001004EBDC6C4FEA6C1CA4EB4C1B4FF0010C0CFA0BFC6345C1D00020FE49085500BF0DF065FC40B90DF089FC28B90DF079FC10B90DF069FCD8B17E
:40E10000E21704EBD2625311F54A52F823202146E31704EBD3635B11A4EB431C012303FA0CF31A432046E31704EBD3634FEA631CEB4B43F82C201AE0E21704EBD2625311C2
:40E14000E74A52F823202146E31704EBD3635B11A4EB431C012303FA0CF39A432046E31704EBD3634FEA631CDD4B43F82C20E21704EBD2625311DA4A3C3A52F8232021460A
:40E18000E31704EBD3635B11A4EB431C012303FA0CF31A432046E31704EBD3634FEA631CCF4B3C3B43F82C2068F082FDCD4941F8240000BF00BF0DF0FEFB40B90DF022FC42
:40E1C00028B90DF012FC10B90DF002FC08B1012000E0002001281BD1E21704EBD2625311BF4A52F823202146E31704EBD3635B11A4EB431C012303FA0CF31A432046E317AD
:40E2000004EBD3634FEA631CB54B43F82C201AE0E21704EBD2625311B14A52F823202146E31704EBD3635B11A4EB431C012303FA0CF39A432046E31704EBD3634FEA631C5E
:40E24000A74B43F82C2000BF002D7DD0E21704EBD2625311A24A283A52F82320E31704EBD3635B11A4EB431C012303FA0CF31A40002A4CD1C4EB04109B4901EB8000406A9A
:40E28000E8BBE21704EBD2625311954A283A52F823202146E31704EBD3635B11A4EB431C012303FA0CF31A432046E31704EBD3634FEA631C8A4B283B43F82C204FF00108CC
:40E2C000C4EB0410884901EB8000806800787E280DDAC4EB041001EB800080680078401CC4EB0411804A02EB81018968087021460120FEF739FEC4EB04117B4A00E007E0DC
:40E3000002EB8101896808782146FEF72AFE53E0C4EB0412744B03EB8202516A714A52F8240068F0DFFCE0B3E21704EBD26253116B4A283A52F823202146E31704EBD363FC
:40E340005B11A4EB431C00E090E0012303FA0CF31A432046E31704EBD3634FEA631C604B283B43F82C204FF00108C4EB04105E4901EB8000806800787E280DDAC4EB0410D6
:40E3800001EB800080680078401CC4EB0411564A02EB81018968087021460120FEF7E4FD00E009E0C4EB04114F4A02EB8101896808782146FEF7D5FDC4EB04124A4B03EB1F
:40E3C0008202127B002A51D0E21704EBD2625311434A143A52F82320E31704EBD3635B11A4EB431C012303FA0CF31A40F2BB0DF0E2FA40B90DF006FB28B90DF0F6FA10B9D2
:40E400000DF0E6FA98B3C4EB0411374A02EB8101887B214604F0F1F9C4EB0410324901EB8000806A58B1C4EB04120B4603EB8202916A2C4A52F8240068F054FCB0B100BFEC
:40E44000E21704EBD2625311254A143A52F823202146E31704EBD3635B11A4EB431C012303FA0CF31A432046E31701E02DE00BE004EBD3634FEA631C194B143B43F82C2025
:40E4800000BF4FF0010820E000BFE21704EBD2625311134A143A52F823202146E31704EBD3635B11A4EB431C012303FA0CF31A432046E31704EBD3634FEA631C084B143BA2
:40E4C00043F82C2000BF4FF00108601CC4B29C2CFFF699ADB8F1010F14D107E0000B0010DC0B0010F4070010001609089248D0F8F0100120DFF844C200DF4FF000084420A6
:40E50000F9F7E2FF8E48007848B9FEF711FD30B14420F9F7D9FF01208949087009E00EF01EF830B98748006818B968F0C1FB85490860FEF7D9FC044609E5002107E0824834
:40E5400050F8210008B101207047481CC1B20529F5DB0020F8E70020002107E07A4A283252F8212002B101204A1CD1B20529F5DB70470020002107E0734A283252F82120C0
:40E5800002B108464A1CD1B20529F5DB704770B500240DF010FA40B90DF034FA28B90DF024FA10B90DF014FA68B39B2428E0E31704EBD3635D11644B143353F82530E51777
:40E5C00004EBD5656D11A4EB45160125B5402B40E51704EBD5656D11A4EB45160125B540AB420BD1C4EB0413584D05EB83035B7B012B03D1564B1B5D03B903E0601EC4B230
:40E60000002CD4DC00BF204670BD0121504A1154704701460020FF2906DA4D4A525C0AB1012200E000221046704700210CE0464850F82100444A503252F82120104008B18B
:40E6400001207047481CC1B20529F0DB0020F8E700210CE03C4850F821003B4A643252F82120104008B101207047481CC1B20529F0DB0020F8E7002200210CE0324850F8B2
:40E680002100314B8C3353F82130184008B101207047481CC1B20529F0DB1046F8E700B5002304E01846FFF7B0FF581CC3B29C2BF8DB00BD1FB5044626A30FCB8DE80F0030
:40E6C00084B137F07BFE3BF0C6FB00210A2068F065FD0D226946FF2037F09DFD01202149087002E000201F4908701FBD1D48007870471D48007870470146C1EB0110134A4C
:40E7000052F8200070470146C1EB01100F4A02EB800000797047014641B1202905D0252902D0262904D100BF00BF00BF002001E0012000BF00BF70470019002081F80808CD
:40E740001400002010000020A00B001000160908000B00100102050A0B111214181921242B0000000C0000200D00002070B504460025FE4890F82805012804D0022808D05C
:40E7800003280BD100E000BF204621F084FB054606E0204624F02FFD054601E0002070BD00BF2846FBE710B5F148007800F0010080B10120FFF7DAFF00280AD0EC48006838
:40E7C00040F00800EA4908600846006820F001000860D1E0E648007800F0020080B10220FFF7C4FF0028F4D0E148006840F00800DF4908600846006820F002000860BBE0B2
:40E80000DB48007800F0400080B14020FFF7AEFF0028DED0D648006840F00800D44908600846006820F040000860A5E0D048007800F0800080B18020FFF798FF0028C8D0AF
:40E84000CB48006840F00800C94908600846006820F0800008608FE0C548007800F0040080B10420FFF782FF00280AD0C048006840F00800BE4908600846006820F0040026
:40E88000086079E0BA48007800F0080058B10820FFF76CFF00286FD0B548006820F00800B349086068E0B248007800F0100058B11020FFF75BFF00285ED0AD48006820F045
:40E8C0001000AB49086057E0A948007800F0200078B12020FFF74AFF60B3A548006820F02000A34908600846006840F40040086042E09F48008800F4807058B14FF4807025
:40E90000FFF734FFB0B19A48006820F480709849086031E09648008800F4004058B14FF40040FFF723FF28B19148006820F400408F49086020E08E48008800F4007058B1EE
:40E940004FF40070FFF712FFB0B18948006820F40070874908600FE08548008800F4804050B14FF48040FFF701FF28B18048006820F480407E49086010BD7E48007B05284E
:40E9800001D1012070470020FCE710B57A49486E68F0C9F9B0F5FA7F24D3774890F8700000B30020744981F87000744981F8D2009FED730A084680ED140A00216E4880F8D4
:40E9C00042109FED6F0A80ED110A00206B4981F8CD009FED6C0A684880ED120A002081F8CA000CE06449486E68F09DF96649884205D3614890F8700008B9FFF7BEFF634931
:40EA0000486A68F090F943F69821884208D35F4890F8300020B100205C4981F830000EE05A49486A68F07FF95749884207D3574890F8300018B9FFF7A0FF00B100BF5449ED
:40EA4000086C68F070F942F21071884208D3504890F84C0020B100204D4981F84C000EE04B49086C68F05FF94749884207D3484890F84C0018B9FFF780FF00B100BF4549CD
:40EA8000D1F83C0168F04FF943F69821884208D3404890F8480120B100203E4981F848010FE03C49D1F83C0168F03DF93649884207D3384890F8480118B9FFF75EFF00B135
:40EAC00000BF3549486C68F02EF9B0F57A6F08D3314890F8500020B100202F4981F850000EE02D49486C68F01EF92749884207D3294890F8500018B9FFF73FFF00B100BF61
:40EB00002649486A68F00FF944F62061884208D3224890F8300020B10020204981F830000EE01E49486A68F0FEF81749884207D31A4890F8300018B9FFF71FFF00B100BF07
:40EB40000E4890F8D20030B90CF034FB18B19FED0C0A0CF0A9FA084890ED120ADFED090AB4EE600AF1EE10FA1FD119E0781A00102C0000209018001090110010A8170010FB
:40EB80000000000000007F43E0930400EC140010C81200106C13001018130010B8140010F8A203214C307AF0F9FC10BD10B568F07FF80446F4484466406E6438F24908665F
:40EBC0000846406E096E401A00EE100AB8EE400AED4880ED1A0A0120EB4981F87000EB484462406A6438E94908620846406A096A401A00EE100AB8EE400AE44880ED0A0A27
:40EC00000120E24981F83000E1480464006C6438DF49C8630846006CC96B401A00EE100AB8EE400ADA4880ED110A0120D84981F84C00D848C0F83C41D0F83C016438D549EE
:40EC4000C1F838010846D0F83C01D1F83811401A00EE100AB8EE400ACE4880ED500A0120CC4981F84801CC484464406C6438CA4908640846406C096C401A00EE100AB8EE1C
:40EC8000400AC54880ED120A0120C34981F85000C2484462406A6438C04908620846406A096A401A00EE100AB8EE400ABB4880ED0A0A0120B94981F8300010BD0021B24820
:40ECC00080F842101FED520A80ED110A9FEDB40B80ED0A0B9FEDB20B80ED0C0B80F841101FED580A80ED120A70470120AE490873704710B567F0DCFFA349486667F0D8FF40
:40ED0000A2494862A04890ED120A5FED620AB4EE600AF1EE10FA07D01FED660A80ED120A4FF499703DF052F9A04890F82805062870D2DFE800F06F032F04537000BF9A48A3
:40ED4000407B20B9FFF7BAFF002099498880102195481030DFF85CC200DF012810D0934B93F83025904B597B904BD3F82C0520F03DFE8D49487301F11000DFF83CC200DF45
:40ED80008B488088052804DDFFF7AFFF00208849888044E08448407B30B9FFF78FFF23F0CBF900208249888010217F481030DFF804C200DF012810D07C4B93F830257A4BC2
:40EDC000597B7A4BD3F82C0523F0A9FF7649487301F11000DFF8E0C100DF20E07248407B18B9FFF76BFF1DF070FE10216E481030DFF8C0C100DF01280AD04FF4E1301DF00D
:40EE000071FE6949487301F11000DFF8ACC100DF05E0FFE700BF08206349487300BF00BF10BD10B56048007B062856D2DFE800F003172438465465F0B5F860B15F48007836
:40EE400065F0A6FC38B103205749087367F030FF5B49086002E00120534908733DE000215848007865F015F902204F49087367F01FFF5349086030E05148006867F053FFA7
:40EE8000B0F57A7F0BD301214E48007865F001F903204549087367F00BFF494908601CE04748006867F03FFF40F6C411884204D304203D490873002048730EE0FFF719FFA0
:40EEC0003948407B082806D1FFF770FE0520364908730120487000E000BF00BF10BD102131481030DFF8CCC000DF01280AD000202D4948730420087301F11000DFF8B8C0D8
:40EF000000DF17E004213048DFF8A8C000DF012810D02D48007C40F020002B4908742B48C16B4FF48060DFF8A8C000DF2648DFF888C000DF704710B51C4991F828150129E9
:40EF400006D0022908D0032903D0042908D105E000BF23F07FF805E0002003E0002001E0002000BF00BF10BD10B5002465F01AF838B10E4890F8280501282BD003282ED19F
:40EF800029E02FE02D2D2D0090110010EC140010C81200106C13001018130010B8140010000000000000000090180010781A00108018001049FD080865FC0808CE030010B7
:40EFC00040000020F0030010B01800100019002081F8080800BF1FF011F9044601E0002400BF00BF204610BD10B5FE4991F82815012906D0022908D0032903D0042908D162
:40F0000005E000BF1FF0C2F805E0012003E0012001E0002000BF00BF10BD10B5F14991F82815012906D0022908D0032903D0042908D105E000BF1FF0A0F805E0012003E00C
:40F04000012001E0002000BF00BF10BD70B505460E4636B1012E0DD0022E24D0032E3CD113E00DB9002404E0022D01D1032400E0022434E00DB9002406E0022D01D0092D01
:40F0800001D1032400E0022429E0FFF7C6FF08B9012407E00DB9002404E0052D01D1032400E002241BE0FFF79FFF08B9012413E00DB9002410E0042D09D1FFF755FF20B159
:40F0C000FFF739FF08B1052406E0032404E0052D01D1042400E0022401E0002400BF00BF052C05D0062C03D067F0E2FDBE490860BD48006867F017FEBC49C1F89000084635
:40F1000080F8CA4070BD0020B64991F82815012904D0B44991F82815032900D10120704710B5B24890ED0E1BB0EE410AF0EE610A9FEDAF1B53EC112B51EC100B81F006FF6F
:40F140002FD3AA4890ED0E1BB0EE410AF0EE610A9FEDA91B53EC112B51EC100B81F0BCFD1FD3A24890ED0C1BB0EE410AF0EE610A9FEDA31B53EC112B51EC100B81F0E6FE52
:40F180000FD39A4890ED0C1BB0EE410AF0EE610A9FED9D1B53EC112B51EC100B81F09CFD07D20020914981F8CD0001209849087018E0FFF7A8FF60B1964890F824008B49FD
:40F1C00081F8CD00934890F82410934880F8401005E0914890F84000844981F8CD0000208B49087010BD10B52DED048B10218B48DFF82CC200DF012877D07C4890F8D20019
:40F20000002874D0102179489430DFF814C200DF01286CD00120814908747F48007E81F864007D48407E81F865007B4890ED070A084680ED1A0A6D4890F8CB0081F86C00B4
:40F240006A4890F8CC0081F86D00684890ED1F0A084680ED1C0A654890ED000B084680ED0A0B624890ED020B084680ED0C0B5F4890ED0C0B084680ED060B5C4890ED0E0B1F
:40F28000084680ED080B594890ED150A084680ED100A564890ED160A084680ED0F0A534890F8CD0081F83800504890F8CA0081F83A004E4890ED140A084680ED170A02F022
:40F2C00058FA564880ED180A484890ED130A534880ED150AFCF7B4FC504880ED160A43489430DFF840C100DF04E04CE1FFE700204A490874484890F87000002841D0102158
:40F300004548DFF81CC100DF01283AD0424890F84200424981F83B003F49C86B81F06BFC41EC190B9FED400B53EC102B81F072FA41EC180B81F080F938494864364890ED73
:40F34000120A084680ED120A022239A132484C307AF093FC30B9042236A130484C307AF0ABFD06E005222C494C312C484C307AF0A3FD0021294880F850102748DFF8A4C0B4
:40F3800000DF2E4890F83000F8B110212B48DFF890C000DF012818D02848007E1F4981F874002648407E81F875002448408BA1F876002248007F81F878002048807F81F87F
:40F3C00079001E48DFF85CC000DF1D4890F84C00C0B310211A48DFF848C000DF012859D0174830E0781A00103C000020A8170010000000000080664000000000008066C005
:40F40000000000000080564000000000008056C09018001000170010901100102015001049FD080865FC08080000000000408F40475300005453545200000000EC1400107E
:40F44000C812001026E0407EFE4981F87B00FE48007E81F87A007C31FB480A3002690A6042694A6080698860F74890ED0A0AF54880ED220AF44890ED0B0AF24880ED230A7F
:40F48000F14890ED0C0AEF4880ED240AEE48DFF8BCC300DFEE4890F85000A0B31021EC48DFF8B0C300DF01282DD0E94890ED080AE44880ED260AE64890ED090AE14880ED51
:40F4C000270AE34890ED0A0ADE4880ED280AE04890ED0B0ADB4880ED290ADD4890ED0C0AD84880ED2A0ADA4890ED0D0AD54880ED2B0AD74890ED0E0AD24880ED2C0AD44862
:40F50000DFF848C300DFD44890F84801C0B11021D148DFF840C300DF012811D0CE48807DC200CD491831C748BC307AF0FDFBCA48807DC44981F8B400C748DFF810C300DF2D
:40F54000C64890F83000F0B11021C448DFF804C300DF012817D0C048807DBA4981F8B400BE4890ED060AD0ED050A30EE600ABC48D0ED000A20EE200A084680ED2E0AB74849
:40F58000DFF8C8C200DFAF48DFF8C0C200DFBDEC048B10BD10B5B34890F8D100B2490978884207D0AF4890F8D100AF490870032033F08AFD10BD10B52DED028BAB4890F860
:40F5C00078430E2C20D2DFE804F01F20212216151407251F1F1F232405F052F9F0EE408A05F026F9F0EE000A80EE201A38EEC18A15E000BF00BF05F043F9F0EE408A05F09A
:40F6000017F938EEC08A0AE000BF00BF00BF00BF00BF00BF05F049F9B0EE408A00BF00BFB0EE480ABDEC028B10BD10B52DED0A8BF0EE408AF0EE609A9FED8D0AF4EEC08A93
:40F64000F1EE10FA04D2B0EE680ABDEC0A8B10BD9FED880AB0EE40AAFFF7ADFFB0EE40AA29EE8A0AB0EE409A29EE090AB0EE409A28EEA88AB4EEC89AF1EE10FA0FD238EEDF
:40F68000490A10EE101A084681F058FE41EC1C0BB0EE4C0AF0EE6C0A7FF0F6F801E09FED760BB0EE40BAF0EE60BA51EC1B0B80F0C3FF08EE100AB0EE480AC6E72DE9F041BA
:40F6C0002DED108B05460E461446664890F8D00038B195ED130A6A48D0ED000A30EE200A01E095ED130A10EE107A384681F026FE41EC1F0BB0EE4F0AF0EE6F0A7DF0D8FC0C
:40F70000B0EE40DAF0EE60DA51EC1D0B80F094FF08EE900A384681F011FE41EC1F0BB0EE4F0AF0EE6F0A7EF083FFB0EE40DAF0EE60DA51EC1D0B80F07FFF09EE100A16F034
:40F7400014FDF0EE40AA1AEE900A81F0F7FD41EC1F0BB0EE4F0AF0EE6F0A7EF069FFB0EE40DAF0EE60DA51EC1D0B80F065FF09EE900A1AEE900A81F0E1FD41EC1F0BB0EEAE
:40F780004F0AF0EE6F0A7DF093FCB0EE40DAF0EE60DA51EC1D0B80F04FFF08EE100A9FED35AA324890F84F030A280BD19FED310AF0EE409A9FED2F0AB0EE408A9FED2D0A5E
:40F7C000B0EE40AA05F0A9F8B1EE40EA05F095F8F1EE40EA28EE880A69EE0A0A00EEA90A20EE0E0A84ED010A28EEA90A69EE0A0A00EEC80AD4ED010A40EE2E0AC4ED010A5F
:40F80000B1EE490A20EE080A68EE8A0A00EEA90A20EE0E0A84ED000A29EE290A68EE8A0A00EE880AD4ED000A40EE6E0AC4ED000A94ED000A10EE101A084681F07FFD41EC8F
:40F840001D0B1FE020150010C812001065FC08081813001049FD08086C130010B8140010F46B0A08A81700104A000020781A00102FDDE43E0000000000000000000000004B
:40F88000E46B0A089FEDF70B53EC102B81F060FA41EC1B0B94ED010A10EE101A084681F04DFD41EC1D0B95ED2E1BB0EE410AF0EE610A53EC102B80F0ADFF41EC1C0B96ED45
:40F8C000061BB0EE410AF0EE610A53EC102B51EC1B0B80F0E3FE41EC1B0B96ED081BB0EE410AF0EE610A53EC102B51EC1C0B80F0D5FE41EC1C0B102105F19400DFF86CC326
:40F9000000DF012808D085ED04BB85ED06CB05F19400DFF85CC300DFBDEC108BBDE8F081D44890F8CA00704700B5FFF7F9FF032801D1012000BD0020FCE70721CE4A117053
:40F940005170CE4991F850179170CC4991F85117D170CA4991F852171171C84991F853175171C64991F854179171C44991F85517D171C24991F856171172002006E0BE4950
:40F98000095CBF4A515CBF4A1154401C0928F6DB704770B504460025B4F5E13F02D94FF4E1340225B548D0F84C07A04217D000BFB248C0F84C47042200F24C71B2480068D6
:40F9C00000F2144006F05CFA00BF7620F8F77CFDAE48C16B4FF40060DFF8B4C200DF284670BD1FB5002000900190029003460222A84903902B2064F01EFCA048D0F84C07D8
:40FA0000B0F5E13F05D89D48D0F84C07B0F5966F03D24FF4E130FFF7BCFF64F041FF04469648D0F84C17204663F010F9FFF785FF1FBD924991F8291309B9012000E000201E
:40FA400070471FB500219348007864F0C5FC002001210090CDE90101034602468E4903902B2064F0E8FB1FBD8C480078022803D08A480078012801D1012070470020FCE726
:40FA80002DE9F043C1B00546082D2BD110218448DFF8D8C100DF012823D081481EF02FF880468048077815E001AA39467C481EF031F8FFF7BEFF38B164F0F2FE81460122B9
:40FAC00001A963F00AFEC6B216B97648077003E0781CC7B24745E7DD00BF7148DFF890C100DF7EE0FDB970496D481DF04FFB044668F032FC30B16C4B0A227D210020009407
:40FB000067F0C9FB684966481DF04DFA044668F023FC002865D0644B08227D210020009467F0B9FB5DE0012D1FD15F495C481DF0F4FC044668F010FC30B15B4B0B227D21FF
:40FB40000020009467F0A7FB574955481DF085FC044668F001FC002843D0534B09227D210020009467F097FB3BE0A81E062828D2DFE800F003090F151B2101A948481DF0BC
:40FB80001FF904461EE001A945481DF006FC044618E001A942481DF020FD044612E001A93F481DF051FD04460CE001A93C481DF0D5FE044606E001A939481DF026FF04461C
:40FBC00000E000BF00BFFFF734FF50B1FFF74CFF38B964F065FE0746012201A963F07DFDC6B2012E06D100BF082D04D101202D49087000E00026304641B0BDE8F08370B5AD
:40FC00002A48007888B10820FFF73AFF05464DB10020264908701848007A1949085C1949087202E001202149087020480078C0B9002448E01048005DD0B31248005D401EA7
:40FC400040B21049085500283BDC2046FFF718FF054675B30848005D0949085C094908552FE033E05D091A3432DCE23E49FD080865FC0808A8170010C4180010781A00107D
:40FC800032000020CD1800108C0000100019002081F80808F4030010C9030010280000202015001045000020D61800104400002007E0FFE72DB9082C03D10120FE490870CD
:40FCC00003E0601CC4B2092CB4DB00BF70BD70B50446002500BFF94880F84045012200F5A861F748006800F5027006F0C9F800BF6120F8F7E9FB284670BD70B504460025C6
:40FD000000BFEE4880F83E45012200F23E51EC48006800F2062006F0B3F800BF6120F8F7D3FB284670BD0120E44991F83015032911D1E24991F82815012906D0022906D026
:40FD4000032903D0042903D000BF00BF00BF00BF012000BF00BF704710B52DED028BB0EE408A0024D748008800EE100AB8EE400AB4EEC08AF1EE10FA08DDD248008800EE51
:40FD8000100AB8EE400AB0EE408A0224CE4890ED020AB4EE480AF1EE10FA11D000BF80ED028A042200F10801C548006800F5816006F066F800BF5220F8F786FBFFF7B3FF8E
:40FDC0002046BDEC028B10BD10B5044654B1012C0DD0022C02D0032C13D10DE07F20B94908800FE040F6EC10B64908800AE040F6EC10B449088005E040F2FA20B149088057
:40FE000000E000BF00BF7020F8F75EFB10BD70B504460025A94890F83005A0421BD000BFA64880F83045012200F5A661A448006800F5FC7006F024F800BF2046FFF7C4FF52
:40FE4000A048008800EE100AB8EE400AFFF784FF3D20F8F739FB284670BD70B50446002500BF9648C0F82C45042200F22C519448006800F5FA7006F003F800BF284670BDA9
:40FE800070B50446002500BF8C48C0F83845042200F5A7618A48006800F5007005F0F0FF00BFAE20F8F710FB284670BD70B50446002500BF8148A0F83C45022200F23C5146
:40FEC0007F48006800F5017005F0DAFF00BF284670BD70B50446002500BF784880F83445012200F234517648006800F5FE7005F0C7FF00BF3E20F8F7E7FA284670BD70B5B6
:40FF00000446002500BF6D48A0F83245022200F232516B48006800F5FD7005F0B1FF00BF284670BD70B50446002500BF634880F84947012200F249716148006800F2114091
:40FF400005F09EFF00BF6320F8F7BEFA284670BD10B50120FFF7D1FE0020FFF7B8FE0020FFF7E0FF0420FFF7B4FF4FF6FE70FFF7C6FF0420FFF7ADFF4FF6FE70FFF796FFC0
:40FF80000120FFF744FF012010BD10B54B4890F82805012804D0022807D0032809D100E000BF21F0F1FF044607E024F0DEF8044603E0FFF7CDFF044600BF00BF3D20F8F72B
:40FFC00083FA6120F8F780FA6320F8F77DFA3E20F8F77AFA3F20F8F777FA04213B48DFF8F0C000DF012810D03848007C40F02000364908743748C16B4FF48060DFF8D8C096
:020000040801F1
:4000000000DF3248DFF8D4C000DF204610BD70B504460D46002600BF284880F82845012200F5A5612648006800F5F87005F028FF00BFA220F8F748FA6820F8F745FA3DB12B
:40004000FFF7A3FFFEF751FE4FF4E130FFF718FF304670BD2DED048BA6B0C8274FF00008D8211F4879F001FF502112A879F0FDFE00201C4908731C48DFF870C000DF1C4865
:40008000DFF868C000DF1B48DFF860C000DF1A48DFF858C000DF1948DFF850C000DF1848DFF848C000DF1748DFF840C000DF0C489430DFF838C027E044000020781A0010AB
:4000C0008C00001030000020B0210010B018001049FD08080019002081F8080865FC0808A817001090180010400C001055FC08089011001008120010C8120010181300108E
:400100006C130010B814001000DFFE48DFF8F8C300DFFE48DFF8F0C300DF66F0C9FDFC49C1F88C00002081F8D30001F1A80017F085FFFBF77DF9F74890F84F030A2808D14C
:4001400000210520FFF763FF4FF4E130FFF798FE21E063F027FF40B100210120FFF757FF4FF4E130FFF78CFE15E0EA48D0F83805B0F5966F05D3E748D0F83805B0F5E13F8D
:4001800004D94FF4E130FFF77BFE04E0E149D1F83805FFF775FE4FF4E130FFF75EFEDD4890F83005052808DB0120FFF730FE0120FFF7A3FD0020FFF78AFD64F083FB0646D3
:4001C000D448D0F83815304662F040FD0321D24880F84010DFF844C300DF064631464FF40060DFF83CC300DF00BF0022394641F6FF70DFF830C300DF0546012D7DD0022D47
:400200007BD1DFF824C300DF044604F4805008B1FFF7F5FC04F4006078B163F0C3FE60B10AF0C8FF20B1FFF70CFC0AF0E5FE0FE00AF023FFFFF7D5FB0AE004F4006038B114
:4002400063F0D9FE20B1FFF7F4FB08B1FFF7C9FB04F0040000287DD0FEF78FFB0028FAD01021B248DFF8C8C200DF012873D05022AE49103112A879F09CFDAC48DFF8B4C2CF
:4002800000DFA34818A94EC94EC09DED1C0A103880ED150A66F00CFDA4494866012081F870000A46116E506E66F04CFDA24908609E48406E9D49086602219C4868309E4A18
:4002C00092ED000AB8EE400A17F091FCFFF72CFB38BB8F4890F8C00018B318AA8C49A83104A817F0F2FE9448016804A80AF0BFFA18AA8749A83104A800E0FDE217F05FFF05
:400300000AF0FEFB48B10AF004FC064601F041FA0AF0FFFB0646FBF770FC00200AF0F3FB12E00AF0F3FB78B90AF0F5FB8DED040ACDED050A04A801F02CFA04A8FBF75DFCB9
:4003400001200AF0E0FB00BF714890F8C000F8B16F4801E084E1BBE090F8CF00C0B115F01AFFA8B104AA12A96948FFF7A7F99DED1C0A674880ED160AB8F1000F07D104A86F
:4003800001F007FA04A8FBF738FC4FF001081CE05F4890F8C00020B918A95D48A83017F05CFE5B4818A94EC910304EC09DED1C0A203880ED160A5D4890F8700018B10120E9
:4003C000534981F8D2004FF00008514890F8C00001287DD14E49A831A1F1980017F0CDFE8146B9F1000F23D1494A103202F19801684617F06AFE9DED010AFFEE000A20EE7F
:40040000200A8DED010A9DED000AFFEE000A20EE200A8DED000A3E49103101F1980017F01CFE684601F0B5F96846FBF7E6FB00BF9DED150ADFED410A20EE200ABDEEC00A59
:400440003F4880ED000A00683E490968401A3E4908603B4800683B4908603B480068002807DA394800684EF6602108443649086006E035480068142802DA1420324908602F
:400480009DF87860224A02F1A80104A817F01DFE2D483146026804A801F0A3F81C4A103202F1980102A817F010FE27483146026802A800F0FBFF01F058F9B0EE408A15F0E5
:4004C00044FEB0EE409AF0EE490AB0EE480A00E0BAE0FFF7AAF8B0EE408A0AF06BFE18B1B0EE480A0AF0E0FD094890ED130AB0EE401A154801683046DDED030A9DED020A28
:4005000024E00000B018001055FC0808A0180010A8170010781A001000190020F904090881F80808E1F8080829F808089011001049FD080865FC08081800002000007A44ED
:40054000200000201C00002024000020FBF761F8FBF776FBF0EE408AFE4890F8CF0020B9FBF7C6FB08B1012000E0002082460C21F8489430DFF8E0C300DF01284DD0FBF7D8
:400580009FFB80F00100F34981F8CE00FBF7B0FBF04981F8CF00FAF75EFFEE4981F8D000FAF759FFEB4981F8D1000846C0ED178A80ED188A1E214030B0EE480A17F017FB97
:4005C000FEF7E8FF63F0EEFC78B101F0D6F8E14880ED1A0A01F0D5F8DE4880ED1B0A01F0C8F8DC4880ED190A0AE09FEDDC0AD94880ED1A0A9FEDD90A80ED1B0A80ED198A46
:40060000BAF1000F04D0D348C0ED138A80ED148AD0489430DFF848C300DFD24890F87000012809D1CB4981F8D200CF48416E4FF48050DFF838C300DFFAF7FEFE18B94FF420
:40064000AD703BF0C3FC00BFFEF7CDFDFEF768FDC74A92F83015BF4A92F8CD00FEF7F6FC04F01000F0B1FEF788F9D8B166F020FBC0494862012081F830000A46116A506A5D
:4006800066F060FBBC4908600121BA482830BA4A92ED000AB8EE400A17F0A9FAB548406AB449086204F02000F0B1FEF766F9D8B166F0FEFAB1490864012081F84C00AD4A48
:4006C000116A506A66F03EFBAB4908600121AB484430A94A92ED000AB8EE400A17F087FAA648006CA549C86304F0400010B3FEF744F9F8B166F0DCFAA149C1F83C010120EB
:4007000081F848010A46D2F83811D2F83C0166F019FB9949086001219A48974A92ED000AB8EE400A17F063FA9548D0F83C019449C1F8380104F00800F0B1FEF71EF9D8B134
:4007400066F0B6FA90494862012081F830000A46116A506A66F0F6FA8749086001218A482830854A92ED000AB8EE400A17F03FFA8548406A8449086204F40070D0B3FEF7C1
:40078000FCF8B8B366F094FA80494864012081F850000A46116C506C66F0D4FA7649086001217A484830744A92ED000AB8EE400A17F01DFA7548406C74490864084690EDB5
:4007C0000C0A644880ED1C0A084690ED0D0A614880ED1D0A084690ED0E0A5E4880ED1E0A084690ED0F0ABCEEC00A10EE100A5949A1F8C80004F4806000287DD004216448D6
:40080000DFF854C100DF012876D06148007C00F0020070B14120F7F757FE5920F7F754FE6820F7F751FE5A48007C20F00200584908745748007C00F0080040B16B20F7F75A
:4008400043FE5348007C20F00800514908745048007C00F0040080B1454890F83005032805D19720F7F730FE1A2032F02DFC4848007C20F00400464908744548007C00F0F2
:40088000100040B14020F7F71FFE4148007C20F010003F4908743E48007C00F0200038B1FEF71DFB3A48007C20F02000384908743748007C00F00100B8B3FEF75EF8A0B37B
:4008C00010213448DFF890C000DF01282DD018223049103106A879F06CFA2E48DFF880C000DF2C4890ED050A1A4880ED1C0A294890ED060A174800E01BE080ED1D0A254814
:4009000090ED070A134880ED1E0A224890ED080ABCEEC00A10EE100A0E49A1F8C8001C48007C20F001001A4908741948DFF830C000DFFEF776FAFEF728F8FEF71EF808B1E7
:40094000FDF731FF0349D1F88C0042F2107166F0C9F921E0A817001049FD08080000000065FC0808901100100019002081F80808781A0010EC14001018000020C812001007
:400980006C130010AC140010B814001018130010B01800100017001018B10020FB4981F8D3004020F7F790FD1FE4F84890ED140A7047F648D0ED140AB0EE600A90F8D00060
:4009C00028B1FFEE000A60EE200AB0EE600A7047EE4890ED100A704700B5FEF7A1FF03280BD0FEF79DFF062807D0FEF799FF052803D0FEF795FF042801D1012100E000214F
:400A0000084600BDE14890F8CD007047DF4890F8D200012804D1DE48007808B9012070470020FCE7DA48007B012800D170470020FCE7D748007B032801D1012070470020DD
:400A4000FCE7D348407B082801D1012070470020FCE710B52DED028BCE4890F878430E2C20D2DFE804F01F20212216151407251F1F1F232403F004FFF0EE408A03F0D8FE3C
:400A8000F0EE000A80EE201A38EEC18A15E000BF00BF03F0F5FEF0EE408A03F0C9FE38EEC08A0AE000BF00BF00BF00BF00BF00BF03F0E6FEB0EE408A00BF00BFB0EE480AF9
:400AC000BDEC028B10BDB44909680143B24A1160704770B50446002500BFAE4880F83F45012200F23F51AD48006800F2072005F0C7F900BF6120F7F7E7FC284670BD70B537
:400B00000446002500BFA34880F83545012200F23551A248006800F2FD1005F0B1F900BF3F20F7F7D1FC284670BD70B504460025072C01DD07240225964890F85007A04215
:400B400017D000BF934880F85047012200F5EA619248006800F5836005F092F900BF7720F7F7B2FC8E48C16B4FF40060DFF834C200DF284670BD70B504460025072C01DD65
:400B800007240225834890F85107A04217D000BF804880F85147012200F251717F48006800F2194005F06CF900BF7820F7F78CFC7B48C16B4FF40060DFF8E8C100DF284601
:400BC00070BD70B504460025072C01DD07240225704890F85207A04217D000BF6D4880F85247012200F252716C48006800F21A4005F046F900BF7920F7F766FC6848C16BF2
:400C00004FF40060DFF89CC100DF284670BD70B504460025072C01DD072402255D4890F85307A04217D000BF5A4880F85347012200F253715948006800F21B4005F020F96C
:400C400000BF7A20F7F740FC5548C16B4FF40060DFF850C100DF284670BD70B504460025072C01DD072402254A4890F85407A04217D000BF474880F85447012200F25471B3
:400C80004648006800F21C4005F0FAF800BF7B20F7F71AFC4248C16B4FF40060DFF804C100DF284670BD70B504460025072C01DD07240225374890F85507A04217D000BF5A
:400CC000344880F85547012200F255713348006800F21D4005F0D4F800BF7C20F7F7F4FB2F48C16B4FF40060DFF8B8C000DF284670BD70B504460025072C01DD0724022558
:400D0000244890F85607A04217D000BF214880F85647012200F256712048006800F21E4005F0AEF800BF7D20F7F7CEFB1C48C16B4FF40060DFF86CC000DF284670BD38B515
:400D40000446204678F07AFF052860D3052216A1204678F023FFC0B9154878F06FFF0546134B042221210090002066F094FA11A00AF0C5FE00200FF010FD9E20F7F7A4FB7E
:400D80004FF4C3703BF022F941E015E0A817001090180010781A00102C0000208C0000100019002081F808084345535452000000FC1B0010000000000522FEA1204678F052
:400DC000EDFE20BB63F05BFD054620F0A0FE00BFFA48AFF22001097880F8C0113C2200F5E071F74805F04CF800BF6820F7F76CFBFF2003460322012100903D20FAF7AFFA0E
:400E00004FF48070FFF75FFE6820F7F75DFB38BD10B5EC48FFF793FF30224021EA4878F0FAFF0622E749E84879F046F82C20E64988710622E349C91DE348C01D79F03CF820
:400E40002C20E14948730622DE490E31DE480E3079F032F82C20DC4908750622D9491531D948153079F028F82C20D749C8760622D4491C31D4481C3079F01EF82C20D249C5
:400E800081F82200CF48233078F0D8FEC4B2621CCC492331CC48233079F00EF8C94890F82E0070B1C84878F0C9FEC4B22C20C6490855601CC4B208190722C2492E3178F059
:400EC000FBFF2020FFF7FFFD10BD10B504462046FFF735FF204678F0B1FE402803D82146B94878F087FE2020FFF7EDFD10BD70B504460025032C01DD03240225AF4890F8EA
:400F00009807A04210D000BFAC4880F89847012200F5F361AD48006800F58C6004F0B0FF00BFBC20F7F7D0FA284670BDA648704770B50546A14890F82805012802D0032832
:400F400006D100E000BF284620F07CFF044602E0AFF2A01070BD00BF2046FBE770B50546964890F82805012806D002280AD0032803D0042810D10AE000BF284620F08AFF90
:400F800004460CE0284623F04AF8044607E028461AF049FD044602E0AFF2E81070BD00BF2046FBE710B5854890F82805012806D0022809D0032803D0042804D105E000BF64
:400FC00021F04FF804E000BF00BF9FED810A00BF00BF10BD0020704710B5784991F82815012904D0022906D0032907D100E000BF20F0B3FF04E022F07CFE01E0002000BF1E
:4010000000BF10BD2DE9F04781460D461446C846002600270FE02C21404678F0A3FD064626B9AF4201DA4FF0000806E0AF4201DA06F101087F1CAF42EDDD00BFB8F1000F81
:4010400009D01EB1A6EB0800207006E0404678F0F5FD207001E0002020702078102801DC207810B94FF0000800244046BDE8F08700B5FFF7CBFC08B9002102E05548B0F822
:40108000C810084600BD4D4890F85707704710B5044600BF494880F85747012200F257714A48006800F21F4004F0EAFE00BF8120F7F70AFA002010BD4048B0F8E20400EE5F
:4010C000100AF8EE400A9FED441A80EE810A7047404890F8D30070470146052911D2DFE801F00305070A0D0000200AE03C2008E04FF4967005E04FF4167002E04FF4B460BE
:4011000000BF00BF70473EB5054600BF2B4880F80051012200F580712948C03804F0B0FE00BF00200290254991F80001FFF7D4FF0446E0B28DF80800200A8DF809000220B8
:4011400002A903461922CDE900100021084666F0D0F83EBD2148406870472049486070471E4890ED020A70471C4880ED020A70471A48407B70471948007B704710B50446B2
:401180000E4890F82903A04231D000BF0B4880F82943012200F22931114804F071FE00BF7120F7F791F90F48C16B4FF40060DFF838C01BE04345475053000000781A001055
:4011C000C001006870170010301700108C00001000000000A817001000007A4490180010290300680019002081F8080800DF10BDF0B52DED0C8B85B0B0EE408AF0EE608A3A
:4012000001279FED950B53EC102B51EC180B7FF063FD0AD2BF1EB0EE480AF0EE680A7BF0ABFFB0EE408AF0EE608AB0EE480AF0EE680A7BF0ADFFB0EE409AF0EE609A51EC8F
:40124000190B7FF07BFC44B220467FF0D4FC53EC182B7FF0B1FE9FED820B53EC102B7FF077FD41EC1A0BB0EE4A0AF0EE6A0A7BF08FFFB0EE409AF0EE609A51EC190B7FF004
:401280005DFC45B2C5EB051188007FF0B4FC41EC1A0B20467FF0AFFC53EC182B7FF08CFE9FED710B53EC102B7FF052FD53EC1A2B7FF05AFF7FF0C0F90646304680F03EF808
:4012C00041EC190B8DED029B04FB07F368A20F216A48009578F062F9684805B0BDEC0C8BF0BD67480078012800D170470020FCE763480078022801D1012070470020FCE722
:4013000010B504465E480470AF20F7F7DDF810BD10B5044621465B4878F06CFC0B225949594804F0ADFD10BD10B50446214655480B3878F05FFC0B2252490B3952480B385F
:4013400004F09EFD10BD10B5504991F82815012906D0022908D0032903D0042908D105E000BF20F082FE05E0002003E0002001E0002000BF00BF10BD0020444991F82815EA
:40138000022900D1012070470020404991F82815042900D10120704710B500243B4890F82805012806D002280AD0032803D0042805D106E000BF20F05BFE044603E000BFF6
:4013C00000BF002400BF00BF204610BD2F4890F82903022801D1012070470020FCE710B5FFF714FB48B12A4890ED120ADFED290AB4EE600AF1EE10FA05D1274A27A1284816
:4014000078F0B6F806E0224B4C3324A20C21244878F0C4F8224810BD10B51D4890ED120ABCEEC00A10EE100A80B2FF2805D11A4A1AA11C4878F09CF80CE0154890ED120A2B
:40144000BCEEC00A10EE100A83B217A20421154878F0A4F8134810BD00000000000000000000000000004E40000000000020AC4025642A256427252E32662200D61900103B
:4014800028000020851B00100D010068781A00109011001000007F4384EF000825730000E5190010460000202575000070B52DED048B84B004460E461546BF480078B0421C
:4014C00002D1B5F5FA7F08DDBB4806700020BB49087004B0BDEC048B70BDB848007838B9B748D4E9001206C00120B4490870F0E70A2D00DAEDE700EE105AB8EEC00ADFED00
:40150000B10AC0EE808A94ED010AAD48D0ED010A30EE600A20EE280A8DED030A94ED000AD0ED000A30EE600A20EE280A8DED020A9DED030AA448D0ED010A30EE600A8DEDB3
:40154000010A9DED020AD0ED000A30EE600A8DED000A9E4890ED000A0AF099F910B19FED9C0A01E09FED9B0AB0EE409A964890ED010ADDED010A00EE890A80ED010A90EDD0
:40158000000ADDED000A00EE890A80ED000A17F0F3F9B0EE408AB0EE480A0AF078F910B1B0EE480A01E09FED8C0AB0EE408A9FED8B0AB4EEC08AF1EE10FA02DD9FED860A92
:4015C00001E0B0EE480A814880ED000A94ED010A7B4880ED010A94ED000A80ED000A00BF77E770B52DED048B84B005460E4614467B480078B04202D1B4F5FA7F08DD784832
:40160000067000207749087004B0BDEC048B70BD7448007838B97449D5E9000205C1012070490870F0E70A2C00DAEDE700EE104AB8EEC00ADFED630A80EE808A95ED010A58
:401640006948D0ED010A30EE600A20EE080A8DED030A95ED000AD0ED000A30EE600A20EE080A8DED020A9DED030A6048D0ED010A30EE600A8DED010A9DED020AD0ED000AD0
:4016800030EE600A8DED000A594890ED000A0AF0FEF810B19FED4E0A01E09FED4E0AB0EE409A524890ED010ADDED010A00EE890A80ED010A90ED000ADDED000A00EE890A58
:4016C00080ED000A17F058F9F0EE408AB0EE680A0AF0DDF810B1B0EE680A01E09FED3E0AF0EE408A9FED3D0AF4EEC08AF1EE10FA02DD9FED390A01E0B0EE680A3C4880EDEE
:40170000000A00EE104AF8EEC00A9FED2E1A81EE200AD0ED000A374890ED001A70EEC10A20EE200A344880ED000A90ED000A3348D0ED000A70EE600A90ED000AB6EE001A33
:4017400000EE810A80ED000A95ED010A264880ED010A95ED000A80ED000A254890ED000A244880ED000A00BF4EE7184890ED000A70471F4890ED000A70471F4890ED000A07
:4017800070471E4890ED000A704700200B49087070470B4991ED010AD0ED010A30EE200A81ED010A91ED000AD0ED000A30EE200A81ED000A7047000051000010500000103E
:4017C0003C00001000007A44440000104C000010CDCC4C3F90C2753E00000000CDCC32427500001074000010540000105C00001064000010680000106C0000107000001038
:4018000070B5F64804780125F548007806285BD2DFE800F003041905265B5AE000BFF148407F20B10120ED49087001250AE0ED4890F83D0018B10320E849087002E0002004
:40184000E649087045E0E74890F82D0020B10220E2490870012502E00020E049087038E0E04890F82D0020B10220DC490870012529E0DC48407F78B10120D8490870D948BE
:4018800090ED040AD848D0ED000A30EE600AD54880ED040A012516E0D24890F83D0078B10320CE490870CF4890ED0C0ACE48D0ED000A30EE600ACB4880ED0C0A012502E013
:4018C0000020C649087004E000BF0020C349087000BF00BFC1480078A04205D0BD20F6F7F3FD072031F0F0FB35B1C048D0F854110120DFF8FCC200DF70BD70B504460025E6
:40190000052C01DB022519E0002C01DC032515E0B348047000BFB74880F89947012200F29971B548006800F2614004F0A9FA00BFBE20F6F7C9FD072031F0C6FB284670BD2D
:4019400010B51620F6F7C0FD5020F6F7BDFD1720F6F7BAFD1820F6F7B7FD252031F0B4FB10BD4FF416770121A04880F8541022F02BFC804622F070FF23F042F9FFF7E0FFBC
:401980000020964908709B4890F89907944908700846007818B108460078052802DB0120FFF7ABFF904800210160416000240AE000208C4901EB041108738A4901EB0411E2
:4019C0004873601C84B2052CF2DBDFF830C200DF81466922012165F04AFA30B1DFF81CC200DF8146012165F071FADFF810C200DF814649460220DFF8F8C100DFB8F1000F82
:401A000074D10321794880F8541000BF002239460720DFF8ECC100DF0546012DF6D0022DF4D1DFF8E0C100DF0646304622F00CFC304622F01CFF304623F0F2F806F0010043
:401A40000028E3D0674A1832111F081F22F09CFD6449487701F138023431081F22F04FFF604981F83D0001F128022431081F23F016F95C4981F82D0009F09DFF40B909F01F
:401A8000C1FF28B909F0B1FF10B909F0A1FF08B3544890F82D00012824D15248407F012809D15048D0ED040AB0EE600A19214E4816F09DF816E04B4890F83D00012811D1C5
:401AC0004848D0ED0C0AB0EE600A1921464816F08EF807E09FED4C0A434880ED000A002041494860FFF78CFE90E7FFE70020DFF81CC100DF00BFFEE73848007808B1012004
:401B000070470020FCE72DE9F05F2DED028BB0EE408A05460F46904699460C9E4FF0000BDA460FFA88F445E0A21905EBC20105EBC40016F0D5FEF0EE408AF4EEC88AF1EEAE
:401B400010FA2FDDC8EE280AB0EE600AA01905EBC000D0ED010A05EBC40090ED011A30EEC11A05EBC400D0ED010A41EE000AC7ED010AA01905EBC000D0ED000A05EBC40091
:401B800090ED001A30EEC11A05EBC400D0ED000A41EE000AC7ED000AA14678EE680AB0EE608A0EE038EE680AB0EE408AA01904B20AF1010A04FB06F0484502DABAF1280F39
:401BC000B2D300BFB5EEC08AF1EE10FA01DD4FF0010B5846BDEC028BBDE8F09F4D0000204C000020F4190010500000200019002081F80808781A00108C000010F904090826
:401C0000E1F8080829F80808000000003D0309082DE9F04F2DED028B83B005460E4691469B46F0EE408ADDE90E4A00200290AAF10100A04201D2044602E0002C00DA002494
:401C400006EBC401284616F04BFEB0EE408AB4EEE88AF1EE10FA28D2109858B9BBF1000F03D000274FF0FF380FE0AAF101074FF001080AE0BBF1000F04D0AAF101074FF079
:401C8000010802E000274FF0FF3838EEC80AF0EE408A3B46224649463046B0EE680ACDF80080FFF730FF029020E0C8EE880AB0EE600A06EBC400D0ED010A95ED011A30EE7A
:401CC000C11AD5ED010A41EE000AC9ED010A06EBC400D0ED000A95ED001A30EEC11AD5ED000A41EE000AC9ED000A00BF029803B0BDEC028BBDE8F08F2DE9FF4F2DED020B7B
:401D00002DED068B8BB00E461746F0EE408A99464FF0000AF2EE020AB2EE040A7CF054F9B0EE40AA1FED480AB0EE408A07F10C040025B9F1020F02D24FF0010A85E14FF0F0
:401D4000000B2BE01398D0ED010A06EBCB0090ED011A70EEC10AB0EE600A16F0BFFBB0EE409A1398D0ED000A06EBCB0090ED001A70EEC10AB0EE600A16F0B0FB39EE000A45
:401D8000B0EE408AB4EECA8AF1EE10FA02D25D46B0EE48AA0BF101000FFA80FBCB45D1D3A846A9F1010000B205900598804503D1A8F101000FFA80F808F1010206EBC201CF
:401DC00006EBC80007F1500217F0D2F8B0EE408AB5EEC08AF1EE10FA01D2012000E0002087F8580097F8580010B14FF0FF3000E001200690B5B96A1C06EBC20106EBC500FB
:401E0000139A17F0CAF8B0EE408AB5EEC08AF1EE10FA01D24FF0010A97F8580078B3681C05B22CE00598854216D16A1E06EBC20106EBC500139A17F0B0F8B0EE408AB5EED4
:401E4000C08AF1EE10FA01D24FF0010A97F85800A8B9681E05B212E0069A2A4406EBC20106EBC500139A17F098F8B0EE408AB5EEC08AF1EE10FA02D20698281A05B206EB45
:401E8000C50103C9C4E905010698284406EBC00106C9C4E9071204F11C0204F1140104F1240016F0E1FF657094ED090A8DED040A94ED0A0AB1EE400A8DED030A03AA04F1D8
:401EC0001401139817F086F8B0EEC00AB0EE408A94ED060AD4ED0A0A08EE200A84ED020A94ED050AD4ED090A08EE200A84ED010AD6E90001CDE90701D6E90201CDE90901CA
:401F00009DED0A0ADDED080A30EE600A84ED040A9DED090ADDED070A30EE600A84ED030AD6E90001C4E90B01D6E90212C4E90D12D6E90212C4E90F12B9F1020F7ED9BAF12C
:401F4000000F7BD1387A00EE100AB8EE400AF7EE080A20EE200AB0EE409AA8460120CDE90089029097F85830B0EE490A07AA3146201DFFF74DFE40EA0A0A069828440FFAD6
:401F800080F80020CDE90089029097F85830B0EE490A09AA3146201DFFF73AFE40EA0A0A9DED0A0ADDED080A30EE600A84ED040A9DED090ADDED070A30EE600A84ED030ADE
:401FC000A846787A00EE100AB8EE400AF7EE080A20EE200AB0EE409A0120CDE90089029097F85830B0EE490A04F12C023146201DFFF70EFE40EA0A0AD4E90112C4E90D12B5
:40200000069828440FFA80F897ED010A20EE280AF0EE409AF4EEC99AF1EE10FA01DDB0EE699A0020CDE90089029097F85830B0EE490A04F13C023146201D00E004E0FFF747
:40204000E7FD40EA0A0A00BF00BF50460BB0BDEC068B06B0BDE8F08F10B52DED028BF0EE408A044694ED001AF0EE410A94ED011AB0EE410A16F052FAB0EE408A38EE680A62
:40208000B0EE408A06E0AF4890ED000A38EE000AB0EE408AAC4890ED000AB1EE400AB4EEC08AF1EE10FAEED306E0A64890ED000A38EE400AB0EE408AA34890ED000AB4EE7B
:4020C000C08AF1EE10FAF0DCB0EE480ABDEC028B10BD10B59D48016D012064F02DFF9B48016D0120DFF868C200DF10BD99489A49097800EB0110407B38B1964896490978F3
:4021000000EB011090ED010A70479FED940AFBE790489149097800EB0110407B38B18D488D49097800EB011090ED000A70479FED8B0AFBE787488849097800EB0110407B44
:4021400038B184488449097800EB011090ED020A70479FED820AFBE701468148B0F8E20400EE100AB8EE400ADFED7E0A30EE600ADFED7C0A80EE201A81ED001A784890F8EA
:40218000E02400F2E44000EB8202754890F8E10432F8100000EE100AB8EE400ADFED710A30EE600A9FED6F1AC0EE010AB0EE000A30EE800A81ED010A694890F8EC04087231
:4021C000674890F8EE0448720120704762480078704770B504460025B4F57A7F03DD4FF47A74022503E0002C01DA0024032500BF5B48A0F8E244022200F2E2415A48006844
:4022000000F5D57003F03CFE00BF1620F6F75CF9252030F059FF4D48016D0220DFF830C100DF284670BD2DE9F04104460D4616460027B4F5FA7F03DD4FF4FA74022703E0B6
:40224000002C01DA00240327484800EB850030F81600A04222D000BF444800EB850020F81640424A02EB850202EB46013E4A126802F5D67202EB850202EB4600022203F09B
:40228000FFFD00BF5020F6F71FF9252030F01CFF2E48016D0220DFF8B8C000DF3846BDE8F08170B5044600250A2C02DD0A24022503E0012C01DA0124032500BF2848A0F8A9
:4022C000EC44022200F2EC412748006800F5DA7003F0D6FD00BF1720F6F7F6F8252030F0F3FE1A48016D0220DFF864C000DF284670BD70B5044600250A2C02DD0A24022503
:4023000003E0012C01DA0124032500BF1448A0F8EE44022200F2EE411348006800F5DB7003F0AEFD00BF1820F6F7CEF8252030F0CBFE0648016D0220DFF814C000DF2846EC
:4023400070BD0000E46B0A08E06B0A080019002081F80808F41900104D00002000000000781A00100000C8428C0000105C1F001010B50220FE4908700020087164F098FC2C
:40238000FB498860002088600120487041F288304880012008750021F548017664F088FCF349C8610021F248C1610121417541F28831C182152141620220EE49087010BDB2
:4023C00010B5ED480078ED490870ED4800784870EC4800788870EC480078C870FFF7C8FF10BD0421018000214180012181800021C1800181704770B50446042C01DD002063
:4024000070BD44BBE148B0F87E0728B9DF48B0F8800708B9012523E0D748007862F03BF800EE100AB8EE400ADFEDD90A20EE200ABCEEC00A10EE106AD448B0F87E07B042D7
:4024400006D8D248B0F88007B04201D3012000E00020054604E0C949085D62F099F9054694B925B164F024FCCA4908600CE064F01FFCC8490968401A41F65831884201D2D3
:40248000012000E0002005460DB10120B8E70020B6E770B504460025012C11DA84B9B648007861F0F8FF00EE100AB8EE400ADFEDB80A20EE200ABCEEC00A10EE100A85B24D
:4024C000284670BD2DE9F04106463007070E042F02DD0020BDE8F0810025002410E03819042805DAA549085D62F052F9804601E04FF00308610008FA01F00543601CC4B216
:40250000102CECDB2846E5E72DE9F0470746884615461E464FF00009002448E004EB8400934911F82000B84240D104EB840001EB80000079404539D14FF00109012D00D0F2
:402540005EB104EB84008A4901EB8000457004EB840001EB8000468028E086480078401EA04206D1002004EB8401814A02F8210017E0804A1278521E02EB82027C4B03EB80
:40258000820104EB840203EB8200142277F011FC002178480078401E00EB8000744A02F8201074480078401E72490870641CB9F1000F03D16F4800788442AFDBB9F1000FF5
:4025C0002ED16C480078202802D10120BDE8F087012D00D016B36748007800EB8000644901F820706348007800EB800001EB800080F804805F48007800EB800001EB8000DD
:4026000045705C48007800EB800001EB8000468058480078401C5749087001E00220D5E70020D3E77CB5002600250024CEE0002604EB84004E4911F8200000B9C9E004EB0F
:4026400084004B4901EB80004088B0B104EB84020B4603EB8202518804EB840203EB8202D06864F03FFB40B164F022FB04EB84013F4A02EB8101C86001263EB904EB840068
:402680003B4901EB80004078012819D104EB8400374911F82000022809D104EB8401344A02EB81010879FFF70DFF054608E004EB84012F4A02EB81010879FFF79CFE054670
:4026C000A6B904EB84002A4901EB8000407801280CD104EB840001EB80008068A84205D004EB840001EB800085600126F6B304EB84001F4911F82000022816D104EB8400C9
:4027000001EB800001799DF8000061F387108DF800009DF8000020F03E008DF80000CDF80150684630F082FB4EE004EB8401104A02EB81010879C11700EB117109119DF805
:40274000042061F347128DF8042004EB8401084A02EB81010879C11700EB11710911A0EB01119DF8042061F3440215E02CE00000241200207C000010070400107800001054
:40278000060400100504001008040010781A001000404E3F800000108DF804209DF8050065F301008DF8050004EB84000F4901EB8000007C9DF8051060F387018DF80510D3
:4027C00001A830F03BFB00BF601CC4B2202CFFF62EAF00BF7CBDFFF7F3FD05E0FFF722FF2820DFF80CC000DFF8E700002412002021F80808FE490870704770B504460D46D1
:40280000E21704EBD2625311FA4A02EB830212682146E31704EBD3635B11A4EB43160123B3401A432046E31704EBD3635E11F14B03EB86031A60F04804702846FAF779FCF9
:402840001F2D03D029460C2064F0A8FC002C3DD00421EA48DFF8A8C300DF012818D0E74890F82E1090F82E00401CE44A82F82E0002F110004454103890F82E001E2803DB4A
:402880000020114681F82E00DC48DFF878C300DF0421DD48DFF868C300DF012816D064F007FADA4941F83400084600EBC4000079FF2807DA084600EBC4000079401C01EB8A
:4028C000C4010871D048DFF83CC300DF1E2030F0FBFB70BDCE48007F012800D170470020FCE7CB48407F08B9012070470020FCE710B56FF01BFC01280FD16FF0F7FB60B1EF
:402900006EF07CFB012808D174F07EFC012804D1FFF7E7FF08B1012010BD0020FCE770B50446607B01281FD1A06868B1D4E9010164F0D8F900286AD000221146204617F0AE
:4029400032FE0120E07362E04FF4FA61606864F0C9F900285BD00220A0731C210820FFF74CFF09F0A7F852E0A07B022802D10020A0734CE0207B012849D10020E07309F03C
:402980001AF828B909F024F810B909F03BF830B109F090F81D210320FFF72FFF37E0FFF7A7FF48B1FBF7D7FD30B909F077F820210020FFF722FF2AE06EF020FB012804D078
:4029C0001F210420FFF719FF1FE06FF0AFFB012804D012210320FFF710FF16E06FF086FB20B911210120FFF708FF0EE0FBF7B3FD38B1FBF7BEFD054629460920FFF7FDFE0C
:402A000003E01E213120FFF7F8FE09F053F8207B617B884202D03820F5F756FDE07B08B9607B207370BD00207A4908707047F0EE400A9FED791A20EE811AB0EE410A9FED1B
:402A4000771A30EE011AB0EE410AB1EE001A20EE011AB0EE410AB6EE001A30EE011AB0EE410A9FED6F1AB4EEC10AF1EE10FA03DD9FED6B1AB0EE410ABCEEC01A11EE100A16
:402A800080B27047674800780B2801D1012070470020FCE7634800780C2801D1012070470020FCE75F480078012800D170470020FCE75C480078092801D101207047002038
:402AC000FCE758480078062801D1012070470020FCE700B52DED028B81B0534890F82200012820D1504890F8230001281BD1FFF7E8FF58B9FFF7DDFF40B9FFF7D3FF28B95A
:402B0000FFF7C8FF10B9FFF7BDFF38B10120464981F8240064F0CCF8434948600020424981F823004EE04049086864F0FCF8B0F57A7F47D33C4890F82200012842D10421DE
:402B400039480830DFF8B8C000DF01283AD0DFED370A9FED360A73F06BFBB0EE408AFFF766FF31494883DFED310A9FED300A73F05FFBB0EE408AFFF75AFF2B490883012030
:402B800081F820000220C8770020087702208877002048774520F5F797FC0020224981F82200012081F82300FFF73DFF1E480830DFF850C000DF1E48D0F81C120120DFF8CB
:402BC00074C000DF184890F82400D8B31649486864F0A9F840F6C411884248D3164800680090164890F8E0241548032103682AE06A00002035170020600000200417002050
:402C000049FD080865FC0808F4160020F4140020A41400206B00002000007A440000FB4500FF7A475D000020CC140020000000000019002081F80808DC030020781A00107A
:402C4000D803002013E0FB4835F030F8FA4800680090FA4890F8E124F94803210368F548973035F023F80020F64981F8240001B0BDEC028B00BDF4480078C0F3800070477B
:402C8000F1480078C0F340007047EF48007800F001007047EC480078072801D1012070470020FCE7E9490870704710B502F026FC30B1002213466021E54823F0BFFA3AE0B0
:402CC00002F087FC30B1002213462721E04823F0B5FA30E002F02CF930B100221346D221DC4823F0ABFA26E002F08BFC30B1002213460621D64823F0A1FA1CE002F03FFC88
:402D000030B1002213463121D14823F097FA12E002F042FC30B1002213460621CC4823F08DFA08E002F0F2FB28B100221346FC21C74823F083FA10BD10B5002402F0DEFB7D
:402D400070B902F01CFC58B902F026FC40B902F0DDFB28B902F0ECF810B902F052FC00B10124204610BD70B504460225102C02DA0025B94804708420F5F7A6FB284670BD5B
:402D800010B502F0BBFB88B10820FFF7ECFF002213461321B14823F051FAB048A8490860AF48A54908600020AB49887002F0AEF888B10D20FFF7D7FF002213461321A7484C
:402DC00023F03CFAA5489E490860A5489A4908600020A149887002F0ECFBC0B10E20FFF7C2FF00221346F0219C4823F027FA00221346F0219948C03023F020FA97489049FF
:402E0000086097488C49086000209349887002F0D8FBA0B10F20FFF7A6FF0022134627218E48C03023F00AFA8C48C030844908608B4828308049086001208749887010BD8F
:402E400010B50020FFF78FFF01217D48006823F010FA02208049887010BD10B5002402F04DFB40B902F0ADFB28B902F0A2FB10B902F04CF800B10124204610BD734800786C
:402E8000704710B50121774823F0F3F910BD10B52DED028B6B48408B00EE900AF8EE600AB0EE600A0521704814F0A1FE6E4890ED000AF6EE000A30EE200ABCEEC00A10EEB9
:402EC000100A84B264480078102878D2DFE800F0D139780809D03A0A0B5F0C4C4D0D0F0E00BF00BF00BF00BF00BF00BF00BF08F062FD40B908F086FD28B908F076FD10B92C
:402F000008F066FDE0B1FDF750FDB0EE408A08F0BEFC30B9FDF749FDB0EE408A6BF08CFA70B16FF06CFBDFED510AC0EE208A71F0ECFF38EE800AB0EE408AFFF778FD04465F
:402F40009AE000BF08F037FD68B1FDF72EFDB0EE408A08F09CFC30B106F058FFB0EE408AFFF765FD044687E000BF08F024FD68B1FDF71BFDB0EE408A08F089FC30B106F064
:402F800052FFBCEEC00A10EE100A84B274E008F012FD98B1FDF709FDB0EE408A08F077FC60B106F033FFF0EE408A73F0A3FD38EE800AB0EE408AFFF73AFD04465CE057E0A7
:402FC0006CF0B0FD07280FD2DFE800F00508040F06070B0000BF00BF00BF00BF4FF6FF7426E01848048B23E000BF08F0E4FC40B908F008FD28B908F0F8FC10B908F0E8FC1E
:40300000A8B1FDF7D2FCB0EE408A08F040FC70B16FF0F5FADFED150AC0EE208A71F075FF38EE800AB0EE408AFFF701FD044600BF00BF21E058010800DC030020781A00107B
:40304000D8030020CC1400206B0000205C000020E8790220287902205D000020A8740220E87C0220A87A02201002002000007A4500BF4FF6FF7400BF00BF2046BDEC028B01
:4030800010BD502600274FF000080020F84908700121F84880F88011F748DFF8E0C300DFF748DFF8D8C300DFF648DFF8D0C300DF08F077FA0020F049083981F822000120AD
:4030C00081F82300002081F82400FFF74CFE0220ED4988700020FFF7E5FD6FF074F90020EA4908700321E34880F8801100BF002231460720DFF898C300DF84B2022C0DD12E
:40310000DFF890C300DF074607F0020030B1FFF7BEFEE149088001202FF0D6FF012C7DD1DE4890F88503092803D150206CF081FD00E000BF00BF01F0E9FE60B10120D8495D
:4031400048706AF0C6FD30B96AF017FF6AF0C1FD08B1FFF796FE36F07BFEE0B10CF044FBC8B109F09BFA142803D009F097FA152811D1FFF783FE70B9FFF76FFE18B1FFF7DA
:403180005FFEFFF7FDFDFFF7D7FD08B1FFF78DFD0120FFF787FDFFF794FC58B9FFF789FC40B9FFF77FFC28B9FFF774FC10B9FFF769FC80B3FFF76EFD68BB404663F0B3FDFD
:4031C00042F21071884226D3FFF75FFD40B9B5480368B548002102684FF6DA602AF0E9FDFFF74EFD40B9AF480368AF48002102684FF6C5502AF0DDFDFFF73DFD40B9A94817
:403200000368A948792102684FF46F402AF0D1FD63F04EFD80461021974800E08DE0DFF88CC200DF012809D0282293490839A04876F0BFFD9048DFF87CC200DFFFF749FC15
:403240006FF09FF89C48FFF76AFB9C48FFF767FB9B48FFF764FB9B48FFF761FB9A48FFF75EFB9A48FFF75BFB9948FFF758FB6AF0F9FA6CF0F7F908F09EFB40B908F0C2FB0F
:4032800028B908F0B2FB10B908F0A2FB08B1012000E0002005466DF0B1FE012806D008F009FC1DB11F210320FFF7A7FABDB3012088490870FFF715FB30B1FFF70BFB20BB9D
:4032C00085480078142820DB08F0F4FB6EF02EFF012804D012213420FFF78FFA2BE06EF005FF20B911213420FFF787FA23E06DF085FE012804D01F213420FFF77EFA1AE0BE
:403300001E213420FFF779FA15E073480078142811DA71480078401C6F4908700BE0FFE76C48007838B10020FFF764FA00206A4908706849087008F045F90027D7E64E4807
:40334000083890F8220008B9012070470020FCE710B50D21614876F088FD10BD70B50023012115E0CC1701EBD46465115B4C641C04EB85042468CD1701EBD5656D11A1EB58
:4033800045160125B5402C4004B10B46481CC1B24029E7DB184670BD4548807F70474448C07F704738480078022801D1012070470020FCE710B5FFF7F5FF18B16CF0B8FB7D
:4033C000044602E03A4890F82140204610BD324800887047B0F57B4F01DB4FF6FF2000EE900AF8EE600AB1EE001AC0EE811AB0EE610ADFED3B0A70EE600AB0EE600ADFED0B
:40340000390A80EE201AB0EE410A70471A480838408B704710B51648007808B1FF2010BD08F0C9FA40B908F0EDFA28B908F0DDFA10B908F0CDFA08B1012000E0002020B127
:403440000B48007808B9012000E0002040F0FC00E5E70D4800780D2801D1012070470020FCE7094800780E283ED10120704700006A00002000190020D414002055FC0808E6
:4034800004170020F41600205D0000206B000020E1F8080829F8080868000020781A0010E87C0220DC030020D803002049FD0808A414002065FC080824DB001034DB00100E
:4034C00044DB001054DB001064DB001074DB001084DB00100D0200200C020020341700200000FB4500007A44002070472DE9F0472DED048B07460C4692469846DDF83090C4
:4035000001F016FD30B1A078FD2803D1BDEC048BBDE8F087FFF7A5FF28B1FC480068C078404500D0F2E70025FFF793FF18B120466AF004FC0DE0B7F52C4F01D1002508E093
:40354000B7F56F4F04D12078AC2801D1012500E0DCE75021EE48DFF8BCC300DF012865D0615D681C205C41EA0026E94808380683B6F57B4F16DBFDF71CFAF0EE408A12F0A8
:40358000E4FDB0EE409AF0EE680A72F051FEB0EE408AFFF74CFADE4908394883012081F8200007E0DA48083846830020D849083981F82000A81C205C00F00300D449083962
:4035C000C877A81C205CC0F381000877A81C205CC0F301108877A81C205C8009487763F067FBCB4908390860012081F82200E81C205C400981F82100C548DFF81CC300DFDB
:4036000001F05CFC58B1C548016D012063F094FCC248016D0120DFF808C300DF06E0BF48D0F81C120120DFF8F8C200DF00BF6DE7BC48007808B1012070470020FCE770B5E3
:4036400004460025B84890F84F03FF2800D18CE0092C06D1B44890F88403032801D0012583E0012C06D1B04890F88403032801D001257AE0062C06D1AB4890F88403032844
:4036800001D0012571E0042C14D1A74991F84F0301F021FF07280BD0A34890F87C03172808D1A14991F84F0301F015FF012801D101255AE0072C14D19B4991F84F0301F0D0
:4036C0000AFF08280BD0984890F87C03172808D1954991F84F0301F0FEFE012801D1012543E0022C14D1904991F84F0301F0F3FE09280BD08C4890F87C03172808D18A4952
:4037000091F84F0301F0E7FE012801D101252CE00A2C14D1844991F84F0301F0DCFE0B280BD0814890F87C03172808D17E4991F84F0301F0D0FE012801D1012515E0032C81
:4037400013D1794991F84F0301F0C5FE0A280BD0754890F87C03172807D1734991F84F0301F0B9FE012800D10125284670BD10B5012401F0C3FE00B10024204610BD70B569
:4037800004460E460025FFF7F2FF002841D001F095FB28B10B2C01D00C2C3AD1012538E0D6B9012C03D0092C01D0062C08D12046FFF745FF054605B300205A49887028E03D
:4037C00058488078C8B12046FFF739FF0546A5B10020544988701CE05248807868B1012C03D0092C01D0062C08D12046FFF727FF054615B101204B4988700AE0FFF718FFDF
:4038000038B92046FFF71BFF054615B1012045498870012D04D1FFF70BFF08B1FFF710FB284670BD2DE9F0418CB0074688460025002F6AD0F220012102220023CDE905327D
:40384000CDE90710042010210193CDE90231049097201A46194600900AA822F0FEFA0AA9384621F04CFF044604F0F204384622F031FD0646F22C0CD1012E0AD14DB94146F6
:403880000C20FFF77CFF20B10C20FFF76CFA01250DE0F22C0BD1022E09D145B941460B20FFF76DFF18B10B20FFF75DFA0125F220012102220023CDE90532CDE9071010211C
:4038C0000193CDE9023197201A461946049300900AA822F0C2FA0AA9384621F010FF044604F0F204384622F0F5FC0646F22C1DD1012E1BD1D5B941460920FFF740FFA8B1E9
:403900000920FFF730FA01252CE0EDE0D8030020D414002049FD080865FC08080019002081F808085D000020781A0010F22C0CD1022E0AD14DB941460120FFF720FF20B1FA
:403940000120FFF710FA01250CE0F22C0AD14EB945B941460620FFF712FF18B10620FFF702FA01259620012100220592CDE90621089010210192CDE90221392013461146AF
:40398000049200900AA822F068FA0AA9384621F0B6FE044604F09604962C09D145B941460420FFF7ECFE18B10420FFF7DCF901259620012100220592CDE9062108901021B3
:4039C0000123CDE9013239201346CDE90312009011460AA822F041FA0AA9384621F08FFE044604F09604962C09D145B941460720FFF7C5FE18B10720FFF7B5F90125922043
:403A0000012102220023CDE90532CDE9071086210193CDE9023121201A461946049300900AA822F01AFA0AA9384621F068FE044604F09204922C09D145B941460220FFF78F
:403A40009EFE18B10220FFF78EF901259A20012102220023CDE90532CDE907108621CDE9013266201A46CDE90313009019460AA822F0F3F90AA9384621F041FE044604F09F
:403A80009A049A2C09D145B941460320FFF777FE18B10320FFF767F901259A20012102220023CDE90532CDE9071086210193CDE9023166201A461946049300900AA822F01C
:403AC000CCF90AA9384621F01AFE044604F09A049A2C09D145B941460A20FFF750FE18B10A20FFF740F9012515B16720F4F7ECFC28460CB0BDE8F0818E480078082801D140
:403B0000012070470020FCE78A4800780F2801D1012070470020FCE786480078032801D1012070470020FCE7824800780A2801D1012070470020FCE77E480078042801D101
:403B4000012070470020FCE77A480078072801D1012070470020FCE7764800787047764890F820007047744890F8220008B1012070470020FCE77148704710B5704890F8DB
:403B80007C03122805D100221346D7216D4822F055FB10BD00B5FFF7C7FF10B9FFF702FC08B1012000E000200146084600BD664909780143644A117070472DE9F047814657
:403BC0000C4692461D46DDF8208060480068C078A84240D1002320225D49204638F032F918B920215A4876F01EF90123202258492031204638F026F920B920215448203080
:403C000076F011F90223202251494031204638F019F920B920214E48403076F004F9032320224B496031204638F00CF928B920214748603076F0F7F80AE010214448603092
:403C400002F0E5FF06466DF05BFE0120FFF7AFFF4220F4F739FCBDE8F0872DE9F04107460C4690461D46069E38480068C078A8425ED1002320223749204638F04AF918B986
:403C80002021344876F0CFF80123202231492031204638F03EF920B920212E48203076F0C2F8022320222B494031204638F031F920B920212748403076F0B5F803232022AC
:403CC00024496031204638F024F920B920212148603076F0A8F8042320221E498031204638F017F920B920211A48803076F09BF8052320221749A031204638F00AF920B9B9
:403D000020211448A03076F08EF8062320221149C031204638F0FDF820B920210D48C03076F081F80220FFF742FF4220F4F7CCFBBDE8F0815D000020CC140020A4140020DB
:403D4000781A0010A87A02206B000020D80300204E170020CE1700200021FE4A1180FE4A1180FE4A11707047F8B504460E460025012C01DD01240225F94890F8E004A042A4
:403D80000DD000BFF64880F8E044012200F59C61F448006800F5D47002F072F800BF8520F4F792FBF048D0F854110220DFF8BCC300DF06F01FFBEC48D0F808120120DFF889
:403DC000ACC300DF70F0F7FCE748016D0220DFF89CC300DFFDF7B4FDE54800680090E548224603210368E44833F060FF2820F4F76BFB2846F8BD2DE9F0412BF06AF80446E8
:403E000046F0CCFF8046D64890F84F5390F884630024B2E0002798E0C5216943D74A02EB810101F5C67101EB4611891C085D3A46214606F0DFF8C5216943D04A02EB810144
:403E400001F5C67101EB4611091D085D3A46214606F02EF9C5216943C84A02EB810101F5C67101EB4611891D085D3A46214606F095F9C5216943C14A02EB810101F5C67111
:403E800001EB46110831085D3A46214606F04AF9C5216943B94A02EB810101F5C67101EB46110A31085D3A46214606F0B3F9C5216943B24A02EB810101F5C67101EB4611F7
:403EC0000C31085D3A46214606F0E0F9C5216943AA4A02EB810101F5C67101EB46110E31085D3A46214606F00DFAC5216943A34A02EB810101F5C67101EB46111031085D79
:403F00003A46214606F03AFAC52169439B4A02EB810101F5C67101EB4611085D3A46214606F007F8C5216943944A02EB810101F50B7101EBC601891C31F8141008B23A46A9
:403F40002146FEF770F9781CC7B2022FFFF664AFC5206843894901EB800000F5C67000EB4610143000EB8400D0ED000AB0EE600A204605F003FE601CC4B2022CFFF64AAF10
:403F800098F803100020FFF7EFFEC52169437B4A02EB810101F50B7131F8361008B2FEF718F9C5216943754A02EB810101F50B7101EBC601C879FEF79CF9C52169436F4AF9
:403FC00002EB810101F50B7101EBC6018879FEF768F9BDE8F0812DE9F8438046FEF771FD58B9FEF766FD40B9FEF75CFD28B9FEF751FD10B9FEF746FDA0B15D480068009083
:404000005C480022032103685B48E63833F04EFE534890F88403042803D10021012072F0CEFEE7E04E4890F84F4390F8845300268CE0002776E0B8F1000F0DD05049C85DA9
:40404000002239466FF082FF4D49891CC85D0022394670F011F81FE0C5216143474A02EB8101383105EB051201EB82010931885D002239466FF06AFFC52161433F4A02EB65
:404080008101383105EB051201EB82010B31885D002239466FF0F0FFC5216143374A02EB8101383105EB051201EB8201C91C885D00233A4631466FF0A2F9C52161432F4A55
:4040C00002EB8101383105EB051201EB8201491D885D00233A4631466FF054FAC5216143264A02EB8101383105EB051201EB8201C91D885D00233A4631466FF0E7FAC5210D
:4041000061431E4A02EB8101383105EB051201EB8201491C885D00233A4631466FF0CBF8781CC7B2022F86DBC5216143134A02EB8101383105EB051201EB82014031885D75
:404140000022314672F0F8FF701CC6B2022EFFF670AF17E0200200202202002024020020781A00108C0000100019002081F80808DC030020D803002058010800083F09088F
:404180003C1E0010C5206043F74901EB8000383005EB051100EB8100D0ED0C0AB0EE600A002070F005F9C5216143EF4A02EB8101383105EB051201EB8201898C88B20021AD
:4041C0006EF0D3FDC5216143E74A02EB8101383105EB051201EB820191F82800002170F002FA0021084672F0EAFD0021084672F070FE00BFBDE8F883F8B50746FEF761FC38
:4042000058B9FEF756FC40B9FEF74CFC28B9FEF741FC10B9FEF736FC50B1D44800680090D348002201210368D24833F03FFDA6E0D14890F84F5390F8846300249BE000219D
:4042400020469FEDCE0A6FF0D8FB002120469FEDCC0A6FF087FD7FB3CA4800EB8400D0ED000AB0EE600A002120466FF0D9FAC548103000EB8400D0ED000AB0EE600A00218F
:4042800020466FF0BAFBBF48083000EB8400D0ED000AB0EE600A002120466FF08DFCB948183000EB8400D0ED000AB0EE600A002120466FF057FD5CE0FFE7C5206843AA4932
:4042C00001EB8000383006EB061100EB81000E3030F9140000EE900AF8EEE00AB0EE600A002120466FF09CFAC52068439E4901EB8000383006EB061100EB8100163030F9F1
:40430000140000EE900AF8EEE00AB0EE600A002120466FF072FBC5206843934901EB8000383006EB061100EB8100123030F9140000EE900AF8EEE00AB0EE600A002120469C
:404340006FF03AFCC5206843874901EB8000383006EB061100EB81001A3030F9140000EE900AF8EEE00AB0EE600A002120466FF0F9FC601CC4B2022CFFF661AF00BFF8BDA5
:4043800010B504462046FFF737FF2046FFF723FEFFF731FD10BD70B5774890F84F4390F88453C52114FB01F16F4A02EB810101F5157105EB850231F8220001215AF0F0FEEA
:4043C000C52114FB01F1684A02EB810101F5157105EB850201EB8201488801215AF014FFC52114FB01F1604A02EB810101F5157105EB850201EB8201888801215AF038FFEF
:40440000C52114FB01F1584A02EB810101F5157105EB850201EB8201C88801215AF05CFFC52114FB01F1504A02EB810101F5157105EB850201EB820108895AF081FFC52178
:4044400014FB01F1484A02EB810101F5157105EB850201EB820148895AF09FFFC52114FB01F1414A02EB810101F5157105EB850201EB820188895AF0BDFFC52114FB01F1DE
:40448000394A02EB810101F5157105EB850201EB8201887B5AF0D9FFC52114FB01F1324A02EB810101F5157105EB850201EB8201087C5BF020F8C52114FB01F12A4A02EB20
:4044C000810101F5157105EB850201EB8201C87B5AF0E6FFC52114FB01F1234A02EB810101F5157105EB850201EB8201487C5BF02DF870BDF8B505460C4600261E4890F882
:404500008403032813D100BF1B4880F88553012200F285311C4800684D3001F0B1FC00BFAB20F3F7D1FF2C202EF0CEFD78E0D4B9FEF7C7FA58B9FEF7BCFA40B9FEF7B2FA57
:4045400028B9FEF7A7FA10B9FEF79CFA58B107480068009006482A460321036805481A3033F0A4FB5CE011E0083F0908DC030020D803002072000800781A00100000C8C255
:404580000000C8421C1E00108C00001024B3FE480068C078A0421FD0FEF793FA88B9FEF788FA70B9FEF77EFA58B9FEF773FA40B9FEF768FA28B9FEF77CFA10B9FEF76AFA7C
:4045C00050B1F24800680090EF482A4603210368EF4833F06BFB23E0FEF773FA58B9FEF768FA40B9FEF75EFA28B9FEF753FA10B9FEF748FAA0B1E4480068C078A0420FD17D
:4046000000BFE44880F88553012200F28531E24800684D3001F034FC00BFAB20F3F754FF3046F8BD70B50446002500BFD94880F87D47012200F27D71D748006800F24540A1
:4046400001F01EFC00BF284670BD70B5D14890F84F5390F88443C52115FB01F1CF4A02EB810101F52E7104EB440201EB42014878FFF7D8FFC52115FB01F1C84A02EB8101BF
:4046800001F52E7104EB440201EB42018878012133F014FDC52115FB01F1C04A02EB810101F52E7104EB440201EB4201C878002133F004FDBA48D0ED000ABBEE091A60EEE9
:4046C000810AB0EE600A002071F0FBF9B448D0ED000A9FEDB41A60EE810AB0EE600A002070F02FFEAE48D0ED000AB3EE091A60EE810AB0EE600A002070F0C9FC032C01D060
:40470000042C25D1C5216943A44A02EB810101F2D62111F8340000216DF040FDC52169439E4A02EB810101F2D62101EBC401487800216CF04BFBC5216943984A02EB810198
:40474000383104EB041211F822000021FFF7D2FE70BD2DE9F0418F48B0F85A77B0F85C47B0F85E57B0F86067B0F86C8790F878030A2827D1A74206DB002C04DD611E88B286
:4047800000215AF00DFDAE4204DA691C88B200215AF0A2FDBD4203DA002138465AF068FDA64203DD002120465AF096FDB04503DD002130465AF005FFA84503DA0021284684
:4047C0005AF0FFFEBDE8F08110B5012033F027FD0146754880F83910002033F020FD72494874012033F01BFD04462146012020F077FF002033F013FD04462146002020F0AB
:404800006FFF10BD10B5FFF720FFFEF752F910B9FEF740F918B10021012033F096FB0020FFF7AEFDFFF7D0FF01206DF09FFC10BD5848B0F88C0300EE100AF8EE400A9FED66
:404840005B1A80EE810A70475948007801280BD15048B0F88C0300EE100AF8EE400A9FED551A80EE810A70474A48B0F88C0300EE100AF8EE400A9FED4D1A80EE810AF2E77D
:40488000444890EDE40AB8EEC00AF0EE400A4A48B0F9000000EE100AB8EEC00A30EE801ADFED421A81EE210A70473A4890EDE40AB8EEC00AF0EE400A3D48007801280ED1FB
:4048C0003448B0F88C0300EE100AB8EE401AF0EE001A81EE210A30EEC00AF0EE400A3648B0F9000000EE100AB8EEC00A30EE801ADFED2E1A81EE210A70472648B0F89403F2
:404900002E49B1F90010084400EE100AF8EEC00A9FED261A80EE810A70471E48D0EDE60A9FED221A80EE810A704710B502460020234BB3F900309A4204D1224BB3F90030CA
:40494000994243D01E4B1A801E4B19801C4BB3F900301C4CB4F900401B1B03EB83035B000C4CD4F8904363430A4CB4F88C4393FBF4F3144C248804EB840403EB44031BB23F
:404980000E4C238000231FE0D8030020DC0300208C000800781A00108C000010083F0908F46B0A0800000000E87C022000007A44240200200000FA442202002020020020F5
:4049C0002602002028020020F94C238010BDF8B504460D46002641F65830844201DD0446022600BFF348A0F88C43022200F56371F1480068543001F043FA00BF0220F3F7BF
:404A000063FD1F202EF060FBA5B1EC480068C078A8420FD0E74890F8840303280AD0E84800680090E548224603210368E54833F03DF919E0C5B9FEF744F858B9FEF739F877
:404A400040B9FEF72FF828B9FEF724F810B9FEF719F848B1DA4800680090D848224603210368D84833F022F9D748D0F854110220DFF858C300DF00214FF480700DF05BFFEE
:404A80003046F8BD70B504460025B4F5FA4F03DD4FF4FA44022504E014F5FA4F01DACC4C032500BFC348C0F89043042200F56471C1480068583001F0E3F900BF0620F3F792
:404AC00003FD1F202EF000FBBF48D0F854110220DFF8F8C200DF00214FF480700DF02BFF284670BD70B50446002541F65830844201DD0446022500BFAE48A0F894430222D2
:404B000000F56571AC4800685C3001F0B9F900BF0720F3F7D9FC1F202EF0D6FA284670BD10B52DED028BB0EE408A00249FEDA90AB4EEC08AF1EE10FA05DD9FEDA60AB0EEEA
:404B4000408A02240BE09FEDA40AB4EEC08AF1EE10FA04D29FEDA00AB0EE408A0324954890EDE60AB4EE480AF1EE10FA0BD000BF80EDE68A042200F566718F480068603051
:404B800001F07EF900BF0520F3F79EFC1F202EF09BFA2046BDEC028B10BD70B50446002500BF8448C0F87843042200F55E7182480068403001F064F900BF0920F3F784FC0C
:404BC0001F202EF081FA284670BD70B50446002500BF784880F84F43012200F24F3176480068173001F04CF900BF0820F3F76CFC5A20F3F769FC1F202EF066FA284670BD93
:404C000070B50446002500BF6A48C0F87C43042200F55F7168480068443001F031F900BF0A20F3F751FC1F202EF04EFA284670BDF8B504460D460026032C13D100BF5D481F
:404C400080F88443012200F561715B4800684C3001F016F900BF0B20F3F736FC2C202EF033FA71E035BBFDF72CFF58B9FDF721FF40B9FDF717FF28B9FDF70CFF10B9FDF7C2
:404C800001FFB8B100BF4B4880F88443012200F56171494800684C3001F0F2F800BF48480068009045482246032103684B4832F0FDFF49E025B341480068C078A8421FD041
:404CC000FDF7FFFE88B9FDF7F4FE70B9FDF7EAFE58B9FDF7DFFE40B9FDF7D4FE28B9FDF7E8FE10B9FDF7D6FE50B13548006800903248224603210368384832F0D7FF23E048
:404D0000FDF7DFFE58B9FDF7D4FE40B9FDF7CAFE28B9FDF7BFFE10B9FDF7B4FEA0B127480068C078A8420FD100BF224880F88443012200F56171204800684C3001F0A0F8C4
:404D400000BF0B20F3F7C0FB3046F8BD70B50446002500BF174880F87647012200F276711548006800F23E4001F08AF800BF284670BD70B50446002500BF0E4880F87747B5
:404D8000012200F277710C48006800F23F4001F077F800BF284670BD01460020704710B5044628220E49204674F0BEFF10BD000022020020781A00108C000010D803002070
:404DC000DC03002004FA07000019002081F808080083FFFF0000FA460000FAC656010800C81D001010B50446C5216143FD4A02EB8100FFF7D1FFC5216143FA4A02EB8101C7
:404E0000887FFFF7CAFEC5216143F64A02EB8101088D0021FFF7DBFDC5216143F14A02EB8101C86AFFF72EFEC5216143ED4A02EB8101088EFFF756FEC5206043E94901EBB2
:404E40008000B0F9320000EE900AF8EEE00AB0EE600AFFF765FEC5216143E24A02EB810191F82000FFF7B1FEC5216143DD4A02EB8101C87FFFF7C4FEFFF78DFA10BD10B57D
:404E8000044600BFD84880F87847012200F5EF61D648006800F5886000F0F2FF00BF10BD10B5044600BFD04880F80141012200F20111CF4800F0E4FF00BF10BDCA4890F883
:404EC0007813082903D0092901D00A2901D1012070470020FCE7C44890F878130A2901D1012070470020FCE7BF4890F87813082901D1012070470020FCE7BB4890F8781333
:404F0000092901D1012070470020FCE70020B64991F84F13432909D0B34991F84F13452904D0B14991F84F13472900D1012070470020AD4991F84F13422909D0AA4991F85B
:404F40004F13442904D0A84991F84F13462900D1012070470020A44991F84F13412900D10120704770B504460025A2480078844211D0012C01DD02250DE09E4804709E4893
:404F8000D0F854110220DFF874C200DF00214FF480700DF0D0FC284670BD934890F84F03C52110FB01F08F4901EB8000408C70478D4890F84F03C52110FB01F0894901EB51
:404FC0008000808C704770B501248D488D490978455C8C480078502823DA8A4800784E281FDAC52169437F4B03EB8102C521694303EB8101888C1E212BF0FAFC044024B191
:4050000080480078401C7F49087001207E4908704FF4CF7036F0DAFF40F2E22036F0D6FF05E0012077490870002077490870204670BD70B50124754800781E2833DA7348CE
:4050400000781A282FDA7149097801EB0111704A02EB4101081D74F0F1FD85B26B49097801EB01116A4B03EB41010A1D6749097801EB011103EB4101488829462BF0B8FCF1
:40508000044024B161480078401C6049087001205D4908704FF4CF7036F098FF40F2E32036F094FF05E0012058490870002056490870204670BD57480078704770B50124CC
:4050C0005548007812287DD15448007800287AD148F60F6052490880012005E04FF6FF714F4A22F81010401C1A28F7DB0021D3E0C52048433B4A02EB800090F8B90203281A
:405100006FD0C520484302EB800090F8B902022867D0C520484302EB800090F8BF0203285FD0C520484302EB800090F8BF0202287DD0C520484302EB800090F8C50203283B
:4051400075D0C520484302EB800090F8C50202286DD0C520484302EB800090F8CB02032865D0C520484302EB800090F8CB0202285DD0C520484302EB800090F8D1020328D9
:4051800055D0C520484302EB800090F8D10202284DD02448007800287DD0C520484302EB800090F8B902E0B9C520484302EB800090F8BF02A8B9C520484302EB800090F84D
:4051C000C50201E0A8E06FE058B9C520484302EB800090F8CB0220B9C520484302EB800022E024E0083F0908781A00108C00001001010068240200200019002081F8080829
:40520000F03A09081C020020C20400201D0200203E3B09081E0200209D0400202A020020441A0010A404002090F8D10270B3F94890F87823C5204843F74B03EB8000807FC2
:40524000824228D1012223E0C5204843F24B03EB8000C07F02EB0213F04D15F81330984215D1FFF728FF38B1FFF725FF02EB021315F8133098420AD102EB0210E74B03EB5C
:4052800040004088E64B23F8120003E003E0521C1A2AD9DB00BF491C6129FFF629AF0120E0490870E0490870DE4800781E282DDCDB48DC49097830F811004FF6FF71884210
:4052C00010D0D84800781A280CDAD548D549097830F81120D348017842F218702BF084FA044008E04FF6FF72CE48017842F218702BF07AFA044024B1CA480078401CC94943
:40530000087040F2E12036F061FE05E00120C54908700020C4490870204670BD70B5C348C3490978445C0125C248007812287DD1BF48007850287ADCBD4800784E2878DA5A
:40534000B44890F87C13C5206043B34A02EB8000C07F81426DD1AF4890F87813C520604302EB8000807F814263D1B348007838B3C5206043114601EB800090F8B9020028DF
:4053800074D1C520604301EB800090F8BF0200286CD1C520604301EB800090F8C502002864D1C520604301EB800090F8CB0200285CD1C520604301EB800090F8D102B8BB06
:4053C000C5206043944901EB800090F8B90203284CD0C520604301EB800090F8B902022844D0C520604301EB800090F8BF0203283CD0C520604301EB800090F8BF02022802
:4054000034D0C520604301EB800090F8C50203282CD0C520604301EB800090F8C502022824D0C520604301EB800003E051E046E01CE029E090F8CB02032817D0C52060437B
:4054400001EB800090F8CB0202280FD0C520604301EB800090F8D102032807D0C520604301EB800090F8D10202280DD1C5206043694901EB8000428C6D48017842F219705B
:405480002BF0B2F9054008E04FF6FF726848017842F219702BF0A8F9054025B164480078401C634908700120644908704FF4CF7036F08CFD4FF4387036F088FD09E00120CB
:4054C0005B49087000205D4908704FF4CF7036F07DFD284670BD0146C52048434E4A02EB800090F804017047012070470020704753480068704752490860704700204549C4
:4055000091F87C13102900D1012070470020414991F84F13142901D1012100E000213D4A92F84F23152A01D1012200E000221143384A92F84F23162A01D1012200E00022E8
:405540001143344A92F84F23172A01D1012200E0002211432F4A92F84F23182A01D1012200E0002211432B4A92F84F23192A01D1012200E00022114301B101207047002026
:40558000244991F87813042905D1224991F87C13022900D10120704700201E4991F87813042905D11B4991F87C130C2900D1012070470020174991F87C13112900D1012054
:4055C00070470020134991F87C130D2900D10120704700200F4991F87C13152900D10120704700200B4991F87C130F2900D1012070470020074991F87C13122900D10120E8
:4056000070470020034991F87C13132900D1012070470000781A0010083F09083E3B0908441A00101D0200202A020020F03A09081C0200209D040020A4040020C2040020E5
:40564000180200200020FB4991F87C13162900D101207047014601EB0110F74A12F8100070470246012109E001EB0110F24B13F81000904201D1C8B27047491C1A29F3DB43
:405680000020F9E72DE9F0410124EA4991F87C03FFF7E7FF00EB0010E74901EB4000051DE44991F87C03FFF7DCFF00EB0010E24901EB4000071D384674F0C0FA86B22A462E
:4056C000314649F2FC102BF093F904462046BDE8F08170B5D74890F84F4390F884530A20DFF858C300DFC52114FB01F1D44A02EB810101F2D62101EBC501487800216BF07B
:4057000065FB0A20DFF834C300DF00209FEDCD0A6BF03BF80A20DFF824C300DFC52114FB01F1C74A02EB8101383105EB051211F822000021FEF7DEFE0A20DFF800C300DFC3
:40574000C52014FB00F0BE4901EB8000383005EB051100EB8100B0F90E0000EE900AF8EEE00AB0EE600A002108466EF059F80A20DFF8C8C200DFC52014FB00F0B04901EB90
:405780008000383005EB051100EB8100B0F9160000EE900AF8EEE00AB0EE600A002108466EF02BF90A20DFF894C200DFC52014FB00F0A34901EB8000383005EB051100EBB4
:4057C0008100B0F9120000EE900AF8EEE00AB0EE600A002108466EF0EFF90A20DFF85CC200DFC52014FB00F0954901EB8000383005EB051100EB8100B0F91A0000EE900A07
:40580000F8EEE00AB0EE600A002108466EF0AAFA0A20DFF828C200DFC52114FB01F1884A02EB8101383105EB051201EB8201C87800231A4619466DF0E2FD0A20DFF8FCC132
:4058400000DFC52114FB01F17D4A02EB8101383105EB051201EB8201487900231A4619466DF090FE0A20DFF8D4C100DFC52114FB01F1734A02EB8101383105EB051201EBDB
:405880008201C87900231A4619466DF01FFF0A20DFF8A8C100DFC52114FB01F1684A02EB8101383105EB051201EB8201898C88B200216DF05AFA0A20DFF880C100DFC5216F
:4058C00014FB01F15E4A02EB8101383105EB051201EB8201487A002211466EF037FB0A20DFF858C100DFC52114FB01F1544A02EB8101383105EB051201EB8201C87A0022B6
:4059000011466EF0B9FB0A20DFF830C100DFC52114FB01F14A4A02EB8101383105EB051201EB8201487800231A4619466DF0C3FC0A20DFF808C100DFC52014FB00F0404990
:4059400001EB8000383005EB051100EB8100D0ED0B0AB0EE600A00206EF0B4FD0A20DFF8DCC000DFC52014FB00F0354901EB8000383005EB051100EB8100D0ED0C0AB0EE43
:40598000600A00206EF014FD0A20DFF8B0C000DF00209FED2D0A70F03FF90A20DFF89CC000DF00209FED290A6FF0A2FD0A20DFF88CC000DFC52114FB01F1214A02EB81011D
:4059C000088D0021FFF703F80A20DFF870C000DF70BD10B501241E4800780E283CDA1C48007800EB40001B4901EB4000007970B11748007800EB400001EB4000428814482A
:405A0000017842F210702AF0EFFE044008E04FF6FF720F48017842F210702AF0E5FE04400B480078401C0A49087040F2E62036F0CDFA14E0781A00103E3B090821F808082B
:405A4000083F090800000000B81E05BFB81E053F2B020020B23E09080020EE490870204610BD10B5002413E004EB4400EA4A02EB8000411CE94874F04BFA38B904EB4400BF
:405A8000E54911F82000E649087003E0601CC4B2082CE9DB00BF10BDF8B504460E460025012C01DD01240225DE4890F8E104A0420DD000BFDB4880F8E144012200F2E141C0
:405AC000D948006800F2A91000F0DAF900BFAA20F2F7FAFCD548D0F854110220DFF850C300DF04F087FCD148D0F808120120DFF840C300DF6EF05FFECC48016D0220DFF890
:405B000030C300DFFBF71CFFCA4800680090CA48224603210368C94832F0C8F82846F8BDF8B5FCF7CEFF58B9FCF7C3FF40B9FCF7B9FF28B9FCF7AEFF10B9FCF7A3FF58B19E
:405B4000BC4800680090BC4803221146036840F2762032F0ABF894E0B24890F84F4390F88453002689E0C5206043B54901EB8000383005EB051100EB81000E30A94991F8B6
:405B8000E01430F9110000EE900AF8EEE00AB0EE600A304666F051F9C5206043A84901EB8000383005EB051100EB810012309D4991F8E01430F9110000EE900AF8EEE00A4B
:405BC000B0EE600A304666F053F9C52060439C4901EB8000383005EB051100EB81001630904991F8E01430F9110000EE900AF8EEE00AB0EE600A304667F010F8C52060433F
:405C00008F4901EB8000383005EB051100EB81001A30844991F8E01430F9110000EE900AF8EEE00AB0EE600A304666F0DAFFC5216143834A02EB8101383105EB051201EB51
:405C400082010931774A92F8E024885C314666F0B6FFC52161437A4A02EB8101383105EB051201EB82010B316E4A92F8E024885C314666F093FF701CC6B2022EFFF673AF06
:405C800000BFF8BD10B52DED028BB0EE408A002400BF6C4880ED138A042200F14C016248006800F24C4000F0EBF800BFAD20F2F70BFC2046BDEC028B10BD70B50025594864
:405CC00090F87843082C03D0092C01D00A2C01D1012505E0FFF73EF908B1022500E000252846FFF7CCF870BDF8B504460D4600264C4890F88403032814D100BF4948A0F8CF
:405D00008247022200F282714748006800F24A4000F0B6F800BFC220F2F7D6FB2C202DF0D3F975E00DBBFCF7CCFE58B9FCF7C1FE40B9FCF7B7FE28B9FCF7ACFE10B9FCF778
:405D4000A1FE90B1322C01DD322402E0002C00DA0024384800680090374822460321036836488D3831F0A2FF52E065B332480068C078A84227D0FCF7A4FE88B9FCF799FE0D
:405D800070B9FCF78FFE58B9FCF784FE40B9FCF779FE28B9FCF78DFE10B9FCF77BFE90B1322C01DD322402E0002C00DA002421480068009020482246032103681F488D38F2
:405DC00031F074FF24E0FCF77CFE58B9FCF771FE40B9FCF767FE28B9FCF75CFE10B9FCF751FEA8B114480068C078A84210D100BF0C48A0F88247022200F282710A4800684A
:405E000000F24A4000F03CF800BFC220F2F75CFB3046F8BD2B020020903A0908D86F00081E020020781A00108C0000100019002081F80808DC030020D8030020EF0108000D
:405E4000083F0908B0210010FE480078704710B55EF0A8F840B1FC4890F83503012803D001200CF08FFD0AE05EF0F9FD38B1F64890F83503022802D002200CF083FD10BDAB
:405E80002DE9F04104460E46174600255EF0DDFD08B9042514E0B4F1D04F10D3E019401EEA4988420BD8A4F1D0483A464146304610F08AFD08B1002502E0102500E00825E4
:405EC00025B1E34800882843E14908802846BDE8F0812DE9FE4F06468946174698460020009083464FF4807200233846414673F093FA05464FF4807200233846414673F0EE
:405F00008BFA924615B9BAF1000F2AD0ADB1002411E006EB0420029009EB042001904FF48072DDE90110FFF7ABFF009000984BEA000B601CC4B2AC42EBD3BAF1000F12D071
:405F400006EB0520029009EB052001901FFA8AF2DDE90110FFF794FF009000984BEA000B01E04FF0400B5846BDE8FE8F10B5044610222146B74873F0D7FE1022B549B6482A
:405F8000FFF77EFF10BD2DE9F04180460C46164600255EF05AFD08B9042514E0B4F1D04F10D3A019401EA94988420BD8A4F1D04732463946404610F09CFD08B1002502E05F
:405FC000102500E0082525B1A14800882843A04908802846BDE8F0812DE9FF5F86B007468846DDF850B0DDE90801381A78EB01007ED204F000FE81460125AFE3062D0CD2C7
:40600000DFE805F00B0C09070503944E08E0944E06E0944E04E0944E02E000BF934E00BF00BF012206F1170105A8FFF7ACFF9DF81400612801DB00200590012206F14C0191
:4060400004A8FFF7A0FF9DF81000052801DB002004909DF8140058457ED19DF8100003287BD10024C8E04FF0000A9FE09DF81400C52110FB01F07E4901EB800038309DF87D
:40608000101001EB011100EB8100C01C005D029006F1940101EB440101EB0A00012202A9FFF7EEFE4D4506D19DF80810714800EB440000F80A109DF81400C52110FB01F08D
:4060C0006B4901EB800038309DF8101001EB011100EB8100401D005D029006F1980101EB440101EB0A00012202A9FFF7C9FE00E038E34D4507D19DF808105E48001D00EBAB
:40610000440000F80A109DF81400C52110FB01F0574901EB800038309DF8101001EB011100EB8100C01D005D029006F19C0101EB440101EB0A00012202A9FFF7A1FE4D456F
:4061400007D19DF808104B48083000EB440000F80A109DF8140001E0FEE2F7E0C52110FB01F0434901EB800038309DF8101001EB011100EB8100401C005D029006F1A00109
:4061800001EB440101EB0A00012202A9FFF778FE4D4507D19DF8081036480C3000EB440000F80A100AF1010000F0FF0ABAF1020FFFF65CAF9DF81400C52110FB01F02C49BB
:4061C00001EB800038309DF8101001EB011100EB81004030005D029006F192010819012202A9FFF74DFE4D4504D19DF808102148801E0155601CC4B2022CFFF634AF9DF895
:406200001400C52110FB01F0194901EB800038309DF8101001EB011100EB810090ED0C0A8DED030A042203A906F1C400FFF728FE4D4504D19DED030A034880EDFF0A9DF8FC
:40624000140019E088000010781A0010FF1F006892000010901B001018010068901700682C130068C80E0068640A006800060068083F0908441E0010C52110FB01F0FE4948
:4062800001EB800038309DF8101001EB011100EB8100808C80B20190022201A906F1D600FFF7EEFD4D4504D1BDF80410F348A0F80E149DF81400C52110FB01F0EE4901EBCD
:4062C000800038309DF8101001EB011100EB810090F828000290012202A906F50470FFF7CFFD4D4504D19DF80810E44880F848159DF81400C52110FB01F0DF4901EB800022
:4063000038309DF8101001EB011100EB810090F842000290012202A906F21920FFF7B0FD4D4504D19DF80810D44880F8511500200290012202A906F24140FFF7A1FD4D45AB
:4063400004D19DF80810CD4880F879170024AAE14FF0000A74E19DF81400C52110FB01F0C54901EB800000F5C6709DF8101000EB4110801C005D019006F5987101EB840111
:4063800001EB4A00022201A9FFF77AFD4D4506D1BDF80410BA4800EB840020F81A109DF81400C52110FB01F0B34901EB800000F5C6709DF8101000EB4110001D005D01906D
:4063C00006F59C7101EB840101EB4A00022201A9FFF756FD4D4507D1BDF80410A848083000EB840020F81A109DF81400C52110FB01F0A14901EB800000F5C6709DF810100A
:4064000000EB4110801D005D019006F5A07101EB840101EB4A00022201A9FFF731FD4D4507D1BDF804109648103000EB840020F81A109DF81400C52110FB01F08E4901EBA0
:40644000800000F5C6709DF8101000EB41100830005D019006F5A87101EB840101EB4A00022201A9FFF70CFD4D4507D1BDF804108348203000EB840020F81A109DF814002A
:40648000C52110FB01F07C4901EB800000F5C6709DF8101000EB41100A30005D019006F5AC7101EB840101EB4A00022201A9FFF7E7FC4D4507D1BDF804107148283000EBF0
:4064C000840020F81A109DF81400C52110FB01F0694901EB800000F5C6709DF8101000EB41100C30005D019006F5A47101EB840101EB4A00022201A9FFF7C2FC4D4507D144
:40650000BDF804105E48183000EB840020F81A109DF81400C52110FB01F0574901EB800000F5C6709DF8101000EB41100E30005D019006F5B47101EB840101EB4A00022229
:4065400001A9FFF79DFC4D4507D1BDF804104C48383000EB840020F81A109DF81400C52110FB01F0444901EB800000F5C6709DF8101000EB41101030005D019006F5B07118
:4065800001EB840101EB4A00022201A9FFF778FC4D4507D1BDF804103948303000EB840020F81A109DF81400C52110FB01F0324901EB800000F5C6709DF8101000EB4110A9
:4065C000005D019006F5947101EB840101EB4A00022201A9FFF754FC4D4507D1BDF804102748083800EB840020F81A109DF81400C52110FB01F0204901EB800000F50B708F
:406600009DF8101000EBC100801C30F81400019006F5D67101EB840101EB4A00022201A9FFF72EFC4D4507D1BDF8041014487C3000EB840020F81A100AF1010000F0FF0AD8
:40664000BAF1020FFFF687AE9DF81400C52110FB01F0094901EB800000F5C6709DF8101000EB4110143000EB840090ED000A8DED030A06F58B6105E0083F0908781A001048
:40668000E01E001001EB8400042203A9FFF7F8FB4D4506D19DED030AFE4800EB840080ED000A601CC4B2022CFFF652AE9DF81400C52110FB01F0F84901EB800000F50B70B8
:4066C0009DF8101030F831000190022201A906F5D570FFF7D5FB4D4504D1BDF80410EF48A0F8E2149DF81400C52110FB01F0EA4901EB800000F50B709DF8101000EBC10037
:40670000C0790190022201A906F5DB70FFF7B8FB4D4504D1BDF80410E048A0F8EE149DF81400C52110FB01F0DB4901EB800000F50B709DF8101000EBC10080790190022246
:4067400001A906F5DA70FFF79BFB4D4504D1BDF80410D248A0F8EC14681CC5B2052D7FF74DAC00BF0AB0BDE8F09F38B504460D461420CB4A0023009020462946FFF72CFCFA
:406780001520C74A0023009020462946FFF724FC1620C34A0023009020462946FFF71CFC1720BF4A0023009020462946FFF714FC1820BB4A0023009020462946FFF70CFC8B
:4067C0001920B74A0023009020462946FFF704FC38BD70B505460E46B249691A76F100001ED2AE4890F8300540B1012809D0022802D003280BD107E07F2409E040F6EC1401
:4068000006E040F6EC1403E040F2FA2400E000BF00BF00EE104AB8EE400AF9F79DFA00BF70BD2DE9FE4306460F469D494539711A77F1000054D204F0DEF9804601244CE0A9
:40684000062C0CD2DFE804F00B0C09070503964D08E0964D06E0964D04E0964D02E000BF954D00BF00BF012205F1170102A8FFF78AFB9DF80800612801DB002002900122B2
:4068800005F14C0101A8FFF77EFB9DF80400052801DB002001909DF80800C52110FB01F07D4901EB800038309DF8041001EB011100EB810090ED0C0A8DED000A0422694612
:4068C00005F1C400FFF7DCFA444504D19DED000A724880EDFF0A601CC4B2052CB0DD00BFBDE8FE8310B504466C4880F83043012200F54C717148FFF7C3FA10BD2DE9FC414C
:4069000004460D4616461F466D490020891BB84114D26B490020091BA8410FD30020FFF7E1FF684903C9CDE900019DF8070000F00F0010B10120FFF7D5FF00BFBDE8FC818B
:406940002DE9FE4F06468946174698460020009083464FF4807200233846414672F05CFD05464FF4807200233846414672F054FD924615B9BAF1000F2AD0ADB1002411E0A5
:4069800006EB0420029009EB042001904FF48072DDE90110FFF7F7FA009000984BEA000B601CC4B2AC42EBD3BAF1000F12D006EB0520029009EB052001901FFA8AF2DDE945
:4069C0000110FFF7E0FA009000984BEA000B01E04FF0400B5846BDE8FE8F70B505460E463949691A76F100003CD2012004F0DEF805F054FE142803D005F050FE152818D12B
:406A000004F0F9F80446254890F84F03C52110FB01F0214901EB80021521204604F0EFF81E4991F87807FEF73BFA0120FAF765FF02E00020FEF734FA022404E0204604F017
:406A40008CFA601CC4B2052CF8DD40F2644200231E4801681E48FFF773FF104991F85807FAF751FB70BD2DE9F84305460E4616492731691A76F1000068D24FF007081249E1
:406A80001331691A76F1000001D24FF00908FF2000901FE008220010083F0908781A0010C64EB93B2514AA3B901700682C130068C80E0068640A00680006006830030068AA
:406AC000D2D19A3BF86F00086D0CAA3B8C000010B01D0010012436E0062C0CD2DFE804F00B0C09070503FA4F08E0FA4F06E0FA4F04E0FA4F02E000BFF94F00BF00BF012243
:406B000007F117016846FFF73EFA9DF800004044C0B200909DF80000132812DD9DF8000061280EDA0122694607F11700FFF7A8F904F061F8A04204D19DF80010E94880F8BF
:406B40004F13601CC4B2052CC6DD00BFBDE8F8832DE9F04105460E46E349691A76F100001ED2E04890F84F7390F88483002414E0C5207843DD4901EB800000F5C67000EBC1
:406B80004810143000EB8400D0ED000AB0EE600A204602F0F3FF601CC4B2022CE8DB00BFBDE8F08170B504460D46D149611A75F100000AD2CB4890F8C90318B10320FDF719
:406BC00031FD02E00020FDF72DFD70BD7FB505460E46C849691A76F1000017D2002005F09BF8002005F08AF81022C349684673F09BF86846FFF7BAF9012404E0204604F088
:406C0000ACF9601CC4B2052CF8DD03DF7FBD2DE9F34F82B0844600BF00210A460B460E460F46002001908046009063E09CF80000A0F13004E5179CF800002E2838D1B8F1E0
:406C4000000F0CD1AD494FF00009A2FB010A03FB01A102FB0919861949EB07071FE0B8F1010F0CD1A6494FF00009A2FB010A03FB01A102FB0919861949EB07070FE0B8F1F6
:406C8000020F0CD14FF47A714FF00009A2FB010A03FB01A102FB0919861949EB070708F1010000F0FF0800200090002213461BE09CF80000C0B1009810B922462B460FE0E3
:406CC000009801280CDB0A214FF0000B9146A9FB010E03FB01E102FB0B19021949EB05030098401CC0B200900CF1010C0198401CC0B2019003990198884297DBB6185F41BE
:406D00003046394604B0BDE8F08F10B5044610227C49204673F008F810BD70B504460D467048A0F84843284603F02AFF06460222754906F11000FFF7A3F870BDFEB50020FD
:406D4000029001900090012540F69851654873F08CF801226D4902A8FFF715F99DF80800401CC0B20190012201A96848FFF788F8002002900122654902A8FFF704F99DF85C
:406D800008009DF80410884206D06148008840F080005F490880DEE001225C49C91E6846FFF7F1F89DF8000013284ED04FF44E714C4873F05AF840F264415348103873F021
:406DC00054F84FF4FF71534873F04FF840F2FE31514873F028F84FF44E72002341494FF0D040FFF776F801240CE0204603F0C8FE064640F26442002343491039FFF769F8CC
:406E0000601CC4B2052CF0DD4FF4FF72002341494248FFF75EF840F2FE3200233E494048FFF757F813200090012269463748C01EFFF726F8002405E021460620FFF76DFF54
:406E4000601CC4B2052CF7DD85E04FF44E7200234FF0D0412348FFF773FD03F0CCFE044603F0A4FE00211F48A0F8481302222D48016810312448FFF786F81A48B0F84803E0
:406E8000062851D040F264411F48103872F0EDFF4FF4FF711F4872F0E8FF40F264420023194910391F480068FFF713F84FF4FF72002318491948FFF70CF8012405E02146D2
:406EC0000620FFF72AFF601CC4B2052CF7DD42E0901700682C130068C80E0068640A006800060068781A0010560CAA3B083F0908ECCD9A3B34CB9A3B9CBE000800CA9A3B58
:406F000040420F00901B0010C01D00102C01006892000010142200101224001000040068001C00688C000010022540F264420023684801686848FFF703FD4FF4FF72002311
:406F400066496748FFF7FCFC40F2FE32002365496548FFF7F5FC2846FEBD70B590B000BF182102A872F081FF01206049088000205F4908705F480FF0B3FC10B100205B4980
:406F800008805A480088002812D1FFF7D7FE5A490880102259490CA872F0C6FE56480088012806D10020524908700CA8FEF7DEFF84E001204E49087010210CA8FFF727FEFD
:406FC0004F4A03C208A8FFF7A0FE102108A8FFF71EFE0D4604464A48D0E90021101BA9411CD2002004F098FE002004F087FE102242490CA872F098FE0CA8FEF7B7FF1821AC
:4070000002A872F032FF012604E0304603F0A5FF701CC6B2052EF8DD03DF4DE0384903C9201A75EB010047D220462946FFF7CEFD20462946FFF7B6FD20462946FFF788FD7B
:4070400020462946FFF70FFD20462946FFF7C5FC2B480CC820462946FFF750FC1E20294A0023009020462946FEF7B6FF20462946FFF7D7FB20462946FFF7ABFB2046294689
:40708000FFF773FB002004F047FE002004F036FE10221A490CA872F047FE0CA8FEF766FF40F2FE31104872F0BEFE40F2FE3200230D490C48FEF70DFFFEF7C9FE0020FEF7F5
:4070C0001AFA10B070BD104890F8300370470C4903C970478C000010B01D00100004006814220010001C006812240010920000108800001000300140900000109CBE00084B
:4071000098000010B20CAA3B781A00101FB50121084663F0C2F80121042063F0BEF80121082063F0BAF80121102063F0B6F8002000900190029003460122FE4903901046B1
:407140005DF079F8002000900190029003460222F949039010465DF06EF8002000900190029003460246F549039005205DF063F8002002220123CDE9012000930390034683
:40718000EF4906205DF057F8002002220123CDE90120009303900346EA4907205DF04BF8002002220123CDE90120009303900346E54908205DF03FF80020009001900290E2
:4071C00001230222E149039009205DF034F800200323CDE90030029003460222DC4903900A205DF028F800200121CDE9000103460A46CDE90210D7490B205DF01CF8002048
:4072000000900190029003460322D349039011205DF011F8002000900190029003460322CE49039012205DF006F800200323CDE90030029003460222C949039018205CF03B
:40724000FAFF002000900190029003460122C549039019205CF0EFFF002000900190029003460122C04903901A205CF0E4FF00200222CDE9000202900346BC4903901B20D4
:407280005CF0D9FF00200222CDE9000202900346B74903901F205CF0CEFF00200222CDE9000202900346B349039020205CF0C3FF002001210090CDE9010103460A46AE491A
:4072C000039021205CF0B7FF002001210090CDE9010103460A46A949039024205CF0ABFF002000900190029003460246A449039025205CF0A0FF00200090019002900346A6
:407300000246A049039026205CF095FF002001210090CDE9010103460A469B49039029205CF089FF002000900190029001230222964903902A205CF07EFF00200121CDE914
:40734000000103460A46CDE9021091492D205CF072FF0020009001900290034602228D49039031205CF067FF0020009001900290034602228849039032205CF05CFF00205E
:407380000121CDE9000103460A46CDE90210834933205CF050FF00200121CDE9000103460A46CDE902107E4934205CF044FF00200121CDE9000103460A46CDE902107949B9
:4073C00035205CF038FF00200121CDE9000103460A46CDE90210744936205CF02CFF00200121CDE9000103460A46CDE902106F4937205CF020FF00200121CDE900010346BB
:407400000A46CDE902106A4938205CF014FF002001210090CDE9010103460A466549039039205CF008FF002001210090CDE9010103460A46604903903B205CF0FCFE00209A
:4074400001210090CDE9010103460A465B4903903C205CF0F0FE00200121CDE9000103460A46CDE9021056493D205CF0E4FE00200121CDE9000103460A46CDE902105149C4
:407480003E205CF0D8FE002001210090CDE90101034602224C49039040205CF0CCFE0020009001900290034602224849039041205CF0C1FE002000900190029003460222A7
:4074C0004349039042205CF0B6FE0020009001900290034602463F49039043205CF0ABFE0020009001900290034601223A49039046205CF0A0FE00200222CDE90002029001
:4075000003463649039047205CF095FE0020009001900290034602223149039048205CF08AFE0020009001900290034602222D49039059E0CA030010F5030010CB030010DC
:40754000E2030010E3030010E4030010E5030010CC030010FD030010D203001011040010CD030010EA030010EB030010EC030010ED030010EE030010F0030010DE03001069
:40758000CE03001005040010F6030010F3030010F7030010E8030010E9030010F8030010F9030010FA030010FB030010D7030010D8030010D9030010DA030010DB030010F3
:4075C000DC030010DD0300100F040010FF030010000400101004001004040010DF030010CF030010D003001049205CF024FE002001210090CDE9010103460A46FE4903909C
:407600004A205CF018FE00200222CDE9000202900346FA4903904D205CF00DFE00200222CDE9000202900346F54903904E205CF002FE002000900190029003460322F14930
:40764000039051205CF0F7FD002000900190029003460322EC49039052205CF0ECFD002000900190029003460322E849039053205CF0E1FD0021E64800785CF00AFD002139
:40768000E44800785CF005FD0021E34800785CF000FD0121E14800785CF0FBFC0021E04800785CF0F6FC0021DE4800785CF0F1FC0021DD4800785CF0ECFC0121DB4800781F
:4076C0005CF0E7FC0121DA4800785CF0E2FC0121D84800785CF0DDFC0021D74800785CF0D8FC0021D54800785CF0D3FC0021D44800785CF0CEFC1FBD1FB50121084662F0B0
:40770000CCFD0121042062F0C8FD0121082062F0C4FD0121102062F0C0FD002000900190029003460322C749039001205CF083FD002000900190029003460322C2490390B5
:4077400002205CF078FD002000900190029003460322BE49039010465CF06DFD002000900190029003460322B949039004205CF062FD00200222CDE900020290034603229E
:40778000B449039005205CF056FD002002220123CDE90120009303900346AF4906205CF04AFD002002220123CDE90120009303900346AA4907205CF03EFD0020022201235F
:4077C000CDE90120009303900346A54908205CF032FD002000900190029001230222A149039009205CF027FD00200121CDE9000103460A46CDE902108F490B205CF01BFDC0
:40780000002001210090CDE9010103460A46874903900C205CF00FFD00200121CDE9000103460A46CDE9021080490C205CF003FD0020009001900290034601227749039011
:4078400019205CF0F8FC002000900190029003460122714903901A205CF0EDFC002002220092CDE9012003467F4903901B205CF0E2FC0020009001900290034602467B49B6
:4078800003901C205CF0D7FC002002220092CDE901200346764903901F205CF0CCFC002002220092CDE9012003467249039020205CF0C1FC00200090019002900346032271
:4078C0006D49039021205CF0B6FC0020009001900290034603226949039024205CF0ABFC002001210090CDE9010103460A466449039025205CF09FFC002001210090CDE92C
:40790000010103460A465F49039026205CF093FC0020009001900290034601225A49039027205CF088FC0020009001900290034601225649039029205CF07DFC0020009095
:407940000190029001230222514903902A205CF072FC0020009001900290034602224D4903902B205CF067FC002000900190029003460222484903902C205CF05CFC002094
:40798000009001900290034601224449039031205CF051FC002001210090CDE9010103460A463F49039032205CF045FC00200121CDE9000103460A46CDE902101C4933206F
:4079C0005CF039FC00200121CDE9000103460A46CDE90210194934205CF02DFC00200121CDE9000103460A46CDE90210114935205CF021FC002055E0DE030010E0030010D6
:407A0000E10300100C0400100D0400100E040010CA030010FD030010EA030010EB030010040400100A0400100B040010F6030010F8030010FA030010F7030010F90300107B
:407A4000FB030010D1030010D2030010D3030010D403001007040010E2030010E3030010E4030010E5030010EC03001009040010ED030010EE030010EF030010D503001066
:407A8000F0030010F1030010F2030010D6030010F303001000040010FF030010E8030010E90300100121CDE9000103460A46CDE90210FE4936205CF0BEFB00200121CDE9DA
:407AC000000103460A46CDE90210F94937205CF0B2FB00200121CDE9000103460A46CDE90210F44938205CF0A6FB002001210090CDE9010103460A46EF49039039205CF023
:407B00009AFB002000900190029003460122EB4903903A205CF08FFB002001210090CDE9010103460A46E64903903B205CF083FB002001210090CDE9010103460A46E14923
:407B400003903C205CF077FB00200121CDE9000103460A46CDE90210DB493D205CF06BFB00200121CDE9000103460A46CDE90210D6493E205CF05FFB00200090019002907B
:407B800003460122D24903903F205CF054FB002000900190029003460222CE49039041205CF049FB002000900190029003460222C949039042205CF03EFB002000900190C9
:407BC000029003460122C549039043205CF033FB002000900190029003460122C049039044205CF028FB002000900190029003460122BC49039045205CF01DFB002000900B
:407C00000190029003460122B749039046205CF012FB002002220092CDE901200346B349039047205CF007FB002001210090CDE9010103460A46AE49039048205CF0FBFAD3
:407C400000200222CDE90002029003460246A94903904A205CF0EFFA00200222CDE90002029003460246A44903904B205CF0E3FA0020009001900290034602469F490390AF
:407C80004C205CF0D8FA002002220092CDE9012003469B4903904D205CF0CDFA002002220092CDE901200346964903904E205CF0C2FA01200021009101910B460246CDE9BB
:407CC000021091494F205CF0B6FA01200021009101910B460246CDE902108C4950205CF0AAFA0020009001900290034603228849039051205CF09FFA002000900190029064
:407D0000034603228349039052205CF094FA0020009001900290034603227F49039053205CF089FA00216A4800785CF0B2F900217A4800785CF0ADF90121794800785CF016
:407D4000A8F90021684800785CF0A3F900216E4800785CF09EF900216C4800785CF099F90121704800785CF094F901216E4800785CF08FF901216D4800785CF08AF9002146
:407D80006B4800785CF085F900216A4800785CF080F90021454800785CF07BF91FBD1FB50020009001900290034602466249039001205CF040FA00200090019002900346C3
:407DC00002465D49039002205CF035FA0020009001900290034602465749039003205CF02AFA0020009001900290034602465249039004205CF01FFA00200090019002904D
:407E0000034602464C49039005205CF014FA0020009001900290034602464749039006205CF009FA0020009001900290034602464149039007205CF0FEF9002000900190E2
:407E40000290034602463C49039008205CF0F3F90020009001900290034602463649039009205CF0E8F9002000900190029003460246314903900A205CF0DDF9002000902E
:407E800001900290034602462B4903900B205CF0D2F9002000900190029003460246264903900C205CF0C7F9002047E0FB030010D7030010D8030010D9030010FC03001002
:407EC000DA030010DB030010DC030010DD030010FD030010CF030010D003001001040010020400100304001004040010DF030010DE03001005040010060400100804001067
:407F0000E0030010E10300100A0400100B0400100C0400100D0400100E040010EA030010EB030010F6030010F8030010FA030010F7030010F9030010C9030010009001908B
:407F4000029003460246FE4903900D205CF073F9002000900190029003460246F849039011205CF068F9002000900190029003460246F349039012205CF05DF90020009052
:407F80000190029003460246ED49039017205CF052F9002000900190029003460246E849039018205CF047F9002000900190029003460246E249039019205CF03CF900208E
:407FC00000900190029003460246DD4903901B205CF031F9002000900190029003460246D74903901C205CF026F9002000900190029003460246D24903901F205CF01BF964
:40800000002000900190029003460246CC49039020205CF010F9002000900190029003460246C749039021205CF005F9002000900190029003460246C149039022205CF07E
:40804000FAF8002000900190029003460246BC49039023205CF0EFF8002000900190029003460246B649039024205CF0E4F8002000900190029003460246B1490390252004
:408080005CF0D9F8002000900190029003460246AB49039026205CF0CEF8002000900190029003460246A649039027205CF0C3F8002000900190029003460246A04903904C
:4080C00028205CF0B8F80020009001900290034602469B49039029205CF0ADF8002000900190029003460246954903902A205CF0A2F80020009001900290034602469049E5
:4081000003902B205CF097F80020009001900290034602468A4903902C205CF08CF8002000900190029003460246854903902D205CF081F800200090019002900346024665
:408140007F4903902E205CF076F80020009001900290034602467A4903902F205CF06BF80020009001900290034602467449039030205CF060F80020009001900290034620
:4081800002466F49039031205CF055F80020009001900290034602466949039032205CF04AF80020009001900290034602466449039033205CF03FF800200090019002906C
:4081C000034602465E49039034205CF034F80020009001900290034602465949039035205CF029F80020009001900290034602465349039036205CF01EF800200090019001
:408200000290034602464E49039037205CF013F80020009001900290034602464849039038205CF008F80020009001900290034602464349039039205BF0FDFF0020009044
:4082400001900290034602463D4903903A205BF0F2FF002000900190029003460246384903903B205BF0E7FF002000900190029003460246324903903C205BF0DCFF002083
:40828000009001900290034602462D4903903D205BF0D1FF002000900190029003460246274903903E205BF0C6FF002000900190029003460246224903903F205BF0BBFF5E
:4082C0000020009001900290034602461C49039040205BF0B0FF0020009001900290034602461749039041205BF0A5FF0020009001900290034602461149039042205BF023
:408300009AFF0020009001900290034602460C49039043205BF08FFF0020009001900290034602460649039044205BF084FF0020009001900290034602460149039001E082
:40834000C903001045205BF076FF002000900190029003460246FE49039046205BF06BFF002000900190029003460246F849039047205BF060FF002000900190029003463E
:408380000246F349039048205BF055FF002000900190029003460246ED49039049205BF04AFF002000900190029003460246E84903904A205BF03FFF002000900190029087
:4083C00003460246E24903904B205BF034FF002000900190029003460246DD4903904C205BF029FF002000900190029003460246D74903904D205BF01EFF0020009001901C
:40840000029003460246D24903904E205BF013FF002000900190029003460246CC4903904F205BF008FF002000900190029003460246C749039050205BF0FDFE0020009066
:408440000190029003460322C249039051205BF0F2FE002000900190029003460322BE49039052205BF0E7FE002000900190029003460322B949039053205BF0DCFE1FBD5A
:408480001FB50024FFF78BFC0CE00020B44901EB041189680870B24901EB0411C9680870601CC4B2542CF0DB5BF0BFFC5BF0B0FD0121022061F0F1FE00200090019002909D
:4084C00003460122A749039016205BF0B4FE002001210090CDE9010103460A46A24903901E205BF0A8FE002001210090CDE9010103460A469D4903901A205BF09CFE5CF083
:40850000BBF9FF281CD05BF04AFD0C2816D2DFE800F015060A070B0E0C0D0F10111200BFFFF7EAF80BE000BF00BF00BF00BF00BF00BF00BF00BFFEF7E9FD00E000BF00BFBC
:408540001FBD10B500208A4908705EF075FBFA205EF0DBFBFFF794FFEFF7C8FE002211468448DFF814C200DF002010BD38B50446002560680090009D206880F3088800BF65
:40858000A84738BD10B50120794908705EF090FB77494860012061F031FD1CE0612061F0CFFC78B145F25550744908600120486040F6B83088604CF6CC40086002206C49B7
:4085C000087008E06A4948685EF0ADFB642802D9032067490870664800780128DED010BD10B572B66FF0040000F038FA6FF0010000F034FA4FF0FF3000F030FA042000F0BA
:408600002DFA052000F02AFA062000F027FA072000F024FA082000F021FA092000F01EFA0A2000F01BFA0B2000F018FA0C2000F015FA0D2000F012FA0E2000F00FFA0F2004
:4086400000F00CFA102000F009FA112000F006FA122000F003FA132000F000FA142000F0FDF9152000F0FAF9162000F0F7F9172000F0F4F9182000F0F1F9192000F0EEF906
:408680001A2000F0EBF91B2000F0E8F91C2000F0E5F91D2000F0E2F91E2000F0DFF91F2000F0DCF9202000F0D9F9212000F0D6F9222000F0D3F9232000F0D0F9242000F054
:4086C000CDF9252000F0CAF9262000F0C7F9272000F0C4F9282000F0C1F9292000F0BEF92A2000F0BBF92B2000F0B8F92C2000F0B5F92D2000F0B2F92E2000F0AFF92F200F
:4087000000F0ACF9302000F0A9F9312000F0A6F9322000F0A3F9332000F0A0F9342000F09DF9352000F09AF9362000F097F9372000F094F9382000F091F9392000F08EF92A
:408740003A2000F08BF93B2000F088F93C2017E0C90300100C0400100D0400100E04001068791708E6030010E7030010EA030010A00000103D0A0208CD000908003000408E
:4087800000F06CF93D2000F069F93E2000F066F93F2000F063F9402000F060F9412000F05DF9422000F05AF9432000F057F9442000F054F9452000F051F9462000F04EF9E8
:4087C000472000F04BF9482000F048F9492000F045F94A2000F042F94B2000F03FF94C2000F03CF94D2000F039F94E2000F036F94F2000F033F9502000F030F9512000F064
:408800002DF96FF0040000F032F96FF0010000F02EF94FF0FF3000F02AF9042000F027F9052000F024F9062000F021F9072000F01EF9082000F01BF9092000F018F90A2058
:4088400000F015F90B2000F012F90C2000F00FF90D2000F00CF90E2000F009F90F2000F006F9102000F003F9112000F000F9122000F0FDF8132000F0FAF8142000F0F7F8DB
:40888000152000F0F4F8162000F0F1F8172000F0EEF8182000F0EBF8192000F0E8F81A2000F0E5F81B2000F0E2F81C2000F0DFF81D2000F0DCF81E2000F0D9F81F2000F039
:4088C000D6F8202000F0D3F8212000F0D0F8222000F0CDF8232000F0CAF8242000F0C7F8252000F0C4F8262000F0C1F8272000F0BEF8282000F0BBF8292000F0B8F82A20EC
:4089000000F0B5F82B2000F0B2F82C2000F0AFF82D2000F0ACF82E2000F0A9F82F2000F0A6F8302000F0A3F8312000F0A0F8322000F09DF8332000F09AF8342000F097F802
:40894000352000F094F8362000F091F8372000F08EF8382000F08BF8392000F088F83A2000F085F83B2000F082F83C2000F07FF83D2000F07CF83E2000F079F83F2000F0D8
:4089800076F8402000F073F8412000F070F8422000F06DF8432000F06AF8442000F067F8452000F064F8462000F061F8472000F05EF8482000F05BF8492000F058F84A20EB
:4089C00000F055F84B2000F052F84C2000F04FF84D2000F04CF84E2000F049F84F2000F046F8502000F043F8512000F040F862B610BD00BFBFF34F8F2148006800F4E060A8
:408A000020490843001D1E490860BFF34F8F00BF00BFFEE74AF6AA201B49086070472DE9FC4106460C4617469846089D0020009001902078B0280DD16078102802D011289B
:408A400005D103E0142003F067F901E000E000BF00BF00E000BF00BFBDE8FC8100F01F0201219140094A430942F82310704700F01F0201219140064A430942F8231070476C
:408A80000CED00E00000FA050030004080E100E080E200E010B52DED088B0446FE4890F83800002840D1FD4890F8380000283BD194F8DC00032829D103F000F842F210718A
:408AC000884223D9F449086B4FF4FA615EF00AF938B9F249086B4FF4FA615EF003F9002813D00120EC4981F83800EC4981F838005EF0DEF8E84908635EF0DAF8E749086317
:408B00005EF0D6F8E649C1F83004E0E35EF0D0F8E14908635EF0CCF8E04908635EF0C8F8DF49C1F83004F0E794F8DC0038B90020D94981F83800D94981F83800E5E70120E3
:408B4000D54981F83800D54981F83800F7F72DFFF0EE408A02F09BFE00287CD0D4ED310AB0EE600A4FF0FF31CB4808300FF03FF894ED310AC848D0ED020A30EE600AB0EEE7
:408B8000408A28EE080AB0EE408A4FF0FF311030B0EE480A0FF02BF8BF4890ED040A10EE101A084678F0CAFB41EC1B0BB0EE4B0AF0EE6B0A75F068FEB0EE40AAF0EE60AA91
:408BC0009FEDB80B53EC102B51EC1A0B78F0C0F841EC190B77F030FDAF498862084690ED020AB0EEC00AD0ED0A0A30EE200A80ED0A0AD4ED320AB0EE600A4FF0FF311830CE
:408C00000EF0F5FF94ED320AA348D0ED060A30EE600AB0EE408A28EE080AB0EE408A4FF0FF312030B0EE480A0EF0E1FF9A4890ED080A10EE101A084678F080FB41EC1B0BA3
:408C4000B0EE4B0AF0EE6B0A75F01EFEB0EE40AAF0EE60AA00E0F2E39FED920B53EC102B51EC1A0B78F074F841EC190B77F0E4FC8949C862084690ED060AB0EEC00AD0ED9B
:408C80000B0A30EE200A80ED0B0AD4ED350AB0EE600A4FF0FF310EF0AAFF7F49086B5EF042F87D49496B08447B4948635EF000F879490863D4ED310AB0EE600A4FF0FF31D9
:408CC000764808300EF093FF94ED310A7348D0ED020A30EE600AB0EE408A28EE080AB0EE408A4FF0FF311030B0EE480A0EF07FFF6A4890ED040A10EE101A084678F01EFBDF
:408D000041EC1B0BB0EE4B0AF0EE6B0A75F0BCFDB0EE40AAF0EE60AA9FED620B53EC102B51EC1A0B78F014F841EC190B77F084FC5A498862084690ED020AB0EEC00AD0ED02
:408D40000A0A30EE200A80ED0A0AD4ED320AB0EE600A4FF0FF3118300EF049FF94ED320A4E48D0ED060A30EE600AB0EE408A28EE080AB0EE408A4FF0FF312030B0EE480AC5
:408D80000EF035FF454890ED080A10EE101A084678F0D4FA41EC1B0BB0EE4B0AF0EE6B0A75F072FDB0EE40AAF0EE60AA9FED3D0B53EC102B51EC1A0B77F0CAFF41EC190BAB
:408DC00077F03AFC3549C862084690ED060AB0EEC00AD0ED0B0A30EE200A80ED0B0AD4ED350AB0EE600A4FF0FF310EF000FF2B49086B5DF098FF2949496B08442749486383
:408E00005DF056FF25490863D4ED310AB0EE600AFF2126480EF01CFF94ED310A2448D0ED000A30EE600AB0EE408A28EE080AB0EE408AFF210830B0EE480A0EF009FF1D48EA
:408E400090ED000A10EE101A084678F077FA41EC1B0BB0EE4B0AF0EE6B0A75F015FDB0EE40AAF0EE60AA9FED0F0B53EC102B51EC1A0B77F06DFF41EC190B77F0DDFB0E4960
:408E800088620B4890ED000AB0EEC00A0846D0ED0A0A30EE200A11E0102800104C280010883800100000000000000040902C00109030001098340010883C001080ED0A0A85
:408EC000D4ED320AB0EE600AFF21A0F5FD600EF0BFFE94ED320AFE48D0ED000A30EE600AB0EE408A28EE080AB0EE408AFF210830B0EE480A0EF0ACFEF64890ED000A10EEA3
:408F0000101A084678F01AFA41EC1B0BB0EE4B0AF0EE6B0A75F0B8FCB0EE40AAF0EE60AA1FED200B53EC102B51EC1A0B77F010FF41EC190B77F080FBE6492039C862E44881
:408F400090ED000AB0EEC00A0846D0ED0B0A30EE200A80ED0B0AD4ED350AB0EE600AFF21A0F5A0500EF074FED9491839D1F830045DF0D9FED6491839D1F834140144D44885
:408F80001838C0F834145DF093FED1491839C1F8300400BFD04890ED020AD04880ED940A042200F51471CE48006800F51470FCF767FF00BF00BFC848C168CA48C0F88C1596
:408FC000042200F28C51C648006800F51570FCF757FF00BF00BFC04890ED040ABF4880ED960A042200F51671BD48006800F51670FCF746FF00BF00BFB7484169B948C0F87C
:409000009415042200F29451B548006800F51770FCF736FF00BF00BFAF4890ED060AAF4880ED980A042200F51871AD48006800F51870FCF725FF00BF00BFA748C169A9485C
:40904000C0F89C15042200F29C51A548006800F51970FCF715FF00BF00BF9F4890ED080A9E4880ED9A0A042200F51A719C48006800F51A70FCF704FF00BF00BF9648416A4F
:409080009848C0F8A415042200F2A4519448006800F51B70FCF7F4FE00BF00BF8E4890ED000A8E4880ED9C0A042200F51C718C48006800F51C70FCF7E3FE00BF00BF864860
:4090C00041688848C0F8AC15042200F2AC518448006800F51D70FCF7D3FE00BF00BF7E48416B8048C0F8B015042200F5B6617C48006800F51E70FCF7C3FE00BF7648406BFD
:40910000794988427ED9744890ED0A0ADFED770A20EE200A80ED0A0A90ED0A0ADFED740AB4EEE00AF1EE10FA03DD9FED710A80ED0A0A694890ED0B0A6E48D0ED000A20EE73
:40914000200A654880ED0B0A90ED0B0ADFED6A0A20EE200A80ED0B0A90ED0B0ADFED640AB4EEE00AF1EE10FA03DD9FED610A80ED0B0A594890ED000ADFED5C0A20EE200ADE
:4091800080ED000A90ED000ADFED590AB4EEE00AF1EE10FA03DD9FED560A80ED000A57480078401C5549087008460078322801DB0020087000BF514801784A4880F8441777
:4091C000012200F244714648006800F20C40FCF757FE00BF00BF404890ED0A0ABCEEC00A10EE100AC1B24648444A127881540246424B1B78D1183A4A126802F2AE223F4B7B
:409200001B7800E017E1D0180122FCF739FE00BF00BF314890ED0B0ABCEEC00A10EE100AC1B237483230354A127881540246334B1B78D1182A4A126802F538722F4B1B7869
:40924000D0180122FCF71CFE00BF00BF224890ED000ABCEEC00A10EE100AC1B228483238264A127881540246244B1B78D1181C4A126802F51F72214B1B78D0180122FCF727
:40928000FFFD00BF3C21144870F0EFFD5DF010FD1149086300BF084690ED020A0F4880ED940A042200F514710D48006800F51470FCF7E6FD00BF00BF0748C1680948C0F82C
:4092C0008C15042200F28C51054800681AE0C4E0A0380010A83C00104C280010B01D00108C000010781A001080EE360000007A4400007F43F06B0A080000C842F00000106F
:409300005E20001000F51570FCF7BAFD00BF00BFFD4890ED040AFD4880ED960A042200F51671FB48006800F51670FCF7A9FD00BF00BFF5484169F748C0F89415042200F25D
:409340009451F348006800F51770FCF799FD00BF00BFED4890ED060AEC4880ED980A042200F51871EA48006800F51870FCF788FD00BF00BFE448C169E648C0F89C15042219
:4093800000F29C51E248006800F51970FCF778FD00BF00BFDC4890ED080ADC4880ED9A0A042200F51A71DA48006800F51A70FCF767FD00BF00BFD448416AD648C0F8A41516
:4093C000042200F2A451D248006800F51B70FCF757FD00BF00BFCC4890ED000ACB4880ED9C0A042200F51C71C948006800F51C70FCF746FD00BF00BFC3484168C548C0F809
:40940000AC15042200F2AC51C148006800F51D70FCF736FD00BF00BFBB48416BBD48C0F8B015042200F5B661B948006800F51E70FCF726FD00BF4920EFF746F80DE0FFE73B
:409440005DF036FCB44908635DF032FCAE4908635DF02EFCB149C1F83004BDEC088B10BD10B5044602F0A7FA18B9002084F8DC003FE094ED310AB0EEC00ADFEDA90AB4EE72
:40948000E00AF1EE10FA11D294ED320AB0EEC00ADFEDA40AB4EEE00AF1EE10FA06D2032084F8DC002520F3F744FE22E094ED310AB0EEC00AF7EE000AB4EEE00AF1EE10FA94
:4094C00011D294ED320AB0EEC00ADFED970AB4EEE00AF1EE10FA06D2022084F8DC002620F3F727FE05E02620F3F723FE012084F8DC0094F8DD0094F8DC10884206D094F81F
:40950000DC0084F8DD001320EEF7DEFF10BD10B50446F7F74AFA84ED040AF8F70BFE84ED030AF8F7E3FD84ED010AF8F7F1FD84ED000A10BD774A92F878130E297CD2DFE86C
:4095400001F07BB507427CE2E1E0B67B7BB7080900BF00BF9FED750A80ED0E0A9FED740A80ED0F0A9FED730A80ED100A9FED720A80ED110A9FED6A0A80ED120A9FED6F0AA2
:4095800080ED130A9FED6E0A80ED140A9FED6D0A80ED150A9FED6C0A80ED160A9FED6B0A80ED170A9FED6A0A80ED180A9FED690A80ED190A9FED680A80ED1A0AB5EE000A8B
:4095C00080ED1B0A53E19FED650A80ED0E0A9FED640A80ED0F0A9FED520A80ED100A9FED610A80ED110A9FED600A80ED120A9FED5F0A80ED130A9FED5E0A80ED140A9FEDAE
:409600005D0A80ED150A9FED5C0A80ED160A9FED5B0A80ED170A9FED5A0A80ED180A9FED590A80ED190A9FED580A80ED1A0A9FED570A80ED1B0A1AE1DDE09FED550A80ED2D
:409640000E0A9FED530A80ED0F0A9FED520A80ED100A9FED510A80ED110A9FED500A80ED120A9FED350A80ED130A9FED2D0A80ED140A9FED320A80ED150A9FED340A80EDE8
:40968000160AB5EE000A80ED170A9FED450A80ED180A9FED440A80ED190A9FED430A80ED1A0A9FED420A80ED1B0AE0E000BF00BF9FED3F0A80ED0E0A9FED380A80ED0F0ABB
:4096C0009FED3C0A80ED100A9FED3B0A80ED110A9FED3A0A80ED120A9FED390A80ED130A9FED380A80ED140A9FED370A80ED150A9FED360A80ED160A9FED350A80ED170AA2
:4097000068E079E079E079E04C280010B01D00108C000010781A001010280010883800109A99993E295C0F3D0E2DB23DEC51183F46B6F33E5C8FC23EC3F5A83E295C8F3E7E
:40974000713D8A3E14AE873EDD24863EB81E853E9318843E6F12833E2506813E713D0A3F83C0CA3E5C8F823EEDD46C3E2366563E24ED463E74B73B3EC329333EA6422C3E98
:409780000D6F263E06A0213E707C1D3E9A99193E9A99193F8FC2F53E3D0AD73EA470BD3E8FC2753ED7A3703E1F856B3ED578693ECDCCCC3E7B14AE3E52B89E3E745F8E3E69
:4097C00028636C3E4E9D473E97FD2A3E520E163EF967063E9FEDFE0A80ED180A9FEDFD0A80ED190A9FEDFC0A80ED1A0A9FEDFB0A80ED1B0A3BE000BF00BF00BFB7EE000ADD
:4098000080ED0E0AB7EE000A80ED0F0AB7EE000A80ED100AB7EE000A80ED110AB7EE000A80ED120AB7EE000A80ED130AB7EE000A80ED140AB7EE000A80ED150AB7EE000A6C
:4098400080ED160AB7EE000A80ED170AB7EE000A80ED180AB7EE000A80ED190AB7EE000A80ED1A0AB7EE000A80ED1B0A00BF00BF704710B50446DA4804705420EEF724FECB
:409880005D20EEF721FE10BD10B52DED068B3C21D44870F0EAFA3C21D34870F0E6FA41F23C41D24870F0E1FAFF21D0480EF042FAFF21CF480EF03EFAFF21CE480EF03AFA29
:4098C000FF21CD480EF036FAFF21CC480EF032FACB4890F84407CB490870CB4890ED940AC14880ED020AC648D0F88C15BE48C160C54890ED960ABC4880ED040AC048D0F86E
:409900009415B9484161C04890ED940AB64880ED060ABB48D0F88C15B348C161BA4890ED960AB14880ED080AB548D0F89415AE484162B54890ED9C0AAB4880ED000AB04894
:40994000D0F8AC05A8494860AD48D0F8B0054863084690ED040A10EE101A084677F0EEFC41EC1A0BB0EE4A0AF0EE6A0A74F08CFFB0EE409AF0EE609A9FEDA40B53EC102B8E
:4099800051EC190B77F0E4F941EC180B76F054FE95498862084690ED020AB0EEC00AD0ED0A0A30EE200A80ED0A0A90ED080A10EE101A084677F0C2FC41EC1A0BB0EE4A0AEB
:4099C000F0EE6A0A74F060FFB0EE409AF0EE609A9FED8E0B53EC102B51EC190B77F0B8F941EC180B76F028FE7F49C862084690ED060AB0EEC00AD0ED0B0A30EE200A80ED52
:409A00000B0A4920EEF760FDBDEC068B10BD4FF6FF7601217F4880F8581100207E4981F8DC009FED7E0A084680ED380A9FED7B0A7B4880ED000ABFEE000A7A4880ED000A53
:409A400000207949088090217348E83070F00DFAFFF71AFF0120FFF70CFF6F48C43073490860001D72490860001D72490860001D71490860001D714908600830704908603A
:409A8000001D70490860DFF8C0C100DF074639460220DFF8B8C100DF04215E4880F8581100BF002231464CF20300DFF8A4C100DF85B2012DF5D0DFF89CC100DF044604F435
:409AC000004028B14FF416760321524880F8581104F4804028B14FF6FF7604214D4880F8581104F0020090B301214B4880F8D810434890F87873082F04D0092F07D00A2F5A
:409B00000FD109E054F0CCFE534908600EE055F099FD5149086009E055F014F94E49086004E055F0EFFE4C49086000BF00BF4A4800680168384888473748FFF7FBFC9FED0A
:409B4000470A6BF09FFC464880ED000A00BF04F001000028A5D03048C430FFF7D8FC2E48FFF77EFC3C4800683E4942682A4890472948FEF78FFF6AF04DFE92E770B52DED75
:409B8000028BB0EE408A04460225022C72DA9FED360AB4EEC08AF1EE10FA04DD9FED320AB0EE408A0AE09FED310AB4EEC08AF1EE10FA03D29FED2D0AB0EE408A00BF2C485A
:409BC00000EB840080ED008A294A02EB840152E007EAF43DC6BEE43D08ACDC3D3D0AD73DD4000010102800104C28001088280010902C001098300010A0340010A838001011
:409C0000781A0010F0000010B01D0010000000000000004000190020C43C001000000000CC000010E0000010F2000010B0000010B4000010B8000010BC000010C000001066
:409C4000C8000010C4000010F904090881F80808E1F8080829F80808F400001044D8F03BD0000010E8000010003C1C46003C1CC60822001014E0FB4A126802F58B6202EBEA
:409C800084000422FCF7FCF800BFF748D0F854110220DFF8D8C300DFA720EEF715FC00252846BDEC028B70BDF14890F8DC007047F04800797047F0EE400A90ED010AB0EEB8
:409CC000401A9FEDED0AF4EEC00AF1EE10FA03D29FEDE90AF0EE400A81EE200A7047E44890ED5E0A7047E54800787047B0EE401AF0EE601AB0EE410AE14991F830150229A6
:409D000002D19FEDE02A01E09FEDDF2AB4EEE12AF1EE10FA0BDDDA4991F83015022902D19FEDD82A01E09FEDD82AF0EE421A90ED1F2A61EEA12AC2EE220AB4EEE01AF1EE69
:409D400010FA05DDB0EE600A0121D04A117011E0B1EE602AB4EEC21AF1EE10FA07D2B1EE602AB0EE420A0121C84A117002E00021C64A11707047C548007870470020C3495D
:409D800008707047B0EE401AF0EE411ABC4890F83005022802D19FEDBB0A01E09FEDBA0AB4EEE00AF1EE10FA2DDDB94890ED002A31EEC22AB0EE420AB64890ED002AB4EEA0
:409DC000C20AF1EE10FA09DDB14890ED002AB148D0ED002A32EE222AF0EE421AAD4890ED002AB1EE422AB4EEC20AF1EE10FA09D2A74890ED002AA748D0ED002A32EE622AB1
:409E0000F0EE421A00BFB0EE610A70475FED7D0AB0EE600A9748007920B19648D0ED000AB0EE600A70475FED830AB0EE600A9148007950B18F4890ED001ADFED971ADFED16
:409E4000970A41EE210AB0EE600A704710B52DED028BF9F7DBFA00EE100AB8EE400ADFED8F0A30EE600ADFED8C0A80EE201AB0EE418AB2EE040AB4EEC08AF1EE10FA03DD3C
:409E8000B2EE040AB0EE408ABAEE040AB4EEC08AF1EE10FA03D2BAEE040AB0EE408AB0EE480ABDEC028B10BD0146F0EE400AB7EE000AB0EE401A7148007878B3F2EE0A1AA5
:409EC000F4EEE10AF1EE10FA03DBDFED751AF0EE610AFDEEE01A11EE902A10B201EE900AF8EEE11A30EEE10A01F13802431C02EB8302D2ED001A01F1380202EB800292ED67
:409F0000002A31EEC22A01F1380202EB8002D2ED001A40EE021AB0EE611A00BFB0EE410A70470020564991F87813042900D0012070472DE9F04104460D461646FAF7BEFF20
:409F400008B1642000E0C82007464FF00008BC4203DD3C464FF0020819E0FAF7AFFF28B1012C03DA01244FF0030810E04348007828B1322C03DA32244FF0030807E03F48A0
:409F8000007820B9012C02DA01244FF00308022D2BDA00BF434800EB850020F81640414A02EB850202EB46012E4A126802F5947202EB850202EB46000222FBF761FF00BF7E
:409FC0000D20EEF781FA212029F07EF82648D0F854110220DFF894C000DF2348D0F808120120DFF888C000DF01E04FF002084046BDE8F0812DE9F04105460C4616460027A4
:40A00000FF2D02DDFF25022703E0002D01DA00250327022C48DA00BF2248083000EB840020F816501F4A083202EB840202EB46010C4A126802F5987202EB840202EB46002F
:40A040000222FBF71DFF00BF0E20EEF73DFA212029F03AF80448D0F854110220DFF80CC000DF22E08C0000100019002081F80808C43C0010E80000102FDDE43ED400001082
:40A08000781A00100AD7A33C9A99193EE4000010CC000010D000001000007A4400401C460AD74F41D81E001002273846BDE8F0812DE9F04105460C4616460027FF2D02DDFE
:40A0C000FF25022703E0002D01DA00250327022C24DA00BFFE4800EB840020F81650FC4A02EB840202EB4601FA4A126802F59C7202EB840202EB46000222FBF7C1FE00BFD1
:40A100000F20EEF7E1F9212028F0DEFFF248D0F854110220DFF8C4C300DF00E002273846BDE8F0812DE9F04105460C4616460027FF2D02DDFF25022703E0002D01DA0025C9
:40A140000327022C26DA00BFE148183000EB840020F81650DE4A183202EB840202EB4601DC4A126802F5A87202EB840202EB46000222FBF785FE00BF8820EEF7A5F9222035
:40A1800028F0A2FFD448D0F854110220DFF84CC300DF00E002273846BDE8F0812DE9F04105460C4616460027FF2D02DDFF25022703E0002D01DA00250327022C26DA00BF33
:40A1C000C348083000EB840020F81650C04A083202EB840202EB4601BE4A126802F5A07202EB840202EB46000222FBF749FE00BF1020EEF769F9212028F066FFB648D0F8FC
:40A2000054110220DFF8D4C200DF00E002273846BDE8F0812DE9F04105460C4616460027FF2D02DDFF25022703E0002D01DA00250327022C26DA00BFA548203000EB84001C
:40A2400020F81650A24A203202EB840202EB4601A04A126802F5AC7202EB840202EB46000222FBF70DFE00BF8920EEF72DF9222028F02AFF9848D0F854110220DFF85CC221
:40A2800000DF00E002273846BDE8F0812DE9F04105460C4616460027FF2D02DDFF25022703E0002D01DA00250327022C26DA00BF8748103000EB840020F81650844A103230
:40A2C00002EB840202EB4601824A126802F5A47202EB840202EB46000222FBF7D1FD00BF1120EEF7F1F8212028F0EEFE7A48D0F854110220DFF8E4C100DF00E002273846E4
:40A30000BDE8F0812DE9F04105460C4616460027C82D02DDC825022703E0012D01DA01250327022C26DA00BF6948303000EB840020F81650664A303202EB840202EB4601D6
:40A34000644A126802F5B47202EB840202EB46000222FBF795FD00BF0C20EEF7B5F8222028F0B2FE5C48D0F854110220DFF86CC100DF00E002273846BDE8F0812DE9F04109
:40A3800005460C4616460027642D02DD6425022703E0012D01DA01250327022C26DA00BF4B48283000EB840020F81650484A283202EB840202EB4601464A126802F5B072A4
:40A3C00002EB840202EB46000222FBF759FD00BF4D20EEF779F8222028F076FE3E48D0F854110220DFF8F4C000DF00E002273846BDE8F08110B50E20EEF766F80F20EEF7D5
:40A4000063F81020EEF760F88820EEF75DF88920EEF75AF81120EEF757F80D20EEF754F80C20EEF751F84D20EEF74EF8212028F04BFE222028F048FE10BDF0B52DED0E8B76
:40A4400097B00446F0EE408AB6EE000AF4EEC08AF1EE10FA03D2B6EE000AF0EE408A94ED1F0A68EEA80A80EE209A94ED210AB4EEC90AF1EE10FA03D294ED210AB0EE409AD8
:40A48000B7EE000AC0EE09EA94ED208A144890F8D00050B1134890F8E004012805D0B6EE000A28EE000AB0EE408AB0EE000A30EE480A60EE2E9A89EE88EA20210FA86FF003
:40A4C000D4FCCDED0F9A9FED080A29EE800A0DE0E81E00108C0000100019002081F80808A8170010781A00106666E63E8DED110A1FED030A2EEE000A20EE080A8DED140A9C
:40A500008DED16EA002661E00127002537E000EE105AB8EE400AB2EE041AC0EE010A9FEDBC0A30EE800AF0EE40AADFEDBA0A7AEEE00AB0EE600A01A90FA80EF088FF03A9D9
:40A54000B0EE6A0A0FA80EF082FFDFEDB20A7AEEA00AB0EE600A05A90FA80EF078FF01A80EF0FBFDB0EE40BAB0EECB0AB4EEC90AF1EE10FA01DD002703E0681C85B2032D3C
:40A58000C5DB00BF07B123E09DED0F0ADFEDA20A20EE200A8DED0F0A9DED110ADFED9E0A20EE200A8DED110A9DED140ADFED9A0A20EE200A8DED140A9DED160ADFED960AB7
:40A5C00020EE200A8DED160A701C86B20A2E9BDB00BF9DED120ADDED100A30EE600AF0EE080A20EE200A8DED0A0A9DED110ADDED0F0A30EE600AF0EE080A20EE200A8DEDDE
:40A60000090A9DED140ADDED120A30EE600AF0EE080A20EE200A8DED0C0A9DED130ADDED110A30EE600AF0EE080A20EE200A8DED0B0A9DED160ADDED140A30EE600AF0EE76
:40A64000080A20EE200A8DED0E0A9DED150ADDED130A30EE600AF0EE080A20EE200A8DED0D0ABDEEE80A10EE100A00B26B4908800846B0F90000042801DA04200880674831
:40A68000B0F900000C2802DD0C20644908806348B0F90000800000EE100AB8EEC00AF7EE000A80EE80AA002575E000EE105AF8EE400A5A48B0F9000000EE100AB8EEC00AE5
:40A6C00080EE801AF0EE41AA3AEE8A0AF0EE40AA07A9B0EE6A0A0FA80EF0B9FE9DED070A05EB450104F1E80000EB810080ED000A07A9B0EE6A0A09A80EF011FF9DED070A2A
:40A70000DDED080A80EE201A11EE106A304676F015FE41EC1D0BB0EE4D0AF0EE6D0A72F097F9B0EE40CAF0EE60CA9FED3D0B53EC102B51EC1C0B76F00BFB41EC1B0B75F016
:40A740007BFF05EB450204F1E80101EB820148607AEECA0AB0EE600A01A90FA80EF077FE03A9B0EE6A0A0FA80EF071FE7AEE8A0AB0EE600A05A90FA80EF069FE01A80EF0C4
:40A78000ECFC05EB450104F1E80000EB810080ED020A681C85B22148B0F90000401EA84283DC9FED210A1D48B0F90000401E00EB400104F1E80000EB810080ED000A9FEDAA
:40A7C0001A0A1648B0F90000401E00EB400104F1E80000EB810080ED010A9FED130A0F48B0F90000401E00EB400104F1E80000EB810080ED020A94ED3C0AF6EE000A20EE2B
:40A80000200A84ED3C0A17B0BDEC0E8BF0BD00009A99993ECDCC4C3DCDCC8C3FF2000010000000000000F0BF000000000021C74A1170C74A117090ED010AC64981ED010AEB
:40A8400090ED000A81ED000A90ED010AC24981ED010A90ED000A81ED000A9FEDC00AC04981ED010A9FEDBD0A81ED000A704730B52DED028B87B004460D46BA48007830B9B1
:40A880002046FFF7D3FF07B0BDEC028B30BD00EE105AB8EE400ADFEDB40A80EE208A9FEDB30AB4EEC08AF1EE10FA00D2EBE7A94890ED010AAA48D0ED010AB6EE001A60EEA5
:40A8C000810A00EE880AA34880ED010A90ED000AA348D0ED000AB6EE001A60EE810A00EE880A9C4880ED000A94ED010A9A48D0ED010A30EE600AC0EE080ACDED060A94ED76
:40A90000000AD0ED000A30EE600AC0EE080ACDED050A9DED060A9248D0ED010A30EE600A8DED040A9DED050AD0ED000A30EE600A8DED030A94ED010A8648D0ED010A30EE3A
:40A94000600A8DED020A94ED000AD0ED000A30EE600A8DED010A9DED040A20EE000ADDED030A9DED031AF0EE408A40EE818AB3EE090AF4EEC08AF1EE10FA7DDD7448007822
:40A980007249087001207249087070480078E0B3704890ED010A7648D0ED010A30EE200A6C4880ED010A90ED000A7148D0ED000A30EE200A674880ED000A94ED010AD0ED55
:40A9C000010A30EE600A8DED020A94ED000AD0ED000A30EE600A8DED010A9DED020ADFED650A20EE200A80ED010A9DED010ADFED610A20EE200A80ED000A94ED010A5648B9
:40AA000080ED010A94ED000A00E002E080ED000A67E09DED060A20EE080A554880ED010A9DED050A20EE080A80ED000A494890ED010A4B48D0ED010AB6EE001A60EE810A89
:40AA400000EE880A434880ED010A90ED000A4448D0ED000AB6EE001A60EE810A00EE880A3C4880ED000A90ED010A3B4880ED010A384890ED000A00E003E0374880ED000A24
:40AA80002FE0002032490870304908709DED040ADFED390A20EE200A314880ED010A9DED030ADFED350A20EE200A80ED000A9DED020ADFED300A20EE200A264880ED010AA8
:40AAC0009DED010ADFED2B0A20EE200A80ED000A94ED010A204880ED010A94ED000A80ED000A1C4890ED010A84ED010A90ED000A84ED000A00BFC6E600201A49087070471C
:40AB00001248007870471D49087070471B4800787047174870470CB50F4890ED010A0D48D0ED010A30EE600A8DED010A0A4890ED000A0848D0ED000A30EE600A8DED000A89
:40AB40009DED000ADDED010A0CBD00001D0100101C01001004010010FC000010000000000C010010F800001000007A440AD7233C14010010CDCCCC3DCDCC4C3E1E010010EB
:40AB80000146FE48062904D2DFE801F0030406080A0C00BFFA4807E0FA4805E0FA4803E0FA4801E0F54800BF00BF704710B50446012C01DA012402E0052C00DD052420469C
:40ABC000FFF7DEFFF249086040F26442002308460168F048FBF7B4FEEF480470EF4880F82A41012200F59571ED48FBF749F9B420EDF76AFC10BDE94890F82A01704770B55A
:40AC000004460D461646062C62D2DFE804F0610315283B4E1E21E14828306FF026F92A463146DE4828306FF07FF81E22DB492831DC48FBF725F94CE01E21D84846306FF006
:40AC4000F2F82A463146D54846306FF06DF81E22D2494631D3481E30FBF712F939E01E21CE4864306FF001F92A463146CB4864306FF05AF81E22C9496431CA483C30FBF783
:40AC8000FFF826E01E21C54882306FF0CCF82A463146C24882306FF047F81E22BF498231C0485A30FBF7ECF813E01E21BB48A0306FF0DBF82A463146B848A0306FF034F859
:40ACC0001E22B649A031B7487830FBF7D9F800E000BF00BFB420EDF7F7FB70BD70B504460D46062C27D2DFE804F026030A11181F1522AA49283128466FF016F81CE01522F1
:40AD0000A649463128466FF00FF815E01522A349643128466FF008F80EE015229F49823128466FF001F807E015229C49A03128466EF0FAFF00E000BF00BF70BDF8B50446BE
:40AD40000025062C63D2DFE804F0620316293C4F0120FFF715FF0646042231466846FBF712F90098C0B2142803D00098C0B2152800D101254CE00220FFF702FF0646042290
:40AD800031466846FBF7FFF80098C0B2142803D00098C0B2152800D1012539E00320FFF7EFFE0646042231466846FBF7ECF80098C0B2142803D00098C0B2152800D101254B
:40ADC00026E00420FFF7DCFE0646042231466846FBF7D9F80098C0B2142803D00098C0B2152800D1012513E00520FFF7C9FE0646042231466846FBF7C6F80098C0B2142846
:40AE000003D00098C0B2152800D1012500E000BF00BF2846F8BD70B50625012406E02046FFF78CFF00B92546601CC4B2052CF6DD284670BD10B5044657480470B420EDF7AF
:40AE400043FB10BD54480078704710B5012407E02046FFF773FF08B1012010BD601CC4B2052CF5DD0020F8E72DE9F041054600272C460026002D3AD02878002837D02846FD
:40AE80006EF0DCFE0746EE1900E0641CF0F7CEFF00682178405C00F001000028F5D1A6420CD000BFF0F7C2FF0168701E06460078085C00F0010008B1A642F3D1E819401E77
:40AEC000B04202D00020707005E0AC4203D0A64201D1002028702E46AC4208D003E014F8010B06F8010B20780028F8D13070BDE8F08110B50446152221462B486EF014FF67
:40AF00002948FFF7B1FF00202749087540F2511031F05CF810BD244870472DE9F04106460D46002415E0AC4211D0611CC8B21F49FFF7D4FE30466EF081FE07463A461B497C
:40AF400030466EF02BFE10B90120BDE8F081601CC4B2052CE7DB0020F7E738B50446002000906A4601212046FFF749FE40F2644108486EF07AFF20461AE000009017006828
:40AF800000060068640A0068C80E00682C1300688C000010B01D00101F010010781A00102A01006828000068AE180020C3180020FFF7E6FD054640F264420D49FAF760FF77
:40AFC00021460620FBF7A9FE40F264420023094801680748FBF7B4FC38BD10B5044620466EF02CFE08B9012010BD0020FCE70000B01D00108C00001000B589B0022172489D
:40B00000007859F0E9F9012104205FF08DF98020ADF81800BDF8180000EE100AB8EE400A6A4880ED000A0020ADF820008DF822006748006807900020ADF81A0006A9654892
:40B040005FF017FB01A85FF0CDFC3020ADF804000020ADF8100003900120ADF8060001A95C485FF087FC00205B4908700846017858485FF087FB09B000BD1FB500215248E8
:40B08000007859F0A9F9002104205FF04DF9002001210090CDE90101034602224A490390402059F0C8F81FBD10B52DED028BB0EE408A9FED4A0AC8EE000A9FED490A20EE90
:40B0C000800AF0EE408AB7EE000AF4EEC08AF1EE10FA03D2B7EE000AF0EE408A9FED410AF4EEC08AF1EE10FA03DD9FED3E0AF0EE408A3D480068800800EE100AF8EE400A39
:40B10000324890ED001A80EE810AC0EE280AB6EE000A30EE800ABCEEC00A10EE100A84B22B480068844219D000202B4908700846017828485FF026FB611E26485FF0E4FAB6
:40B14000002124485FF0DEFA21480460012022490870084601781F485FF014FB9FED230AB4EEC08AF1EE10FA0BD21B480078012807D10020184908700846017815485FF00B
:40B1800001FB9FED1A0AB4EEC08AF1EE10FA0EDB1148007858B901200F490870084601780C485FF0EFFA01210A485FF0CDFABDEC028B10BD0E4991F82913012901D1012039
:40B1C00000E00020704700000F040010300200202C02002000080040340200206DE2E43E0000344200401C46541000200AD7233C781A001000B587B003A804A905AB06AAA4
:40B20000CDE90010CCA1CF486EF038FB4FF44051049841EA00200399084380B207B000BD2DE9F0432DED028B83B005460C4616464FF00008C146002002902868B0F56F4FDC
:40B2400006D0C1490844002879D0FF2872D14FE16868042870D14FF0080920700AF085FFBA48D0ED000A30EE200ADFEDB90A20EE200ABCEEC00A10EE100A80B20290BDF81F
:40B2800008006070BDF808000012A0700AF071FFAE48D0ED000A30EE200ADFEDAD0A20EE200ABCEEC00A10EE100A80B20290BDF80800E070BDF80800001220710AF073FF84
:40B2C0000746012F06DD072F04DA0AF077FFB0EE408A1AE09F4890ED138A90F8D000A0B19A4890ED000A38EE000AB0EE408A9A4890ED000AB4EEC08AF1EE10FA05DD90EDC0
:40B30000000A38EE400AB0EE408A9FED910A28EE000ABCEEC00A10EE100A80B20290BDF808006071BDF808000012A071FF20E07103E004E0F6E0FFE700BF00BFF3E04FF0A3
:40B340000809002020706868B0F57A4F6DD00CDC7B283BD004DC652828D0682873D117E0CA2840D0CB28F9D14EE04FF60322811A904269D007DC6FF47A410844002864D025
:40B380000128EBD16FE006297DD00729E6D19FE0032060706820A0700020E07020716071A0716E4890F87805E0719FE0132060706520A0700020E070FFF71CFF0290BDF81E
:40B3C0000800A0800020A071E0718FE0332060707B20A0700020E07005F025FE8DED010A0198606082E00B206070CA20A0700020E0705A48B0F87E070290BDF80800E080BB
:40B4000000202071607171E00B206070CB20A0700020E0705148B0F880070290BDF80800E08000202071607160E0132060700020A070FA20E07058F0B2FD20710020607184
:40B44000A071E07152E050E01EE0132060700120A070FA20E07000202071102060710020A071E07142E0132060700220A070FA20E070FFF7BFFE0290BDF80800A080002035
:40B48000A071E07132E016E0132060700320A070FA20E07000202071314890F8420000F01F0060712E4890F84100A0712C4890F84000E0711AE0132060700920A070FA2081
:40B4C000E0700120207100206071A071E0710DE0132060700A20A070FA20E070AA20207100206071A071E07100E000BF00BF1AE04FF00809012020700AF05CFE0290BDF8C1
:40B5000008006070BDF808000012A0700AF04BFEE07054202071C82060718420A0710020E07100E000BF00BFA6F80090404603B0BDEC028BBDE8F08325642E25642E2564D3
:40B540002E2564009CBE00080011E7FFE46B0A0800401C46A8170010EC6B0A08781A0010E87C02202DE9FF4158F027FC0026054658F0DCFBB0460746FB486EF05FFBC4B253
:40B58000012340222146F848CDE90078CDE902560CF045F818B1012004B0BDE8F0810020FAE710B50020F1490870F14908705BF07FFBF0490860FFF7D5FF10B9002005F0DD
:40B5C000ECF810BD10B5EC48007A062870D2DFE800F0035B3490AA76F2F7BDFF90B962F003FF78B963F0E2FF60B962F037F948B901F054F8152805D00020DF494872022008
:40B60000087219E062F02AF928B10020DA4948720120087210E062F0E7FE28B10020D64948720520087207E063F0C0FF20B10020D14948720320087204E1F2F78CFFE8B9C4
:40B6400062F0D2FED0B963F0B1FFB8B962F006F9A0B901F023F8152810D0C448007848B10220C54948720420087266F08EFD0020BE4908700020BE49087004E00220BE49A7
:40B68000487200200872DDE062F0E8F888B1B748007848B10120B84948720420087266F074FD0020B14908700020B149087005E0C4E00120B049487200200872C2E062F04E
:40B6C00093FE80B1A948007848B10520AA4948720420087266F059FD0020A44908700020A349087004E00520A349487200200872A8E063F05BFF80B19C48007848B10320DA
:40B700009D4948720420087200209849087066F03CFD00209649087004E0032096494872002008728EE09448407A022828D1F2F712FFE8B962F058FED0B963F037FFB8B925
:40B7400062F08CF8A0B900F0A9FF152810D088480078002871D0002085490870834908700420854948720220087266F005FD64E00420814948720020087266F0FDFC5CE0D9
:40B780007D48407A01281BD162F068F880B178480078002851D0002075490870734908700420754948720120087266F0E5FC44E00420714948720020087266F0DDFC3CE0F8
:40B7C0006D48407A03281AD163F0F0FE78B16848007850B3002066490870644908700420654948720320087266F0C6FC25E00420614948720020087266F0BEFC1DE05E48A8
:40B80000407A052819D162F0EFFD78B15848007858B1002056490870544908700420564948720520087266F0A7FC06E00420524948720020087266F09FFC03E000204E49CA
:40B84000087200BF00BF4C48807A4B49097A884206D14FF47A71474800685BF043FA68B14548007A444988725BF022FA41490860072027F029FC2E20ECF726FE3E48007A25
:40B88000042803D05BF014FA3B49486010BD3B4890F83005022802D19FED391A01E09FED391AF0EE410AB0EEC01AB4EEE01AF1EE10FA01DD012070470020FCE72F4890F87D
:40B8C0007803072804D02D4890F87803062802D19FED2D0A01E09FED2D0A704710B52DED028BF5F762F8B0EE408AFFF7E7FFF0EE408AB4EEE88AF1EE10FA03D20120BDECF9
:40B90000028B10BD0020FAE710B52DED028B1B4890F87803072804D0184890F87803062802D19FED1A8A01E09FED198AF5F73DF8B4EEC80AF1EE10FA03DD0120BDEC028B7E
:40B9400010BD0020FAE710B52DED028B0B4890F87803072804D0094890F8780306281BD19FED0C8A1AE00000FC1B0010390200203A0200203C020020F0180020781A0010A4
:40B980000AD7A33C9A99193EE3A5AB4083C00041B81E41413D0A0F419FEDCD8AF5F705F8B4EEC80AF1EE10FA03DD0120BDEC028B10BD0020FAE7C749097A042905D1C54985
:40B9C000497A022901D1012100E0002108467047C049097A042905D1BE49497A052901D1012100E0002108467047BA49097A042905D1B849497A032901D1012100E0002170
:40BA000008467047B349097A042904D1B149497A012900D100E0002108467047AD49087A704710B5AB48007A092831D2DFE800F0061B1D1A24193031050000BF00F08FFD40
:40BA400008B108240CE0A448007830B9A348406B00F48010B0F5801F01D1012400E0002419E000BF00BF012415E0F2F7F1FD08B1052400E002240EE0FFF7C4FF08B101247A
:40BA800005E0F2F7E5FD08B1062400E0042402E000BF072400BF00BF204610BD10B503F0A3FE18B101208E49087002E000208C49087010BD01208B490870704710B5854909
:40BAC00048685BF030F910BD87480078704786490870704770B50446002500BF20466EF0ADF8461C3246214680486EF01DF93C227E497F48FAF7C4F900BF284670BD70B507
:40BB00000446002500BF20466EF098F8461C32462146764878386EF007F93C227349783973487838FAF7ACF900BF9A20ECF7CCFC284670BD2DE9FF4704464FF0000958F0B5
:40BB40003CF90026054658F0F1F8B046074620466EF074F800F0FF0A0123402251462046CDE90078CDE902560BF059FD01281BD10220604908702046FFF7C1FF012004F0E9
:40BB80000CFE9E20ECF7A0FC4FF4C37030F01EFA20466EF053F80546234603222121009000205BF078FB24E058F007F90026054658F0BCF8B046074620466EF03FF800F011
:40BBC000FF0A0123402251462046CDE90078CDE902560BF024FD022803D12046FFF77AFF07E09A20ECF770FC0120424908704FF0FF39484604B0BDE8F08770B504460D46E3
:40BC00003022294620466EF006F905223A4920466EF052F92D20607104223749891DA01D6EF04AF92D20A0720C2233490B3104F10B006EF041F90020E07570BD00B587B094
:40BC4000182101A8FFF7D9FF01A8FFF773FF07B000BD2848007870472DE9F04781460F461446C846002548466DF0E8FF08B9A8462BE000260FE02D2140466DF073FF05466B
:40BC800025B9022E01DA4FF0000806E0BE4201DA05F10108761CBE42EDDD00BFB8F1000F09D01DB1A5EB0800207006E040466DF0C5FF207001E00020207020780C2801DC9B
:40BCC000207810B94FF0000800244046BDE8F0878B6C4F41F0180020403E00109C0B0010390200203A0200203B020020741C0010FC01006838020020D818002010B5044650
:40BD000000BFFE48C0F82C43042200F54B71FC48FAF7B6F800BF10BD10B5044600BFF7484461042200F11401F648FAF7A9F800BF10BD10B5044600BFF0480461042200F1D5
:40BD40001001F048001FFAF79BF800BF10BD10B5044600BFE948C460042200F10C01E9480838FAF78DF800BF10BD1CB55AF0A0FFB0F57A7F19D95AF09BFF4EF660218842D4
:40BD800005D95DF004F804465DF004F802E001205DF000F800205CF0B9FF0020009003460122014601905BF099F91CBD10B52DED028B04469FEDD40AB0EE408AD348007898
:40BDC000844212D1D148007858F065FB00EE100AB8EE400ADFEDCE0A20EE200AF7EE000A80EE201AB0EE418A2CE0CA480078844212D1C848007858F04EFB00EE100AB8EE87
:40BE0000400ADFEDC30A20EE200AF7EE000A80EE201AB0EE418A15E0BF480078844211D1BD48007858F037FB00EE100AB8EE400ADFEDB70A20EE200ADFEDB80A80EE201AE1
:40BE4000B0EE418AB0EE480ABDEC028B10BD10B52DED028B04469FEDAC0AB0EE408AB0480078844212D1AE48007858F014FB00EE100AB8EE400ADFEDA60A20EE200ADFEDB0
:40BE8000A90A80EE201AB0EE418A5EE0A648007884421AD1A448007858F0FDFA00EE100AB8EE400AB0EE408ADFED990A9FED9F0A18EE200A9FED9E1AC0EE010A9FED9D0A62
:40BEC00030EE800AB0EE408A3FE09B48007884420ED19948007858F0DEFA00EE100AB8EE400ADFED8B0A20EE200AB0EE408A2CE092480078844212D19048007858F0CBFA3D
:40BF000000EE100AB8EE400ADFED810A20EE200AF5EE000A80EE201AB0EE418A15E07E480078844211D17C48007858F0B4FA00EE100AB8EE400ADFED760A20EE200AF5EE10
:40BF4000000A80EE201AB0EE418AB0EE480ABDEC028B10BD10B52DED028B04469FED6A0AF0EE408A7648007884421ED17448007858F091FA00EE100AB8EE400ADFED640A31
:40BF800020EE200AB0EE408A9FED6E0A38EE400AF0EE040A80EE201AB0EE418AB3EE090A38EE000AF0EE408A19E05B480078844215D15948007858F06EFA00EE100AB8EEAD
:40BFC000400ADFED530A20EE208A9FED5F0A30EE480AF1EE060A80EE201AF0EE418AB0EE680ABDEC028B10BD5849087070472DED028B4FF6FF76DFF858C100DF8146642211
:40C0000001215AF034FFDFF848C100DF814601215AF05CFF5AF04CFE80464E480021016041604D48016041604C48016041605AF03FFE87B231484069464908602F48C0685C
:40C04000454908602D480069444908602B48D0F82C03434908605AF02BFE424908600120414908700220414908705AF021FE4049086001213F48007858F00BF800213E487F
:40C08000007858F006F801213C48007858F001F800202E49087000BF002231460120DFF8E0C000DF0446012CF6D0022CF4D1DFF8D4C000DF054605F00100C0B12648007972
:40C0C000401C2549087125480079401C2349087120480079401C1F49087121480079401C1F4908715CF044F908B15CF00DF9264800780128D0D1F0F77EFB47E0781A00102C
:40C100002C0300681400006800000000D403001000404E3FD3030010EF030010FC7C5740D10300109893823DD203001000E0AB44A470A5C000005CC20D0400100E040010E5
:40C140000C04001000003E4400F80945DD010010F904090820010010380100103001001028010010D8010010DC010010D4010010D001001001040010020400100304001009
:40C18000E1F8080829F808086C0200204FF4FA7138465AF0A7FD88B13A20ECF795F93920ECF792F93820ECF78FF98320ECF78CF94620ECF789F95AF07BFD87B222F0B0FE9E
:40C1C00018B15AF075FD804608E04EF6602140465AF088FD10B10120FFF706FF012058F07AFB012054F071FAE3480078FFF72FFEB0EE408A0A21E1480BF0F9FCE04880ED60
:40C20000000A002054F061FADE480078FFF71FFEB0EE408A0A21DC480BF0E9FCDB4880ED000ADB480078FFF712FEB0EE408A0A21D8480BF0DCFCD84880ED000AD7480078FE
:40C24000FFF788FEB0EE408A0A21D5480BF0CFFCD44880ED000A57F0CEFE00287ED00120D14908700846007800F0010050B10121CE48007857F00DFF0121CD48007857F04C
:40C2800008FF09E00021C948007857F002FF0021C748007857F0FDFEC6480078FFF786FDB0EE408A3221C4480BF0A1FCC34880ED000AC3480078FFF779FDB0EE408A322128
:40C2C000C0480BF094FCC04880ED000A4320ECF7FBF8BE48007802282BD1BD480078FFF739FEB0EE408A0621BA480BF080FCBA4880ED000A4FF49671B84800685AF0F2FC3A
:40C30000002873D00420B14908705AF0D1FCB34908600121B248007857F0BBFE0121B148007857F0B6FE0121AF48007857F0B1FE5CE0A648007804282CD1A5480078FFF7B2
:40C3400086FDB0EE408A0621A8480BF050FCA84880ED000A4FF49671A04800E05AE000685AF0C0FCF0B30120984908705AF0A0FC9A49086001219A48007857F08AFE002199
:40C380009848007857F085FE00219748007857F080FE2BE08E480078FFF708FDB0EE408A062194480BF023FC934880ED000A4FF496718A4800685AF095FC98B1022083495D
:40C3C00008705AF075FC8549086001218448007857F05FFE00218348007857F05AFE0121814800E002E0007857F053FE01201AF031FB20B15AF05CFC804908600AE080495C
:40C400007E4800685AF06EFC20B100217D48007857F03FFE7C4800790A2820DB00207A49087108464079401C4871FFF79EFC764840793C2813DB00207349487108460068E1
:40C44000401C30B10968491C6F4A08461160FFF77EFC1920ECF738F8162026F035FEFFF7AAFA40B9FFF7CEFA28B9FFF7BEFA10B9FFF7AEFAD8B1654800790A2817DB0020BC
:40C480006249087108464079401C4871084640793C280CDB0020487108460068401C30B10968491C594A08461160FFF742FCFFF782FA40B9FFF7A6FA28B9FFF796FA10B981
:40C4C000FFF786FAF0B1524800790A281ADB00204F49087108464079401C4871084640793C280FDB0020487108460068401C30B10968491C464A08461160FFF70DFC192020
:40C50000EBF7E2FF434800790A28FFF6C5AD00204049087108464079401C4871084640793C28F2DB0020487108460068401C30B10968491C374A08461160FFF7DFFB19203A
:40C54000EBF7C2FFA8E503468B4201DB934201DD012070470020FCE72F480078704700B5FFF7FAFF022801D0012000E000200146084600BD704700000E0400105C0100100D
:40C580009C0100100D04001054010010A0010010D203001044010010980100100C04001074010010AC010010D5010010F1030010F2030010D40300104C010010A40100106A
:40C5C000D303001064010010A8010010D4010010EF0300108C010010B4010010D00100100104001002040010030400107C010010B801001084010010B001001040010010BE
:40C60000005C2605FD03001038010010300100102001001028010010DD01001058B1F84991F87B17012904D100EB4001F54A517201E0F44A5072704710B5044600BFF04851
:40C64000C0F83C43042200F54F71EF480068001DF9F716FC00BF10BD10B5EC48D0F854110220DFF8ACC300DFE848016D0220DFF8A0C300DFE24991F8C803F7F781FE6020AC
:40C68000EBF722FF10BD10B5FFF7E6FFDC4890F84F030A2801D10EF0B4FF10BDD84890F83803704710B50446FFF7F8FFA0420BD000BFD348C0F83843042200F54E71D24836
:40C6C0000068F9F7DDFB00BF10BDD24A1278D14B5A701A46107091707047F8B5C9484078382802D0CB2858D111E000210620FFF7ECFFC4480079032808D1CB20C149487047
:40C700006720EBF7E1FE2620EBF7DEFE46E0BC4890F87B07012803D11520FFF7C3FF02E01420FFF7BFFFB948D0F868111020DFF8E0C200DF0020B3494870FFF7A4FFFEF799
:40C74000EAFB0546FEF7E7FB07466DF077FAC4B2FEF751FA06462A462146FEF750FA2020F0F7E7FCF6F7ADF958B9F6F7A2F940B9F6F798F928B9F6F78DF910B9F6F782F94D
:40C7800050B1A54800680090A44802220321036840F276202BF08AFA00E000BF00BFF8BD38B5984840782338082853D2DFE800F004DCDC537E9ADCBA9948007880B9904867
:40C7C00090F87C0317280BD1FF2003460322002100902620EEF7C3FD01209149087039E088480079012808D0854890F87C0317280FD08448407901280BD18A480068102131
:40C8000002688048904701207E4948713120487020E07C480079022803D1794890F8830320B9774890F87C03172813D0022075494871FF200090724890F88313FF23032213
:40C840002620EEF78CFD00210220FFF73EFF26206C49487088E06B480079022819D12720684948700220487164F0DBF9012100202BF06BFB64F039FD044664F0DAFB64F06C
:40C8800059FD044664F0E9FB00210220FFF71DFF0BE05C480079012807D15A4948712320487000210846FFF710FF5DE064F0CFFC022807D12820534948700220487164F04E
:40C8C000B9F90EE04F48007901280AD14D49487164F0B6F926204B49487000210220FFF7F4FE41E064F0B3FC04280BD12A20454948700220487100210846FFF7E6FE64F041
:40C900009FF90EE03F48007901280AD13D49487164F096F926203B49487000210220FFF7D4FE21E03748007902280CD13D480068132102683348904702203249487100206B
:40C94000374908700FE02F48007901280BD100210220FFF7BAFE01202A49487164F070F926202849487000BF00BF38BD00202E4908707047014600202B4A1278012A04D0D3
:40C98000012902D1284A117007E0274A1278012A03D111B9244A11700120704770B50024F7F7C2F830B165F090FB0546FFF7E2FF044613E0F6F7F6FC50B165F08DFB08B18E
:40C9C000012000E000200546FFF7D4FF044605E065F043FB0546FFF7CDFF0446204670BD38B508484078362875D01FDC322826D0332863D034286FD035286ED1D5E00000F9
:40CA0000781A0010403E00108C0000100019002081F8080848020020DC030020D803002067020020580200206502002037287DD065287CD0D3287BD0E328DED12CE2FC48A3
:40CA40000079012808D0FB4890F87C0317280DD1F7484079012809D10120F54948712F20487000210846FFF730FE26E0F0480079022809D0EF4890F84F030A280ED0ED4818
:40CA800090F87C03172809D10220E94948713520487000210220FFF718FE0EE0E448007904280AD10220E24948713320487000210220FFF70AFE62F0FFFBFCE1DC4800793B
:40CAC00001280BD1DA4948713220487000210846FFF7FBFD2EE074E02DE0EBE1D448007902280ED1D2494871342048700021BFEE000A0C2062F01AFC00210520FFF7E5FDAB
:40CB000018E0F5F7CFFF20B1CA4890F84F030A2810D10220C649487138204870F9F700F8C548006813210268C14802E09CE028E197E19047BFE1BE48007904280FD1012073
:40CB4000BB4948713320487000210846FFF7BDFD00219FEDBA0A084662F0E8FB24E062F0D0FF03280DD10220B149487138204870F8F7D6FFB048006813210268AC4890473A
:40CB800012E062F0BEFF01280ED10220A8494871E320487000210520FFF797FD00219FEDA70A084662F0C2FB85E160F015FF60F068FFFFF7DBFE02209D494871362048703B
:40CBC00079E19B480079022802D0FFF7E7FEF8B160F0FDFE032803D060F0F9FE022802D160F04FFF05E060F0F2FE012801D160F0F3FEFFF7BBFE02208D49487160F028FF9C
:40CC000037208B49487000210720FFF75EFD2AE087480079012808D1854948713220487000210846FFF751FD1DE081480079042802D0F4F761FF70B17D48C07901280AD135
:40CC400002207B49C8717E48D0F868114020DFF8F4C100DF07E060F0BAFE042803D15FF086F8FFF783FE26E165F0F7F90446FFF781FE90B15FF07BF836206D494870084670
:40CC8000C079012804D100210520FFF71EFD77E000210220FFF719FD72E0F4F72DFF30B9694890F8D00010B9F6F749FBC0B1F5F708FF58B9F5F7FDFE40B9F5F7F3FE28B9D8
:40CCC000F5F7E8FE10B9F5F7DDFE48B1012058494871D320487000210520FFF7F6FC4FE060F075FE022803D060F071FE01280BD101204F494871D320487000210520FFF779
:40CD0000E4FC5FF034F83BE060F061FE032812D1022047494871652048700846C079012804D100210320FFF7D0FC29E000210846FFF7CBFC24E060F04AFE08BB43480078F6
:40CD400004281DD162F074F880B93620384948700846C079012804D100210520FFF7B5FC0BE000210220FFF7B0FC06E0D3203049487000210520FFF7A8FC01202C49487198
:40CD800099E02B480079022826D1F5F79AFE58B9F5F78FFE40B9F5F785FE28B9F5F77AFE10B9F5F76FFE50B1294800680090294803221146036840F276202AF077FF0220D4
:40CDC0001B4948711C480068132102681848904700210620FFF779FC1548C07901280ED11348007903280AD102201149C8711448D0F868114020DFF84CC000DF30E00C4873
:40CE0000007901282CD160F0E7FD60F03AFEFFF7ADFD012006494871362048700846C079012819D100210520FFF74FFC18E00000403E0010781A00105802002000000000FD
:40CE40000019002081F80808A81700105C020020DC030020D803002000210220FFF735FC29E0F7480079042815D1FFF77FFD0120F3494871362048700846C079012804D151
:40CE800000210520FFF721FC03E000210220FFF71CFC60F0A1FD0EE0E9480079042808D10120E74948713320487000210220FFF70CFC00E000BF00BF60F089FDE14908702E
:40CEC00038BD10B5DE4840782E2875D00CDC252878D004DC1F2814D024286FD12AE02C286DD02D28F9D1DFE0D52869D004DC2F2867D0D428F1D164E1D62877D0D728ECD1CA
:40CF00008FE1CF484079012808D1CD494871CE4800680E210268CA4890470AE0FFF726FD6AF03FF82420C649487000210220FFF7CCFB96E1C2480079022805D1002140F6F0
:40CF4000D83051F082F828B965F087F80446FFF711FDE0B10220BA494871F6F723FA40B9F6F7CAFD28B9F6F77CFA10B9F6F771FA18B12C20B249487002E02520B0494870C0
:40CF8000FFF7F4FC00210220FFF79FFB13E0AC480079012808D1AA4948711F20487000210846FFF792FB06E0A848007818B100210846FFF78AFB54E1B0E003E04EE126E0E3
:40CFC0000FE1DEE064F01AF808B1012000E000200446FFF7CFFC50B10220994948712C20487000210220FFF770FB0FE009E19448007901280AD192494871FFF7B7FC24201F
:40D000008F49487000210846FFF75FFB29E18C480079022810D100214FF43E6051F015F850B100BF0220864948712D20487000210220FFF74AFB36E081480079012818D198
:40D040007F494871F6F7AEF928B9F6F755FD10B9F6F707FA18B124207949487002E0252077494870FFF782FC00210846FFF72DFB19E067F044FF48B100210520FFF725FBB5
:40D08000D4206F494870012048710CE0704890F8500500F0020030B16E48D0F868110420DFF8B4C100DFDCE065480079022809D100BF634948712E20487000210220FFF74F
:40D0C00004FB2AE05E48007901280CD15C4948712C20487069F06EFF69F078FF00210220FFF7F3FA19E067F00AFF48B100210520FFF7EBFAD52052494870012048710CE063
:40D10000534890F8500500F0080030B15148D0F868110420DFF840C100DFA2E048480079022809D100BF464948712F20487000210846FFF7CAFA23E04148007901280CD118
:40D140003F4948712D20487069F040FF69F04AFF00210220FFF7B9FA12E067F0D0FE28B1D620374948700120487109E068F0DFF830B13848D0F868110420DFF8DCC000DF1B
:40D180006FE02F48007902280CD100BF2C4948713220487000205FF0ECFC00210846FFF794FA0DE026480079012809D1244948712E20487069F016FF00210220FFF785FABF
:40D1C0004FE01F48007904280AD169F00EFC01201B4948712C20487000210220FFF775FA3FE01748007904280AD169F0FEFB0120134948712D20487000210220FFF765FAA9
:40D200002FE00F48007904280AD169F0EEFB01200B4948712E20487000210220FFF755FA1FE007480079042808D10120044948711E20487000210220FFF747FA11E00000B6
:40D24000403E00105C0200205802002055020020781A00100019002081F80808FFF7C0FB00BF00BF10BD38B5FE4840782A287BD00BDCA0F11F000B2877D2DFE800F01B4B99
:40D28000767BA8E0FDFCFBFAF9002F286ED008DC2B286CD02C286BD02D286AD02E2864D1EEE2D4287DD0D5287CD0D6287BD0D728F5D163E3EB484079012803D0E948007915
:40D2C000012809D10120E7494871E74800680E210268E44890471CE064F016FBD52809D10220E04948712020487000210846FFF7ECF90EE064F008FBD6280AD0DB480068C8
:40D300000090DB4801220321036840F276202AF0CDFC44E3D3480079012808D0D54890F87C0317280DD0CF484079012809D10120CC4948711F20487000210846FFF7C5F905
:40D3400011E0C8480079022804D0CA4890F87C03172808D00220C34948712220487000210846FFF7B2F91AE3F7E115E3BAE2B0E10FE24CE2BB480079012808D0BD4890F8F1
:40D380007C03172810D0B748407901280CD10120B44948712020487000210846FFF795F914E0BBE2CAE2D9E2AE480079022804D0B04890F87C03172808D00220A949487107
:40D3C0002320487000210846FFF77FF9E7E2A5480079012808D0A74890F87C0317280DD0A0484079012809D101209E4948712220487000210846FFF768F91FE09948007995
:40D40000022804D09B4890F87C03172816D0FF200090984890F88313FF2303222620EDF79EFFFFF7A3FA69F0BCFD02208D4948712420487000210220FFF747F9AFE28948F7
:40D440000079022805D1002140F6D83050F0FDFD28B964F002FE0446FFF78CFA88B102208049487125204870FFF780FA002104E04CE1D1E087E05EE018E00220FFF725F99F
:40D4800013E078480079012808D1764948712320487000210846FFF718F906E07648007818B100210846FFF710F978E2714890F8830303280ED06F4890F88303062809D00C
:40D4C0006C4890F88303022804D06A4890F88303052809D10220634948712620487000210220FFF7F2F825E063F088FD08B1012000E000200446FFF73DFA60B102205949FA
:40D5000048712A20487000210846FFF7DEF82620EAF7DAFF0EE05348007901280AD151494871FFF723FA24204E49487000210846FFF7CBF833E24B480079022813D149490D
:40D5400048710021BFEE000A0B2061F0EFFE27204449487000210220FFF7B7F859F0A8FB464908600EE03F48007901280AD13D494871FFF7FBF924203A4948700021084651
:40D58000FFF7A3F80BE262F0B8FA02280CD1354948712820487000210220FFF796F859F087FB3649086036E062F0ABFA02280DD062F0A7FA012809D044F620612F4800688F
:40D5C00059F090FB90B162F09CFA78B90220254948712B20487000210846FFF776F800219FED270A084661F0A1FE14E01D480079012810D100219FED220A084661F096FEDA
:40D6000001201849487125204870FFF7AFF900210846FFF75AF8C2E162F073FA03280FD10220104948712A20487000210846FFF74CF800219FED120A084661F077FE47E00D
:40D6400062F05FFA02281ED062F05BFA01281AD044F620610948006859F044FB18B362F050FA0FE0403E001058020020DC030020D8030020781A001055020020600200203E
:40D680000000000078B90220FD4948712B20487000210846FFF719F800211FED070A084661F044FE14E0F6480079012810D100211FED0D0A084661F039FE0120F04948719E
:40D6C00025204870FFF752F900210846FEF7FDFF65E1EB480079012808D1E94948712620487000210220FEF7F0FF0EE0E448007902280AD1E2494871FFF738F92920E04973
:40D70000487000210220FEF7E0FF48E163F076FC08B1012000E000200446FFF72BF960B10220D74948712A20487000210846FEF7CCFF2620EAF7C8FE0EE0D148007901281B
:40D740000AD1CF494871FFF711F92520CC49487000210846FEF7B9FF21E1C9480079022808D1C74948712C20487000210220FEF7ACFF0DE0C2480079012809D1C04948715B
:40D7800025204870FFF7F2F800210846FEF79DFF05E1BB48007902280FD100214FF43E6050F053FC48B10220B54948712D20487000210220FEF789FF28E0B1480079012855
:40D7C0000AD1AF49487125204870FFF7CFF800210846FEF77AFF19E067F091FB48B100210520FEF772FFD420A5494870012048710CE0A44890F8500500F0020030B1A2489F
:40D80000D0F868110420DFF884C200DFC7E09C480079022808D19A4948712E20487000210220FEF752FF2AE09548007901280CD1934948712C20487069F0BCFB69F0C6FB2C
:40D8400000210220FEF741FF19E067F058FB48B100210520FEF739FFD52089494870012048710CE0874890F8500500F0080030B18548D0F868110420DFF810C200DF8EE02F
:40D880007F480079022808D17D4948712F20487000210846FEF719FF23E07948007901280CD1774948712D20487069F08FFB69F099FB00210220FEF708FF12E067F01FFBF0
:40D8C00028B1D6206E4948700120487109E067F02EFD30B16C48D0F868110420DFF8ACC100DF5CE066480079022808D1644948713220487000210846FEF7E7FE0DE06048D4
:40D900000079012809D15E4948712E20487069F069FB00210220FEF7D8FE40E05848007904280AD169F061F80120554948712C20487000210220FEF7C8FE30E050480079AD
:40D9400004280AD169F051F801204D4948712D20487000210220FEF7B8FE20E04848007904280AD169F041F80120454948712E20487000210220FEF7A8FE10E040480079BC
:40D98000042808D101203E4948711E20487000210220FEF79AFE02E0FFF722F800BF00BF38BD38B536484078372873D014DC2E2871D008DC1F2822D0212837D02C286FD08A
:40D9C0002D286AD1ACE0302868D0312867D035287AD03628F5D162E1D52876D008DC642874D0652873D0D32872D0D428E9D1E3E1D6286ED0D7286DD0D828E2D11EE22048CC
:40DA00004079012808D11E494871214800680E2102681B48904708E069F0C3FA21201849487000210846FEF750FE67E214480079012808D0134890F87C0317280DD0104868
:40DA40004079012809D101200D4948711F20487000210846FEF739FE11E009480079022804D0084890F87C03172808D00220044948712C20487000210846FEF726FE3DE22E
:40DA8000403E0010781A00100019002081F80808580200202EE17CE002E02EE2AFE0CFE0FE480079022816D100214FF43E6050F0CCFA80B10220F94948712D204870002113
:40DAC0000846FEF702FE2AE0DFE085E165E14AE164E191E1A0E1F1480079012808D1EF4948712120487000210846FEF7EEFD16E067F005FA48B100210520FEF7E6FDD420C7
:40DB0000E64948700120487109E0E54890F8500500F0020018B100210846FEF7D6FDEDE1DE48007902280FD1002140F6E13050F08CFA48B10220D94948712E20487000217D
:40DB40000846FEF7C2FD23E0D4480079012808D1D24948712C20487000210846FEF7B5FD16E067F0CCF948B100210520FEF7ADFDD520CA4948700120487109E0C84890F810
:40DB8000500500F0080018B100210846FEF79DFDB4E1C248007902280FD1002140F6E23050F053FA48B13020BC4948700220487100210846FEF789FD20E0B84800790128CC
:40DBC00008D1B64948712D20487000210846FEF77CFD13E067F093F948B100210520FEF774FDD620AD4948700120487106E067F09EFB18B100210846FEF767FD7EE1A74804
:40DC0000007902280FD1002140F6D26050F01DFA48B13120A14948700220487100210846FEF753FD0BE09D480079012807D19B4948712E20487000210846FEF746FD5DE134
:40DC400096480079022813D1002140F6A15050F0FCF968B193480068112102688F48904702208E49487100210846FEF72EFD0BE08A480079012807D1884948713020487012
:40DC800000210846FEF721FD38E15FF0A5FE5FF0F8FE022081494871362048702EE17F48007902280BD17D4948715FF0D1FE37207A49487000210720FEF707FD19E0774822
:40DCC0000079012808D1754948712F20487000210220FEF7FAFC0CE070480079042808D102206E4948713820487000210620FEF7ECFC03E15FF06BFE022803D05FF067FEC8
:40DD0000012809D1012065494871D320487000210520FEF7DAFC25E05FF059FE032809D102205E4948716520487000210846FEF7CCFC17E05FF04BFEA0B961F079F838B966
:40DD400036205649487000210220FEF7BEFC06E0D3205249487000210520FEF7B6FC01204E494871CAE04D480079022808D14B4948713820487000210620FEF7A6FC0BE099
:40DD800046480079012807D1444948713520487000210220FEF799FCB0E0AFE03F480079042808D101203D4948713620487000210220FEF78AFCA1E03848007904280AD16A
:40DDC00068F013FE0120354948712C20487000210220FEF77AFC91E03048007904280AD168F003FE01202D4948712D20487000210220FEF76AFC81E02848007904280AD1AA
:40DE000068F0F3FD0120254948712E20487000210220FEF75AFC71E02048007904280CD1204800680E2102681C48904701201B49487100210220FEF748FC5FE0FF20009037
:40DE4000174890F8E02400F5737000EB4202144890F8E104115CFF2303221A20EDF77FFAFF2000900E4890F8E02400F5747000EB42020B4890F8E104115CFF2303221B2054
:40DE8000EDF76DFAFF200090054890F8E02400F5757000EB4202024806E00000403E0010781A00105802002090F8E104115CFF2303221C20EDF753FA67F09DFE0446FF20C3
:40DEC00003460322214600901046EDF748FA67F0FEFA0446FF2003460322214600900420EDF73DFAFE48006811210268FD48904700210620FEF7E9FB00E000BF00BF38BD0C
:40DF000038B5F848407829287ED00ADCA0F11F000A287AD2DFE800F01C844CB2DCF7F6F5F4F32F2872D00ADCA0F12A000528F0D2DFE810F091024D02AD02EB022403D428BE
:40DF40007ED0D5287DD0D6287CD0D7285DD193E3E4484079012803D0E2480079012809D10120E0494871DE4800680E210268DD4890471CE063F0C8FCD52809D10220D94941
:40DF800048712120487000210846FEF79EFB0EE063F0BAFCD6280AD0D34800680090D34801220321036840F2762029F07FFE74E3CC48007901280DD0CD4890F87C03172860
:40DFC00004D1CB4890F8840301280DD1C5484079012809D10120C34948711F20487000210846FEF772FB1AE0BE480079022809D0BF4890F87C03172804D1BD4890F88403FA
:40E0000001280CD1022002E0FEE143E3E8E2B54948712020487000210846FEF756FB3CE3B0480079012808D0B14890F87C03172811D0AC48407901280DD10120A94902E049
:40E04000EAE2F9E208E348712120487000210846FEF73BFB11E0A3480079022804D0A44890F87C03172808D002209E4948712220487000210846FEF728FB0EE399480079D7
:40E08000012808D09A4890F87C0317280DD095484079012809D10120924948712020487000210846FEF711FB11E08E480079022804D08F4890F87C03172808D0022089497D
:40E0C00048712320487000210846FEF7FEFAE4E284480079012808D0854890F87C03172812D08048407901280ED101207D4948712220487000210846FEF7E7FA24E01AE1A8
:40E10000C1E098E052E020E076480079022804D0774890F87C03172816D0FF200090744890F88313FF2303222620EDF718F9FEF71DFC68F036FF02206A4948712420487044
:40E1400000210220FEF7C1FAA7E266480079022805D1002140F6D8304FF077FF28B963F07CFF0446FEF706FC58B102205D49487125204870FEF7FAFB00210220FEF7A5FAB0
:40E1800013E058480079012808D1564948712320487000210846FEF798FA06E05548007818B100210846FEF790FA76E2504890F8830303280ED04E4890F88303062809D0A4
:40E1C0004B4890F88303022804D0494890F88303052809D10220434948712620487000210220FEF772FA25E062F008FF08B1012000E000200446FEF7BDFB60B102203949ED
:40E2000048712A20487000210846FEF75EFA2620EAF75AF90EE03348007901280AD131494871FEF7A3FB24202E49487000210846FEF74BFA31E22B480079022813D12949A6
:40E2400048710021BFEE000A0B2061F06FF827202449487000210220FEF737FA58F028FD254908600EE01F48007901280AD11D494871FEF77BFB24201A49487000210846E8
:40E28000FEF723FA09E261F038FC02280CD1154948712820487000210220FEF716FA58F007FD1549086045E061F02BFC02280DD061F027FC012809D044F620610E480068D1
:40E2C00058F010FD08B361F01CFCF0B90220054948712B20487000210846FEF7F6F90DE058020020403E0010DC030020D8030020781A0010550200206002002000219FED46
:40E30000F70A084661F012F814E0F5480079012810D100219FEDF10A084661F007F80120EF49487125204870FEF720FB00210846FEF7CBF9B1E161F0E4FB03280FD1022003
:40E34000E74948712A20487000210846FEF7BDF900219FEDE20A084660F0E8FF36E061F0D0FB02280DD061F0CCFB012809D044F62061DC48006858F0B5FC90B161F0C1FB99
:40E3800078B90220D64948712B20487000210846FEF79BF900219FEDD10A084660F0C6FF14E0CF480079012810D100219FEDCB0A084660F0BBFF0120C949487125204870FB
:40E3C000FEF7D4FA00210846FEF77FF965E1C4480079012808D1C24948712620487000210220FEF772F90EE0BD48007902280AD1BB494871FEF7BAFA2920B9494870002151
:40E400000220FEF762F948E162F0F8FD08B1012000E000200446FEF7ADFA60B10220B04948712A20487000210846FEF74EF92620EAF74AF80EE0AA48007901280AD1A849F1
